:1000000000800020BD01000069E8000021E8000038
:1000100021E8000021E8000021E8000021E80000BC
:1000200021E8000021E8000021E8000069E8000064
:1000300069E8000021E8000061120100651201007A
:1000400069E8000069E8000069E8000069E800006C
:1000500069E8000069E8000069E8000069E800005C
:1000600069E8000069E8000069E8000069E800004C
:1000700069E8000069E8000069E8000069E800003C
:1000800069E8000069E8000069E8000069E800002C
:1000900069E8000069E8000069E8000069E800001C
:1000A000F9BE000005BF000069E8000069E8000033
:1000B00069E8000069E8000069E8000069E80000FC
:1000C00069E8000069E8000069E8000069E80000EC
:1000D00069E8000069E8000069E8000069E80000DC
:1000E00069E8000069E8000069E8000069E80000CC
:1000F00069E8000069E8000069E80000B1F6000066
:1001000069E8000035FC000069E8000069E80000CB
:1001100069E8000069E8000069E8000069E800009B
:1001200069E8000069E8000069E8000069E800008B
:1001300069E8000069E8000069E8000069E800007B
:1001400069E8000069E8000069E8000069E800006B
:100150001116010025160100391601004D16010087
:1001600069E8000051FF000069E8000069E800004C
:1001700069E8000069E8000069E8000069E800003B
:1001800069E8000069E8000069E8000069E800002B
:1001900069E8000069E8000069E8000069E800001B
:1001A00069E8000069E8000069E8000069E800000B
:1001B00069E8000069E8000069E80000564B4CF26D
:1001C000205210B51A804DF628121A8000BF00BFC9
:1001D0000EF04EFB514B4FF010621A60504A9A607D
:1001E000504ADA60504A136813F4807304D14F49BF
:1001F0000B604FF4A85313604D4B1A78110703D5C9
:100200001A7842F008021A704A4B4B492A221A7097
:100210004A4A4B4B8B4204D252F8040F43F8040B6A
:10022000F8E7484B484900228B4202D243F8042B9E
:10023000FAE74649464A002352F8230041F82300D2
:1002400001336F2BF8D1434B434A802103F8011B44
:100250009342FBD1414B3D4A1A60414B8A221A70AE
:10026000A3F5805324225A70A0221A709A7992071B
:10027000FCD59A79D406FCD43A4A937903F00C035E
:10028000082B384BF9D103221A7140225A719A79FE
:100290009006FCD5334A9179324B4906FBD5324A58
:1002A000324911600221516020221A709A7902F0BD
:1002B0000C020C2AFAD12E4B2E4A1A602E4B2F4AD2
:1002C0001A6000225A60072243F8042C2C4AC3F813
:1002D0000C2D62B60EF056FE144B1B68DA0705D5DE
:1002E00028480EF023FC284B284A1A60284B1B781C
:1002F0005B0609D5244C254B22689A4204D121483B
:100300000EF014FC0023236012F00EFD0EF0B6FA7E
:1003100011F014FAFEE700BF0E20054030800440C3
:10032000823F04000100002B10D0034014D0034092
:1003300002D0074000E00740249DFF1F7C6B0100B6
:100340004088FF1F249DFF1FF4A4FF1F0082FF1F92
:100350000000000000E400E05FE400E008ED00E0E1
:100360000050064000400640448004400000030165
:1003700004800440C010050014E000E0FF76010096
:10038000000020207B227E631CE00340A5C3945A1A
:1003900000F00740FFFFFFFFFFFFFFFFFFFFFFFF32
:1003A000FFFFFFFFFFFFFFFFFFFFFFFFFFFFFFFF5D
:1003B000FFFFFFFFFFFFFFFFFFFFFFFFFFFFFFFF4D
:1003C000FFFFFFFFFFFFFFFFFFFFFFFFFFFFFFFF3D
:1003D000FFFFFFFFFFFFFFFFFFFFFFFFFFFFFFFF2D
:1003E000FFFFFFFFFFFFFFFFFFFFFFFFFFFFFFFF1D
:1003F000FFFFFFFFFFFFFFFFFFFFFFFFFFFFFFFF0D
:10040000FFFFFFFFFFFFFFFFFFFFFFFFDEF9FFFF23
:1004100010B5054C237833B9044B13B10448AFF33E
:1004200000800123237010BD249DFF1F00000000E9
:10043000786B0100084B10B51BB108490848AFF3B1
:1004400000800848036803B910BD074B002BFBD0A0
:10045000BDE81040184700BF00000000289DFF1FA6
:10046000786B0100249DFF1F0000000038B5044692
:10047000104621700A491D4612F03EFA01464FF01F
:100480007E5012F0EDFA074912F036FAE56060602E
:10049000256165610EF006FDE061204638BD00BFB4
:1004A000DB0FC9400024744938B50446104621705A
:1004B00009491D4612F020FA01464FF07E5012F015
:1004C000CFFA064912F018FAE560606025616561AF
:1004D0000EF0E8FCE06138BDDB0FC9400024744930
:1004E00038B503780446032B20D8DFE803F01A1848
:1004F0001002C168406912F0F5F80D4905466068C0
:1005000012F0AEFA0146284612F0AAFA38BD0849A0
:10051000406812F0A5FAE16812F0EEF938BDC06843
:1005200038BDC168406912F0DDF838BD002038BD23
:100530000024744970B504460E460EF0B3FC05461F
:10054000E069281A12F084F9E3682361E5616661C5
:10055000A0610146606812F083FA0146A06010486D
:1005600012F07EFA11F054FD11F0EEF912F066F877
:10057000054601464FF07E5012F0B4F8616912F062
:10058000BBF921690646284612F0B6F90146304605
:1005900012F0AAF8E0602046BDE87040FFF7A0BF67
:1005A000000080BF38B50E201C4C0EF013F82188D7
:1005B0001B4B884205461A881DDA0023511AB1F5F3
:1005C000805FAABF1B03C3EB03330131142093FBED
:1005D000F1F10EF0BDFA134B1988F1B923889D4251
:1005E00010DAC3F57F630F33282091FBF3F1BDE8E8
:1005F00038400EF0ADBA9042D4BFC1EB0003C1EB5E
:100600000203DBE740F6FF718D42D4BFC3EB050167
:10061000C3EB0101C1EB0131E3E738BD389EFF1F99
:100620005C9DFF1FA09FFF1F10B5044610F0CEFF7A
:10063000204610BD70B44C88A04220D9012301335C
:10064000DBB21CB2660031F8144084421D46F6D37A
:10065000A04211D005F10045013D965B31F815101F
:1006600032F81530401AF21A00FB02F0641A90FBBF
:10067000F4F4E01870BC7047905B70BC70470226C1
:100680000125E5E700280CDA064A434282FB0320F5
:10069000DA17C2EB600000EB4000A3EB8000C0F172
:1006A0000C007047ABAAAA2A38B5234B1B78002B45
:1006B0002CD015200DF08EFF204B1860204B1B888E
:1006C000984203DA1F4C237863BB38BD1E4A148856
:1006D000A042A4EB0302A8BF20467F2A1CDDC01A5B
:1006E000C001541C90FBF4F4002CEBD0154B1A788D
:1006F0000AB901221A70154D2B689C4204D0144B84
:10070000E1B2187809F084FC2C6038BD11200FF09C
:10071000FDFA0A4B1860D1E7C01AC0EBC01090FB7D
:10072000F2F4E1E70A4B0021187809F071FC00238C
:10073000064A2370136038BD549FFF1F549DFF1F4E
:10074000DC9DFF1F30A0FF1FCC9FFF1F28A0FF1FB5
:10075000B09DFF1F38B50F200FF0D8FA1B4A1C4B75
:1007600012881860C0F53B600830904220DB194BBE
:100770001B889842A3EB0204A8BF1846801A7F2C5E
:10078000C6BFC0010134C0EBC01090FBF4F47CB1D3
:10079000114B1A780AB901221A70104D2B689C422D
:1007A00004D00F4BE1B2187809F032FC2C6038BD50
:1007B000094C237803B938BD094B0021187809F09A
:1007C00027FC0023054A2370136038BD3C9EFF1FA1
:1007D000709DFF1FB89FFF1FDC9FFF1FEC9DFF1F39
:1007E000D29DFF1FF0B40E8886420DD203F1004364
:1007F000013B31F81350854202D9F0BCFFF71ABF14
:1008000032F81300F0BC70471088F0BC704700BF8E
:10081000094B1B880C2B09D8084A80B252F82320B8
:1008200028B143F6FE73984203D9108C70471088A4
:1008300070470349FFF7FEBE869DFF1F644301001A
:10084000004501004B4B4C4A2DE9F0471E881468C7
:100850004A4BB442B3F80080494B33DB4445A8BF50
:100860004446A6421C60C8BF00202DDDC6EB080729
:10087000B7F5804F33DB80037B1C90FBF3F0FFF771
:10088000C7FF404A404B15881B88C0F3C61909FBB7
:1008900005F57F2D8246A8BF7F252BB3A64253DCEA
:1008A0004445D4BFC6EB0404C6EB08049F42CCBF4A
:1008B00003FB04445C43354BC8BF013794FBF7F797
:1008C0001F6013E034461E60C6EB0807A045D4BF86
:1008D000C6EB0800C6EB0400B7F5804FCBDAC0EBDF
:1008E000803090FBF7F0CAE7284A1360284C236851
:1008F000994508D0274B1B88002B34D1264B1B88E9
:100900006BBBC4F80090254C23689A4506D0214B58
:100910001B885A1F032A19D9C4F800A0204C236849
:100920009D420FD01F4B188848B11A4B1E4A1B8896
:10093000D35C834203D0C0B2E9B209F069FB256001
:10094000BDE8F087BDE8F0870024AFE7164AD05C29
:100950002030C0B20AF07F0109F05AFBDCE74846BC
:1009600009F0F6FBCDE7104A4946D05C09F050FB90
:10097000C4E700BF389EFF1F9C9FFF1F5C9DFF1FA9
:10098000489DFF1F5E9DFF1F609DFF1F04A0FF1F6E
:10099000CC9DFF1F849FFF1F2A9EFF1F809DFF1F6E
:1009A0002C9EFF1F929FFF1F288AFF1F2DE9F04FEB
:1009B00001208BB00FF0AAF9DFF850B3CBF800009C
:1009C00000200FF0A3F9B34BB34A1B8810600C2B27
:1009D00000F00582B14A00211F2B117037D0B04FB3
:1009E000B04B3A88B04E53F8225000233370AF4BCF
:1009F000AF4A1B88AF491288013B012A31F91330F5
:100A0000059300F00682AC4B0193AC4B0293DFF8E8
:100A10000083DFF8009300230093A94B1B88012B70
:100A200000F04D82DFF8F0A2A64B0393DAF8004005
:100A3000A54B04930023A54A1288013A032A00F229
:100A40008682DFE812F00101DC0011007101A04B89
:100A5000934F1B783988934A934E52F821500033B4
:100A600018BF01233370C2E72046059311F0F0FE52
:100A7000984911F041FF059B0446184611F0E8FE25
:100A8000954911F039FF0146204611F02DFE12F074
:100A9000F9F80446CAF80040D8F8000011F0D8FE72
:100AA0008C4911F029FF8246009811F0D1FE8A4945
:100AB00011F022FF0146504611F016FE12F0E2F846
:100AC000C8F80000854A864BB2F800E01988854BCB
:100AD000DBF800201B88DFF844C2CEEB040804EBEF
:100AE0000E0AC1EB000E08440499039CC1F800A053
:100AF0000199C4F80080C1F800E002999A420860A8
:100B0000BCF8001080F25281C3EB010C62486545CD
:100B10004FF0000E006880F256816C1C83420CF18D
:100B2000010C0EFB04FE9EFBFCFE00F3928381424F
:100B3000A8BF0146C91A04FB01F191FBFCF19A42DE
:100B400000F317818342C0F21481DFF8D4A1DAF8F0
:100B5000000011F07DFE644911F0CEFE634911F0F2
:100B6000C3FD12F08FF8A0F5FF531C3B082B98BF74
:100B70004FF40050D9F80040DFF8A881044443F650
:100B8000FF77BC42A8BF3C4624EAE4742046CAF87A
:100B9000004011F05DFE8146307805FB00F011F059
:100BA00057FE4FF07A5111F0A7FE0146484611F06A
:100BB00099FD12F067F84E4BB842A8BF38461B7833
:100BC00020EAE070C8F80000002B00F0E380B4F5E4
:100BD000005F00F0DF8006F0C5F9464BD8F8000052
:100BE00001221A70444C2368834205D080B209F078
:100BF000DFF9D8F8003023600BB0BDE8F08F204655
:100C0000059311F025FE3D4911F076FE059B044643
:100C1000184611F01DFE3A4911F06EFE01462046BD
:100C200011F062FD12F02EF80446CAF80040D8F820
:100C3000000011F00DFE314911F05EFE8246009871
:100C400011F006FE2E4933E72046059311F000FE11
:100C50002C4911F051FE059B0446184611F0F8FD91
:100C6000294911F049FE0146204611F03DFD12F0E0
:100C700009F80446CAF80040D8F8000011F0E8FD71
:100C8000204911F039FE8246009811F0E1FD1E491D
:100C90000EE700BFCE9FFF1F7C9DFF1F4E9DFF1FD5
:100CA000C09DFF1FE489FF1FB29FFF1F3689FF1FF2
:100CB000A29FFF1F9C4801002CA0FF1FFC9DFF1F4F
:100CC000349FFF1FC09FFF1F389FFF1F7889FF1FA2
:100CD0006C9DFF1FCDCC4C3FCDCC4C3E348AFF1FCA
:100CE0007089FF1F989FFF1F9A99193FCDCC4C45E3
:100CF000F2A0FF1F289EFF1F3889FF1F6666663F10
:100D0000CDCCCC3D3333733FCDCC4C3DB89DFF1F94
:100D1000409DFF1FD89FFF1FBC9FFF1F9C9DFF1F73
:100D20001C8AFF1F7489FF1F2046059311F090FD58
:100D3000C54911F0E1FD059B0446184611F088FDF8
:100D4000C24911F0D9FD0146204611F0CDFC11F049
:100D500099FF0446CAF80040D8F8000011F078FD69
:100D6000B94911F0C9FD8246009811F071FDB749EB
:100D70009EE63B88002B3FF4E8AEC1EB0E03002B50
:100D8000B8BF5B42092B00F3E5804FF40050DFF859
:100D900008A3EFE6AE4C2378002B3FF423AF06F018
:100DA000DDF80023D8F8000023701BE7C3EB010C2B
:100DB000A8488A42D4BFC3EB020EC3EB010E6545BF
:100DC0000068FFF6AAAE83420EFB05FEC8BF0024F2
:100DD0009EFBFCFE40F3348294FBFCF1AFE69E4B9D
:100DE0001B78002B00F0D5809C4F9D4B39889D4A85
:100DF00053F821009C4E012100231170337011F033
:100E000027FD4FF07C5111F077FD11F03BFF0546B7
:100E1000EDE5964B964A1B8896491278013B31F9CD
:100E20001340002A40F0B08011200EF06FFF0090B8
:100E3000914B0193D3F80090009B994540F3AC800F
:100E40008E4BDFF858821B888D4A012BD8F8003072
:100E5000B2F800A08B4A02922846A3EB040400F0EB
:100E6000CE8011F0F5FC029A52F82A1011F044FDE0
:100E70000146002011F036FC11F004FF009BC9EB85
:100E800004029C42B8BF1C469042C9EB040480F2A5
:100E9000CA8000FB0444013294FBF2F47A4BDFF881
:100EA00000920293D9F80030234403EBD3735B1014
:100EB000C9F80030754B1B88012B7FF4B3AD744B20
:100EC00003931C460F200EF021FF226804929042EB
:100ED000034680F2E980694A1288012A00F02E81D7
:100EE000674A07901288674C0692284611F0B0FCBA
:100EF000069ADFF8B0A154F82210DAF8004011F099
:100F0000FBFC0146002011F0EDFB059BE21A059267
:100F100011F0B8FE059A079B04999A42C1EB020EA4
:100F2000B8BF1A46704580F23381521A00FB022284
:100F30000EF1010192FBF1F2D9F80010554804902E
:100F40000A4402EBD2725210C9F8002073E5D8F8B7
:100F50000000B7E50EF500500130401A11F078FCA2
:100F60003A49DFF834A111F0C7FC0446DAF8000072
:100F700011F06EFC344911F0BFFC0146204611F01F
:100F8000B3FB11F07FFEF5E515200DF023FB00907B
:100F90004EE7344A137022E53B4B0293D3F800909E
:100FA000009B994544DA354BDFF8F0801B88344AC2
:100FB000012BD8F80030B2F800A0324A039228463C
:100FC0001C4400F0EC8011F043FC039A52F82A1004
:100FD00011F092FC11F056FE009B9C42C9EB0402FA
:100FE000A8BF1C46C9EB04049042BABF00FB0444EE
:100FF0000132444394FBF2F4DFF8A49052E711F07D
:1010000027FC029A52F82A1011F076FC11F03AFEF1
:10101000009BC9EB04029C42B8BF1C468242C9EB4C
:1010200004043FF736AF00FB04F494FBF2F435E719
:10103000DFF86C90DFF86480D9F8003003EBD373ED
:101040005B10C9F80030E8E49A99193FCDCCCC3E4A
:10105000289EFF1F7C9DFF1F6C9DFF1FC09DFF1FD3
:10106000E489FF1F4E9DFF1FB29FFF1F808AFF1F55
:10107000549FFF1FB84401002CA0FF1F0E9EFF1FAE
:10108000A49DFF1FB4480100FC9DFF1F349FFF1F5C
:10109000C09FFF1F389FFF1F1C8AFF1F409DFF1F1F
:1010A000D89FFF1FBC9FFF1F6B4A049212680692D5
:1010B000904237DD694A1288012A00F08E80684A22
:1010C00009901188674A08912846079211F0C0FBE1
:1010D000079A0899DFF890A152F82110DAF8004039
:1010E00011F00AFC059B2344059311F0CBFD0599F3
:1010F000099B069A9942C2EB010EA8BF194670459A
:1011000080F29080891A00FB01110EF1010291FB1F
:10111000F2F2D9F800100A4402EBD2725210C9F868
:10112000002088E4D9F80020DFF83CA102EBD2725D
:101130005210DAF80040C9F800207CE4484A0890D0
:101140001188484A07912846069211F081FB069AB9
:101150000799DFF814A152F82110DAF8004011F0D5
:10116000CBFB059BE11A059111F08CFD0599089BBD
:10117000049A9942C2EB010EB8BF1946704558DA7D
:10118000891A00FB01110EF1010291FBF2F2D3E684
:101190000499521A00FB02F292FBFEF2CCE611F027
:1011A00057FB039A52F82A1011F0A6FB01460020C3
:1011B00011F098FA11F066FD009A9442C9EB04030D
:1011C000A8BF1446C9EB04049842BABF00FB04440C
:1011D0000133444394FBF3F40EE72149214A08907C
:1011E00028460C88079211F033FB079ADFF878A0A5
:1011F00052F82410DAF8004011F07EFB014600207E
:1012000011F070FA059B2344059311F03BFD0599FD
:10121000089B069A9942C2EB010EA8BF1946704579
:10122000FFF670AF069A891A00FB01F191FBFEF2FE
:101230006FE7049A891A00FB01F191FBFEF27BE64D
:101240008842D4BFC3EB0004C3EB010405FB04F4E4
:10125000C2E519466EE400BF389FFF1F0E9EFF1FB8
:10126000A49DFF1FB4480100BC9FFF1F08B5244B7D
:101270001B88FBB1234B1B78FBB1234B1B78E3B1DD
:10128000224B1B78CBB1224B1B78B3B1214B2248A8
:101290001A78C2B9214A2249008812880968024492
:1012A000B1EB620F09DD01221A706420BDE808402D
:1012B00005F06CBE174A117801B908BD1370BDE87E
:1012C000084008F019BF154A1649008812880968B5
:1012D0000244B1EB620FF0DD00221A7008F00CFF3F
:1012E000642005F053FE642005F050FE642005F0F4
:1012F0004DFE4FF41670BDE808400DF0F5BD00BF7F
:10130000469FFF1FFD9FFF1FFE9FFF1FFF9FFF1FA9
:1013100000A0FF1F849DFF1F9C9DFF1F989FFF1F24
:10132000B89DFF1F7C9DFF1F38B5114C23202578E9
:101330000DF050F90F4A42F82500131F02F1C400C6
:10134000002253F8041F83420A44FAD123780A4941
:1013500007480A4C0133DBB2322B81FB025108BF34
:101360000023D217C2EB21120370226038BD00BFE8
:10137000629DFF1F489EFF1F1F85EB51949FFF1F1B
:101380002DE9F04FB74DB84E2868B84C83B011F036
:101390005FFAB74911F0B0FA074610200EF0B6FC1C
:1013A00011F056FAB34911F0A7FA394611F09CF939
:1013B00011F068FC31882860884223887EDA1F4655
:1013C00000225B1ADFF8D482DFF8D4E27F2BCABF99
:1013D000D201C2EBC212013392FBF3F3B8F8002042
:1013E000CEF80030192A00F0DF801A2A00F02B8195
:1013F0001E2A00F05B814FF00108C1469E4B1B88FE
:10140000002B66D09D4A1288032A00F20981884287
:10141000C0F25F81B842D4BFC1EB0000C1EB07004E
:10142000791A8B42B4BF03FB00005843944F954B8D
:10143000B8BF013190FBF1F01860388800284FD018
:101440003188D5F800E0884ADFF818A2714500F32A
:101450008280DFF83CC29CF80030002B4CD14FF06A
:10146000010B04288CF800B046D1B8F1000F40F011
:10147000CB81854B1888F0B1B9F1000F1BD02B68D8
:10148000318822888B4280F29C810023541A7E2C62
:101490007E4DD5BFC3EB8313C3EBC3135B00013495
:1014A00093FBF4F42B680134A34203D0C0B2E1B241
:1014B00008F0AEFD2C6003B0BDE8F08F9842D4BFB9
:1014C000C1EB0002C1EB03021F467AE799464FF0D9
:1014D00001081E2A00F0D281694F38880028AFD158
:1014E000694B1B88002BABD1694A11780029E2D0E7
:1014F000137003B0BDE8F08F012800F012810228BC
:1015000000F003810328B4D1624B1B88092BB0D0B3
:10151000B8F1000FADD02B6837882288BB4280F22B
:1015200095810023D71B7E2FDFF86CB1D5BFC3EBAD
:101530008313C3EBC3135B00013793FBF7F7DBF8AF
:1015400000300137BB4203D0F9B24A2008F060FDF9
:10155000CBF800708DE74E4B1A78002AABD00024F0
:1015600001281C7000F0C280022840F03181B8F1DF
:10157000000F00F0C280484D2B68002B00F0BD80AA
:101580000420214608F044FD3F4B2C6018880028B9
:1015900091D0B9F1000F8ED0C0B2002108F038FD13
:1015A0003A4B00221A6086E7DFF8F8A0DFF8F890DF
:1015B0009AF80030BBB1DFF8D0E0BEF800E0BEF131
:1015C000000F10D099F800C09C4500F099805FFA98
:1015D0008EF07F2108F01CFD9AF80030B8F800204A
:1015E00089F800300FE099F800E09E4500F088800F
:1015F000254B0021187808F00BFD9AF80030B8F858
:10160000002089F800301C4B1B88002B3FF45EAF94
:101610001E2A40F02B814FF001084FF0000951E0E5
:10162000884258DBB842A1EB0701A8BF38468B427D
:10163000A0EB070055DA03FB00004B1C90FBF3F313
:10164000104A136048E7DFF85CA09AF80030002BDE
:101650000BBF4FF001084FF000084FF000094FF0AA
:101660000109CBE6AC9DFF1F4C9FFF1F489FFF1F4A
:101670009A99193FCDCCCC3E08A0FF1FC49FFF1FF5
:10168000B49DFF1F409EFF1FE09FFF1F909DFF1F07
:10169000D39FFF1F849FFF1F449EFF1FCE9FFF1FEE
:1016A000B49FFF1F6C9DFF1F689DFF1FDFF8E8A11F
:1016B000744B9AF800801B88B8FA88F84FEA5818DB
:1016C0004FF000099AF8002042B328683188278833
:1016D00098E60020A4E60846C91B8B42A0EB070051
:1016E000A9DB03FB00F393FBF1F3A9E7B8F1000FCB
:1016F00003D0654D2B68002B7FD1644B188846E7DB
:101700004FF001084FF0000978E6B8F1000F3FF400
:10171000B0AEDFF874B1DBF8003030E05C4B1A603B
:10172000DAE6B8F1000F3FF4A4AEB4F800A0F24539
:10173000D4BFC1EB0A03C1EB0E03C1EB0A0ABAF135
:101740007E0FDFF844B1D5BFC3EB8313C3EBC313E4
:101750005B000AF1010A93FBFAFADBF800300AF1A8
:10176000010A534504D05FFA8AF1012008F050FCC9
:101770003888CBF800A002287FF4C4AE53462A680C
:10178000B6F800A02188524559DA0022CAEB010AB6
:10179000BAF17E0FD3BFC2EB8212C2EBC2120AF1C2
:1017A000010A520092FBFAFA0AF1010A9A4504D0A2
:1017B0005FFA8AF1042008F02BFC3888CBF800A0EF
:1017C000A0E69342D4BFC1EB0303C1EB02035DE685
:1017D000032828D12F4B1B88092B8ED0B8F1000F7E
:1017E0008BD0294D2B68002B87D04A20214608F04A
:1017F0000FFC264B2C601888C9E6214608F008FC2F
:10180000224B2C601888C2E640207F218DE80C0016
:1018100008F0FEFB388858459DE80C001DD00228D2
:101820007FF470AE75E704287FF467AFB8F1000F5E
:101830003FF463AF2146402008F0EAFB5DE78A42AF
:10184000D4BFCAEB0202CAEB01029FE79342D4BFA6
:10185000C7EB0303C7EB020364E6DAF800E0118884
:10186000B4F800A08E45FFF668AF60E728683188BD
:1018700027884FF001084FF00009C3E50023DFF887
:1018800018A01FE708A0FF1F449EFF1FE09FFF1F37
:10189000409EFF1F849FFF1F6C9DFF1F08B5114BCB
:1018A0001B88022B09D0052B07D0032B15D0042B46
:1018B0000BD00D4B01221A7008BD7F21412008F08A
:1018C000A7FB094B01221A7008BD7F21092008F0EF
:1018D0009FFB054B01221A7008BD4021092008F02A
:1018E00097FBE6E73E9EFF1FE19DFF1F38B5074BC4
:1018F000074D1B88052B044606D02B68834203D076
:10190000C1B2052008F084FB2C6038BD3E9EFF1F4D
:10191000E89FFF1F38B5124D124C2B88052B12D0B3
:1019200022684AB9022B0ED0033B012B13D90E4A71
:1019300000231370236038BD0021052008F068FBE8
:101940002B88022B04D10021412008F061FBEEE737
:10195000052BE9D1F7E70021092008F059FBE6E75C
:101960003E9EFF1FE89FFF1FE19DFF1F464B1B8808
:101970001D2B70B541D0454D0024454B1B88022BD3
:1019800016D0444B1B88022B54D02888424B002C85
:101990001B780ADB8442A8BF044634B1002B3AD03E
:1019A0002046BDE87040FFF7A1BF002B2FD170BDCE
:1019B0003A4B1B78002B37D015200CF00BFE384B20
:1019C0001860384A1288002ADBD0374A1868118814
:1019D0008142D6DC354B2A881B888342A3EB010663
:1019E000A8BF03465B1AB242BABF02FB03330136FB
:1019F000534393FBF6F31C44C3E72A4B1C888CB17A
:101A00002B4B224D1C78002CB7D02C88B5E7BDE8B5
:101A10007040FFF77FBFFFF741FF2046BDE87040F1
:101A2000FFF764BF194DA8E711200EF06FF91C4BAA
:101A30001860C6E70F200EF069F91A4B1D4A1B8883
:101A40001060002BA1D01C4AC0F53B6311880833FD
:101A50008B429ADB194A288812889342A2EB01052F
:101A6000A8BF1346A842A3EB010306DA00FB033329
:101A7000013593FBF5F31C4488E700FB03F292FB6E
:101A8000F5F31C4482E700BFCE9FFF1FD49FFF1FCA
:101A9000A29FFF1F349FFF1FE19DFF1F549FFF1F49
:101AA000549DFF1F3E9EFF1FDC9DFF1FCC9FFF1F0D
:101AB0006C9DFF1F709DFF1F3C9EFF1FB89FFF1F67
:101AC000F8B510200EF022F9C830B0F5FA7FC0F258
:101AD0009680B0F57A6F0146A8BF4FF47A6101F5A0
:101AE0001673B3F57A6FA8BF4FF47A639BB289B2CD
:101AF000914A924C11802220238008F00BFC21880F
:101B00008F4D904C242008F005FC0E200CF062FD57
:101B100040F6FF71C8308842A8BF084620EAE0704E
:101B200000F2DC5283B28A42A8BF0A46022019465C
:101B300022802B8008F0EEFB2188042008F0EAFBCD
:101B400001200EF0E3F8044600200EF0DFF8A0427A
:101B5000B8BF204600F1C801B1F5FA7FC0F2D180CC
:101B6000B1F57A6FA8BF4FF47A6101F54873B3F508
:101B70007A6FA8BF4FF47A639BB289B2724A734CF2
:101B800011800A20238008F0C5FB21880C2008F072
:101B9000C1FB0F200EF0BAF8C0F53F610431B1F57A
:101BA000AF6FC0F2AB80B1F5FA6FA8BF4FF4FA6126
:101BB00089B2674BC0F54360B0F5AF6F1980C0F2D2
:101BC0009A80B0F5FA6FA8BF4FF4FA6083B2614C07
:101BD000A420238008F09EFB2188A62008F09AFB11
:101BE00015200CF0F7FC00F59671B1F52F7F0BDB9B
:101BF00041F25C23994240F38980194608E040F2A3
:101C00004C434FF4FA7173E740F214534FF42F71C1
:101C1000514A1180514C524D2380062008F07AFB26
:101C20002188504E082008F075FB00274FF4AF7450
:101C3000F9B24D480AF096F955F8043BC3F596738E
:101C400000FB03F086FB0023C017C0EB6310844247
:101C500007F10107A8BF0446062FE9D1434F414EC3
:101C60000025E9B242480AF07DF957F8043BC3F574
:101C7000967300FB03F086FB0023C017C0EB6310D4
:101C8000844205F10105A8BF04460C2DE9D1394F66
:101C9000344E0025E9B238480AF064F957F8043B9D
:101CA000304AC3F5967300FB03F086FB0013C017A0
:101CB000C0EB6310844205F10105A8BF04460C2D5A
:101CC000E8D1A4F11401312931DD40F23A73A4F5D1
:101CD000B97403FB04F482FB0432E417A4EB621230
:101CE00089B232322548264B01801A602A20BDE88D
:101CF000F84008F00FBB4FF4AF6368E74FF4AF61F3
:101D000057E740F214534FF4FA7137E7124A00F5DF
:101D1000617089B2B0F52F7F1180B8BF4FF42F7377
:101D2000FFF678AF8342A8BF03469BB272E740F24A
:101D30006C723221D6E700BF4C9FFF1F489FFF1FE8
:101D4000389EFF1F5C9DFF1F989FFF1F9C9DFF1FDC
:101D50003C9EFF1FB89FFF1FDC9DFF1FCC9FFF1FF6
:101D6000688AFF1FB5814E1B889DFF1F388AFF1FA1
:101D7000BC9DFF1F4089FF1F309EFF1FFA9FFF1F62
:101D8000248AFF1F2DE9F04F0C2083B00CF0EEFBEE
:101D90000C200CF0DBFFC949DFF8A8A314200CF0DD
:101DA000E5FFC749C74809F0ADFD022103200DF04A
:101DB00073F8022104200DF06FF8022105200DF0C8
:101DC0006BF8022106200DF067F801210A200DF0C2
:101DD00063F8012109200DF05FF801210D200DF0BD
:101DE0005BF8012128200DF057F8012114200DF097
:101DF00053F8012116200DF04FF8012117200DF0A6
:101E00004BF8012121200DF047F802211C200DF094
:101E100043F801211B200DF03FF800211B200DF09D
:101E200027F81C200DF02AF8B0FA80F35B091A207D
:101E30008AF800300DF070FA1F2000210DF032FA00
:101E400004200DF01BF8002800F0878105200DF01C
:101E500015F8002800F0B28100239B4C0620237067
:101E60000DF00CF8B0FA80F35B094FF0000B974AC5
:101E7000137006F0A5FD2478002C40F069815846C7
:101E800008F072FA924B934A1B88934812880270AA
:101E90009249934D40F23A72A3F5AF7302FB03F3FC
:101EA00081FB0312DB17A3EB6213323301210D20F8
:101EB0002B600CF0DDFF64200DF016F806254FF4C2
:101EC00016710A200CF044FE00950C237D4A8548CB
:101ED0005D210AF0AFF8002800F0AD8164200DF01C
:101EE00003F821460A200CF033FE4FF496710920C6
:101EF0000CF02EFE00950C23724A7B485C210AF000
:101F000099F8002800F0848164200CF0EDFF214650
:101F100009200CF01DFE4FF4967116200CF018FEEF
:101F200000950C23674A71485B210AF083F800286A
:101F300000F04B8164200CF0D7FF214616200CF0F6
:101F400007FE4FF4967117200CF002FE64200CF08F
:101F5000CBFF214617200CF0FBFD64200CF0C4FFE2
:101F600021460D200CF084FF614A62481268DFF8B8
:101F7000D891614F614D624EDFF8D081002301217D
:101F8000FEF792FA01233C602C60346089F800303F
:101F900004240F200DF0BAFE336803440E20336092
:101FA0000CF018FB3B6899F8002018443860002AB0
:101FB0007DD015200CF00EFB2B681844286004F02F
:101FC000010080F0010004F0D1FFB8F80030002BD0
:101FD00014BF4B20DC200CF087FF013CD9D13368C3
:101FE0003968454A2868474F002BB8BF033300299A
:101FF000B8BF0331891011604349444A09881488E5
:102000009B1000283360B8BF0330414E8210581A2D
:1020100019442A60316038603E4D3F483F49161BE5
:1020200022442E6002600B60BBF1000F40F0AE80D6
:10203000B8F80030002B00F09C80394B01240420BC
:102040001C600CF01BFF18B9364B234A1C70107033
:10205000354B1B881C2B00F0A180344C04F1C805C3
:1020600023200CF0B7FA44F8040F01200CF03CFFD9
:10207000A542F5D19AF8003023B12D4B1B78002BE7
:1020800040F09780002121200CF0F2FE294A2A4BD3
:102090001078187008F004F904F060FF2749284808
:1020A00045F6BF5203B0BDE8F04F0FF045BA11201E
:1020B0000DF02CFE2B681844286080E7001B374683
:1020C00040420F000092FF1F8D9DFF1F3C9FFF1F8E
:1020D000FA9FFF1F0CA0FF1FF89DFF1FB5814E1B2D
:1020E000248AFF1F889DFF1F309EFF1FBC9DFF1F7E
:1020F0003C89FF1F609FFF1F589DFF1F409DFF1FD2
:10210000BC9FFF1FC09FFF1F348AFF1F7089FF1FE6
:10211000389FFF1F2CA0FF1FFC9DFF1F10A0FF1F5B
:10212000C89FFF1F759DFF1FCE9FFF1F449EFF1F6F
:102130004E9FFF1F509FFF1F339FFF1FA5050000ED
:10214000F09FFF1F369FFF1F549FFF1F8E9FFF1F93
:1021500003B0BDE8F04F09F0E9BA06200CF08EFE9E
:1021600000287FF473AE374C034620704FF0010B0C
:102170007DE64FF4FA7004F009FF04F0F3FE06F078
:102180006FFF4FF4AF600CF0AFFE56E7FFF798FC1F
:10219000B8F80030002B7FF450AFEAE72A4B1888DC
:1021A00000283FF45AAF294BC0B2197807F030FF2E
:1021B00053E7012121200CF05BFE67E703200CF0C0
:1021C0005DFEB0FA80F35B0947E603200CF056FE93
:1021D0000028FAD104200CF051FE0028F5D105208A
:1021E0000CF04CFE0028F0D106200CF047FE002831
:1021F000EBD10DF0ABFE04200CF040FE40B9052001
:102200000CF03CFE20B906200CF038FE0028F0D07F
:1022100003200CF033FE0028FAD1ECE704200CF088
:102220002DFE40B905200CF029FE20B906200CF047
:1022300025FE0028DDD003200CF020FE0028FAD176
:10224000ECE700BF8D9DFF1F009EFF1FA89DFF1F95
:102250002DE9F04FB04B1A78012A95B000F0FC82BE
:10226000C0F00982022A00F0D780AC48DFF850E3C2
:1022700090F80080AA48AB4DAB4FAC4EAC4BAD498B
:102280000090AD480390AD489EF800B002902D78C4
:10229000AB483F7896F800E01B780978DFF828C350
:1022A000DFF82893DFF828A30190012A9A4894BF09
:1022B000013200220270A34AA3481370A34A80F897
:1022C00000B01570A248A34A077082F80080A248A7
:1022D000A24A03701170BEF1000F40F01281A04AB3
:1022E00010880D2800F0B8819E4C00202070024616
:1022F00004462DB19A480088002840F0B98105466F
:10230000994806882544002E40F066819748984CED
:10231000029E0078367824780130A0EB4600002C2D
:1023200040F01383019C94F800E0CEEB0004BEF172
:10233000000F40F049830026DFF880E203989EF802
:1023400000E00078A41BA4EB4E043C44CBEB040457
:1023500010B1B7FA87F040099CF800602718BC1B41
:102360001EB11EF1000618BF012699F800009AF868
:102370000090009FC6EB040EC0EB0E00A0EB4900DE
:10238000804497F800C07B4FC3EB0803A3EB4101E7
:102390000C2313FB0C113960774B784F784C79483C
:1023A0001B880088D7F800C0774E2788774C36887E
:1023B000D4F800E0033BC0EBC00403EB4303C7EBDE
:1023C000C70001EB83036444714F33447044714E82
:1023D00057F8244056F820000C3B1D442544054482
:1023E0000AB16D4B19606D4A13689D4200F030814F
:1023F0006B4B6C4819680791079901601B6808933B
:102400006948089B008815605B1A834284BF674B4C
:102410001D6015B0BDE8F08FDFF8B881644E08AFDD
:102420000025E9B2634809F09DFD58F8043BC3F567
:10243000967300FB03F086FB00230135C017C0EB49
:1024400063100C2D47F8040BEBD15B4B3C4DB3F8FC
:1024500000C00195109D09980F99384C444EDFF843
:10246000CCA0DFF8C090DFF8C880029411AA8CCA13
:102470006545ACBF4FF0000E4FF0010E8445D4BF50
:10248000002001208C45D4BF0021012121709445FA
:102490002B490B9D3070D4BF002201220A709C454D
:1024A000464A24481D4E01781D480090D4BF0023A1
:1024B0000123BC451370D4BF002701271A4B164ACD
:1024C0001F70AC450C9D3E4B1B488AF800E0D4BF02
:1024D0004FF0000B4FF0010BAC45D4BF0025012598
:1024E00083F800B089F8005098F80030127896F818
:1024F00000800390DFF8D0C0DFF8D090DFF8D0A0E4
:10250000D3E6304A174814880122182C027040F292
:1025100024820024EDE600BF329FFF1F809FFF1F33
:102520003D9FFF1FE09DFF1FDE9DFF1F38A0FF1F87
:10253000819FFF1F829FFF1F8C9DFF1FE59FFF1F35
:10254000E69FFF1F32A0FF1F33A0FF1F34A0FF1F15
:1025500035A0FF1F36A0FF1F37A0FF1FD29FFF1F10
:102560003AA0FF1F6C9DFF1F4C9DFF1F368AFF1F67
:102570001CA0FF1F889FFF1FA69FFF1F409EFF1FDD
:10258000E29DFF1FC49FFF1F649DFF1F04A0FF1F4C
:10259000784601000040010014A0FF1FD49DFF1FDA
:1025A00010A1FF1FC49DFF1FDE9FFF1F20A0FF1F64
:1025B000B5814E1B309EFF1FFA9FFF1FE79FFF1F35
:1025C000DF9DFF1FCE9FFF1F31A0FF1FD09FFF1F6A
:1025D000D19FFF1F4089FF1F012E00F07382022E42
:1025E00000F0D282032E7F4B00F0F3811E78029B15
:1025F0009CF800E01878039B99F800C093F80080DD
:10260000019B9AF800401F78A6EB4E03A4EB8404CC
:10261000CCEB030CC0EB80760CEB0403C0EB860024
:10262000034403EB480303EB810327B16E490978A8
:10263000002940F02E83012600996C480978C1F1E9
:10264000060101EB4101334403EB81010160A3E684
:102650006749684B0968D1E6002D3FF445AE664AEC
:10266000664E14880122182C327040F2768174462E
:10267000A0F10D0544E6DFF8D081614E08AF0025DA
:10268000E9B2604809F06EFC58F8043BC3F5967354
:1026900000FB03F086FB00230135C017C0EB63107D
:1026A000062D47F8040BEBD1574BDDF820A01A8814
:1026B000DDF82490554CDDF82880554BDDF82CC012
:1026C000DFF888B10C980D9D19889245ACBF4FF08A
:1026D000000E4FF0010E4A45D4BF00270127277096
:1026E00042454C4C8BF800E00EEB0703D4BF0026AC
:1026F00001266245D4BF4FF0000E4FF0010E267048
:1027000082423344DFF848B1434E8BF800E0D4BF37
:10271000002701277344AA423770D4BF4FF0000E40
:102720004FF0010E3B443D4F3D4E87F800E07344AF
:102730003C4F0097DBB2012933703B4E3C468CBFC7
:10274000002701273770AA424FF00006267040F399
:102750001181824200F38081012940F27D8162452E
:1027600040F30F81424500F3B082012940F2AD826F
:102770004A4540F30F819245C0F2C782012940F2D9
:10278000C4822A4E3778012F40F20B8109B1009C98
:102790002770274F3F88002F00F0BC82002B40F0AD
:1027A000B982244B1B88013B9BB2062B00F2B282FC
:1027B000214B1B78002B00F0AD82204B1B68012BB6
:1027C00040F0EF801E4BDFF88CC0D3F800E00C2304
:1027D0009EFBF3F703FB17E3ACF80030194B03271C
:1027E0001F70DEE0368AFF1FE79FFF1F889FFF1FD5
:1027F000C49DFF1F10A1FF1FCE9FFF1F6C9DFF1FD9
:10280000B5814E1B889DFF1FFA9FFF1FFD9FFF1F75
:102810001E9FFF1FFE9FFF1F00A0FF1F01A0FF1FA5
:10282000949DFF1F3D9FFF1FA49FFF1F4A9FFF1FF7
:10283000B09FFF1F529FFF1F3A9EFF1FC89FFF1FA1
:1028400020A0FF1F188AFF1F688AFF1FFC9FFF1F21
:10285000FF9FFF1F8C9FFF1FDFF85882824E08AF3B
:102860000025E9B2814809F07DFB58F8043BC3F527
:10287000967300FB03F086FB00230135C017C0EB05
:1028800063100C2D47F8040BEBD1794B0C9D1F887E
:102890000B9B0A98099A089EDFF81CA2DFF81C928D
:1028A0000F99744CDFF818C20394BB42ACBF4FF0D1
:1028B000000E4FF0010EAF42D4BF00250125874224
:1028C000109B84F800E0D4BF002001209742D4BFC1
:1028D00000220122B742D4BF4FF000084FF0010898
:1028E0008AF800209F42644A89F80000D4BF002380
:1028F000012362481370129A80F800808F4260486A
:102900008CF80050D4BF002101219742017055DCA2
:1029100000220D985B4D5C4E2A708742D4BF002781
:1029200001275A4A3770009259485A4A5A4E5B4D0D
:10293000077892F800E05A485A4A02905A4896F8A6
:1029400000B02D7812780190AFE4019C46B1267852
:10295000002E40F08481441EEEE40C3C0122C8E4C9
:1029600094F800E00138CEEB0004BEF1000F7FF4D4
:10297000E3ACE0E482427FF7F2AE624555DC012928
:1029800053D942457FF7F4AE4A4500F3B981012996
:1029900040F2B6819245BFF6F4AE009C434E01234F
:1029A0002370032945D1AA4243DD824241DC3378BA
:1029B000062B3ED1009A072313703CE0119A9742F0
:1029C000D4BF00220122A4E7002E3FF4B4AC0126BC
:1029D000B2E41C780398029B9CF800601B7890F886
:1029E00000C099F8007001989AF8008090F800E013
:1029F000A4EB4604E71BA8EB8800C3EB83743844C0
:102A0000C3EB8403034403EB4C0303EB8103BEF1EC
:102A1000000F40F04381012600992548097833448E
:102A20000C2414FB01310160B6E4009A1F4E05230B
:102A30001370009B1B781149114A0F4891F80080D0
:102A400011780C4A337003920378DFF874C0DFF812
:102A50006C90DFF864A067E7009C144E06230329FE
:102A60002370E8D1A1E700BFB5814E1BBC9DFF1FBD
:102A7000FA9FFF1F8C9DFF1F819FFF1F809FFF1FDD
:102A8000829FFF1FA29DFF1F1E9EFF1F3D9FFF1FD6
:102A9000DE9DFF1F38A0FF1FDF9DFF1FE09DFF1F72
:102AA000E59FFF1F329FFF1FE69FFF1F4A9FFF1FEB
:102AB000889FFF1F388AFF1FD19FFF1FD09FFF1FD6
:102AC00031A0FF1F964CDFF864E2207805909EF855
:102AD000004002980494059C007802900134A4EB15
:102AE00040040498002840F0AB80019890F800E082
:102AF0000498261ACEEB06000490BEF1000F40F0B9
:102B00009A8074460398874E00780190049836782E
:102B10000396041BA4EB460401983C44CBEB04044D
:102B2000002800F08380B7FA87F040099CF8006025
:102B30002044871B1EB10398061C18BF012699F874
:102B400000009AF80040BE1B301AA0EB44008044FD
:102B50000298C3EB0803A3EB4103002863D1BEF145
:102B6000000F40F0AA807344002C76D100290CBFDE
:102B700000206FF0090000996B4C097803440C2089
:102B800010FB0131216007E4029C019E247802942D
:102B9000664C367801969AF8006094F800A0614C73
:102BA000634899F800E094F800909DF80440847020
:102BB00080F806E080F803909CF800C09DF808407B
:102BC000DFF87C91DDF808E080F808800470077178
:102BD00080F805C0C671417280F801A04FF000086E
:102BE00001200021524C0E465FFA88FA4F46F44607
:102BF00007E0022809D00A290BD014F801CF17F8F2
:102C0000010F844501F10101F3D101360A29F6B221
:102C1000F3D1092E5ED808F10108B8F1100F22D0C7
:102C200019F80A0FDDE74FF0000E9CE701987DE7E9
:102C3000CEEB040004900298041C18BF012461E745
:102C40000298002834D0019890F800E0BEF1000FFF
:102C5000EED1601E0490744654E700208BE7841B7D
:102C60000126FFF769BB2E4832490478C86B0399E7
:102C7000013409782044CBEB000008440021009B7C
:102C80001C78294B401A0C2111FB04011960FFF735
:102C900083BB1BF1000618BF0126CDE4214909784A
:102CA00000293FF4B8AE1BF1000618BF0126B3E6B9
:102CB000019890F800E030461BE7039800280CBF0D
:102CC0004FF0000E4FF0090E4DE7009C1A4E042302
:102CD000237066E612481749047851F828000399D2
:102CE000013409782044CBEB00000844002BC5D008
:102CF000BAF1000FC2D1BBF1000FBFD00121BEE776
:102D0000009C0D4E032323704BE6009C0A4E0223C9
:102D1000237046E6094B1B68012B7FF442AE5DE54C
:102D2000368AFF1FE79FFF1F889FFF1F1CA0FF1F02
:102D3000049EFF1F7C89FF1F4A9FFF1FC89FFF1F24
:102D4000484501002DE9F04F3A4B1B788BB0002B22
:102D50006BD10E200BF03EFC0FF07AFD0146364899
:102D6000364E374DFDF7E6FB3348FDF7B9FB0FF064
:102D700089FF80F30C003060FFF76AFA2C68012CA1
:102D80007AD0022C00F0C582032C00F049842D4E2D
:102D90002D4C33682D4A2E4E0993099B31681288B9
:102DA0002360591A013A9142274F00F2AD82294E11
:102DB00032689A1A092A00F29682274E32689A1AC5
:102DC0000D2A00F28B82254E32689A1A252A1AD9CA
:102DD000234B1B88002B40F09B81224B1B78002B40
:102DE00040F09681FEF7A0FA1F4B1B881B3B9BB25D
:102DF000022B04D81D4B1B78002B40F08C8104F073
:102E0000D7F8236833601A4D2A689B1A502B00F2BA
:102E10000A82184B1B88012B00F0258207F09EF8D0
:102E200006F058FF0BB0BDE8F08F08F00BFB0BB0BD
:102E3000BDE8F08F8D9DFF1F609FFF1F9C9FFF1FB0
:102E4000C89FFF1F10A1FF1F5C9FFF1F208AFF1F4D
:102E5000349EFF1F189EFF1FF09DFF1FF49DFF1F54
:102E6000469FFF1F849DFF1FCE9FFF1F6C9DFF1F6E
:102E7000409FFF1FA09FFF1FDFF84093AB4AB9F8A8
:102E800000001378834204D0C3B21846137007F0D1
:102E900057F8DFF82C83A64AB8F800301178994229
:102EA00004D0A44F3978002940F0B087A24A336893
:102EB0001288A24E9A42C0F28D81A14A1278002A4D
:102EC00040F08881DFF8FCA2BAF8003023B99D4BAE
:102ED0001B88002B00F0A4859B4A9C4B11881B8803
:102EE0009B4A0B4412685B1093429A4A126880F224
:102EF0001E8500219342B4BF01230B460491029327
:102F0000ACBF4FF0010B8B4605910E200BF062FB1E
:102F1000914B924A1B6803930133002B8446176838
:102F200040F38A87802BA8BF80238D4A8D49127871
:102F30000191002A00F058810978914200F05481F3
:102F4000B8F80010DFF878E2994201F06181794920
:102F5000AEF80030844B4FF0010E81F800E0197894
:102F6000DFF864E2814B01981B7802708EF8001044
:102F7000002B40F03883029B002B40F02F83A7F2F8
:102F800052339C4533DA6F4B1B88002B2FD0BBF19B
:102F9000000F40F02883764B1B881BB1059B002B4C
:102FA00040F02183049B13B3724B1A78FAB9DFF80F
:102FB0001C9299F8004001221A70002C40F0FD8408
:102FC0006D4B1B78002B42F0BC846C4B1B78002BA4
:102FD00002F048876A4B1B784BB96A4B1B7833B1B8
:102FE000B8F8003053490A33A8F800300A700E20B0
:102FF0000BF0F0FA6FF454731F44874202DC5D4B10
:1030000000221A70604B1B88002B00F0BA845F4BC3
:103010005F4A1B78117899426DD0002B6BD05949CB
:103020000878002800F0B3875A4991F800C0BCF135
:10303000000F40F0AA87584FDFF894E197F800A0FE
:10304000564C574F8EF800C04FF0010E0194039775
:1030500084F800C087F800C081F800E0BAF1000FE2
:1030600008D000240C70019F03994FF0010E87F8DF
:1030700000E00C7040490978002901F06C80494C4F
:1030800094F800E0BEF1000F41F01D81DFF81081DF
:103090004FF0010C88F800E084F800C0374C247829
:1030A00094B1DFF82CE19EF800C0BCF1000F41F0B4
:1030B0000081DFF8E0904FF0010889F800C08EF839
:1030C0000080002901F04C803749097899B13448D3
:1030D0000178002941F0F380DFF8B8E0334F2F4C3E
:1030E0008EF800104FF0030E87F800E02D4F21708E
:1030F00001243970047013702D4B1B88A3F11B023F
:10310000012A40F271861D2B00F08F86294C40E683
:10311000FEF7ACF866E6284B1B78002B3FF46FAE49
:103120002B68012B7FF46BAE6BE600BF339FFF1F54
:10313000F89DFF1F759DFF1F389EFF1F10A1FF1FE9
:10314000849DFF1F209EFF1F9C9DFF1F989FFF1FB8
:10315000B89DFF1F7C9DFF1F14A0FF1F589DFF1FE0
:103160000AA0FF1FD09DFF1F0BA0FF1F1E9EFF1F69
:10317000569FFF1F959DFF1F32A0FF1F33A0FF1F0B
:1031800034A0FF1F35A0FF1F529FFF1FA29DFF1FEE
:10319000449DFF1F909FFF1F36A0FF1FE49FFF1F4E
:1031A0003A9EFF1F459DFF1F6C9DFF1F188AFF1F42
:1031B000CE9FFF1F5C9FFF1FD29FFF1F509FFF1FCF
:1031C0000CA0FF1FD89DFF1FD19DFF1F3D9FFF1F1C
:1031D000749DFF1F31688E4A069106988D491060D4
:1031E00002220B602A606DE68B49DFF8A0E20978C5
:1031F00000293FF4B7AE9EF8000081423FF4B2AE22
:1032000003984B2840F3C7871833802BB8F8000089
:10321000A8BF802398423FF4A5AE80480380804831
:10322000012303709EE605F017FC7E4B1B788BB9DB
:103230007D4B1B7873B97D4B1B785BB97C4B1B783E
:1032400043B97C4B1B782BB97B4B1B7813B903F02C
:1032500085FE01E003F08EFE23682B60774B1B8810
:10326000012B7FF4DBAD764B764A19681778764EE2
:10327000A92303FB01F10029744BB8BF01F57F516D
:103280001868734BB8BF3F3189132A225439183854
:1032900002FB00111D786FF0140202FB071232606E
:1032A0006C49002D00F04A810B689A4200F30084BB
:1032B00080F24481684D2878002840F0E88767480C
:1032C0000068D0F17F0048BF0330801001301B1A26
:1032D0009A4200F333810B601A4630E1FEF746FB59
:1032E000236833606FE5FDF761FBFEF749F85C4B3F
:1032F0001B88032B00F0A3855A4B1B88032B00F07F
:10330000A2852368336058E5FDF79CFA3B6833607B
:103310004DE5554A34681288A24204DB464B1B78BF
:10332000002B00F00684514E394833680793504B08
:10333000079900681B88091A994200F2AD80002B9A
:1033400000F0AA804B4B198800293FF4DFAE314BC7
:1033500049481B680088A342B8BF23469A4201F33C
:10336000B681464A8342A8BF03461360DFF8208136
:1033700088F80010354FFDF765FA38687F2840F36C
:1033800000863F4B7F3883FB0032C317C3EB6203D9
:1033900003EB4303A0EB830073303A4B02931B888B
:1033A0003860002B40F02287204B01931B78002BC4
:1033B00000F06E84344C2378002B00F06984DFF831
:1033C000D490DFF8BCA04FF0000B0CE003F17300C9
:1033D000C0B298F8001006F04BFE23780BF1010BF9
:1033E0005B4540F355843B6859F8040F1844A0F13D
:1033F0007F038AFB0321DA17C2EB610202EB420270
:103400007F28A3EB8203E1DCFDF73CF9E0E700BF96
:10341000E49DFF1F589FFF1F0BA0FF1F0CA0FF1F65
:10342000759DFF1F3A9EFF1F909FFF1FE49FFF1F88
:10343000459DFF1F749DFF1F849DFF1FA09FFF1FC1
:103440001C8AFF1FB29FFF1F109EFF1F20A0FF1F9F
:10345000E19DFF1F249EFF1FEC9FFF1FE89FFF1FA2
:10346000A29FFF1F349FFF1F389EFF1F10A1FF1F49
:103470001C9EFF1F6A9DFF1F5C9DFF1F489DFF1F35
:10348000ABAAAA2AB29DFF1FE089FF1FD19DFF1F93
:10349000C69FFF1FB889FF1F8F4B90491B68088884
:1034A0008F49A342B8BF23469A4200F31F838D4C35
:1034B00009888342A8BF0346236000297FF456AFE2
:1034C0009A42C8BF0B4640F31883801AB0F5804F6C
:1034D000AABF9B03C3EB8333013093FBF0F0FDF7EE
:1034E00097F9C0F3C6100FF0B3F97F4B0446188864
:1034F0000FF0AEF97D49074620460FF0FDF9014671
:1035000038460FF0F9F921460FF0EEF84FF07E51F2
:1035100004460FF08FFB002841F0CE80744920460E
:103520000FF0A6FB002840F0C18620460FF0D0FB2C
:10353000C0B2DFF8108288F800001BE70A606D4B0C
:10354000188858B36C4B256853F82040B5FBF4F34A
:10355000772C04FB135300F3C282C3EBC30303EBCA
:10356000031393FBF4F36548654C50F8230024687B
:10357000644BA0F2FF7004FB00F000F57D3000F515
:10358000607000EB4004C0EBC40083FB00430344C5
:10359000C017C0EBA3400B3802440A605A495B4B8A
:1035A0000888198800F27C704300B3F57C6FA1F1A4
:1035B00064014FEA4100B5BF5549564903FB022259
:1035C0005A4381FB02311144D317C3EBE123C118E5
:1035D00081F30C0128200BF0BBFA1FE4BAF800308D
:1035E000002B3FF4CCAC4C4B1B685A1C002A40F318
:1035F000AC81802A00F3A881484C49494948248875
:10360000098800682144B0EB610FC0F24986A3F13C
:1036100048020F2A3FF6EBAC473BA9F80030E6E43E
:10362000414BD6F800801988414540F38F803F4BCD
:103630001B78002B40F08A80DFF80C9199F800008D
:103640007F2840F30F86A3F155337F3803F1004301
:1036500083FB0032C317C3EB620303EB4303A0EB0E
:1036600083007330324B02931B88C0B289F800008C
:10367000002B41F00E802F4B01931B78002B00F0A4
:1036800098842D4C2378002B00F093842B4FDFF887
:10369000B0804FF0000A0AE003F17300C0B206F0F8
:1036A0000BFD23780AF1010A534540F3828457F851
:1036B000043F99F800001844A0F17F0388FB032120
:1036C000DA17C2EB610202EB42027F28A3EB82030E
:1036D000E2DCFCF7D7FFE1E7589FFF1F5C9DFF1F6F
:1036E0006A9DFF1F489DFF1F509DFF1FCDCCCC3D05
:1036F0000000FE42669DFF1F24450100FC3D0100C5
:10370000B49FFF1F4D26128124A0FF1FE89DFF1FBD
:1037100081DFFF8183200882889FFF1F4C9FFF1F4E
:10372000489FFF1FAC9DFF1F389EFF1F849DFF1FFA
:10373000B29DFF1FE49FFF1FE089FF1FB889FF1F95
:10374000ABAAAA2AC69FFF1F869FFF1FB64F3868E5
:103750007F2800F3D981FCF795FFDFF8449399F8AF
:103760000040844200F03982B04B1B88002B43D1CB
:10377000AF4AB04812680088914205DC8242D4BF4B
:10378000C1EB0203C1EB0003411AB1F5804FA6BFA4
:103790009B030131C3EB833393FBF1F0FDF738F862
:1037A000C0F3C6100FF054F8A34B804618880FF0F2
:1037B0004FF8A249824640460FF09EF80146504617
:1037C0000FF09AF841460EF08FFF4FF07E51804681
:1037D0000FF030FA002840F0D586994940460FF0A6
:1037E00047FA002840F05F8540460FF071FAC0B2FA
:1037F000DFF8B08288F800007F2C40F3B483914852
:103800007F3C80FB0430E317C3EB600000EB40001B
:10381000A4EB800073308C4B01931B78C0B289F805
:103820000000002B40F01683884B04931B78002B7C
:1038300040F0FB84864B03931B78002B40F03F87BE
:10384000844B0293039B1B78FBB1834B1B88012B9A
:1038500000F0EA85022B00F09387032B01F0AB8187
:10386000042B01F05C83052B01F04684062B01F04C
:103870009485072B01F02A87082B02F02780092B5B
:1038800002F0F3800A2B02F0CC82019B1B78002B04
:1038900000F04E84029B6F4C1988002900F0BE8412
:1038A00038687F2840F3D382664B7F3883FB003231
:1038B000C317C3EB620303EB4303A0EB8300733036
:1038C0003860002940F07884019B1B78002B00F0C1
:1038D0009081624C2378002B00F08B81DFF8C8A127
:1038E000DFF8C0814FF0000B0CE003F17300C0B2B1
:1038F00098F8001006F0BCFB23780BF1010B5B4538
:1039000040F377813B685AF8040F4E4A1844A0F1FF
:103910007F0382FB0321DA17C2EB610202EB420252
:103920007F28A3EB8203E0DCFCF7ACFEDFE79342E9
:103930004FF0000B80F2F5800123CDF808B0CDF8F0
:1039400014B00493FFF7E1BA80244549454B464A39
:1039500009881B8812680B44B2EB630FBFF647ABB4
:10396000424B1B78002B40F0A783B8F80030404A48
:10397000A3423FF43CAB3F4B148001221A70FFF787
:1039800036BB334F3C4C304830493C4A3B70237087
:1039900003700B70FFF7AFBB394B1B78002B7FF424
:1039A00026AB039B374A243B83F34703D9B25B2002
:1039B000136006F02DFB99F80040032C30D1DFF89E
:1039C000EC8098F80030002B42F01A832E4F3B78A1
:1039D000002B42F008832A4C2378002B42F0F68219
:1039E0002A4B1B78002B42F0E482294A1380294B92
:1039F0001B78002B42F0D0820C4B7F221A8098F863
:103A000000306BB93B785BB923784BB9224A7F21F0
:103A10000720138006F0FCFA7F210B2006F0F8FA4D
:103A20001E4B1F68FFF7E3BA20A0FF1F6A9DFF1F10
:103A3000489DFF1F5C9DFF1F509DFF1FCDCCCC3DBF
:103A40000000FE42ABAAAA2AE49FFF1F459DFF1F6C
:103A50003A9EFF1FB29DFF1F529FFF1FE089FF1F6D
:103A6000489FFF1F4C9FFF1FAC9DFF1F6C9DFF1FBA
:103A70000CA0FF1F759DFF1F909FFF1F749DFF1FD0
:103A800035A0FF1F989DFF1F34A0FF1F33A0FF1F0D
:103A90002A9EFF1F36A0FF1F849FFF1F589DFF1FF8
:103AA000869FFF1FC69FFF1FB889FF1F32A0FF1F01
:103AB000B94D2878002840F00E83B8480068D0F14E
:103AC0007F0048BF033003EBA0030133B4480B6011
:103AD0009A42B8BF0260FFF632AD1A462FE5C3EB3B
:103AE0000313D800631C90FBF3F33CE5AD4B09884E
:103AF0001A6000297FF43AAC13469842D4BFC2EB57
:103B00000003C2EB0303E0E4A74B7F3883FB0032E2
:103B1000C317C3EB620303EB4303A0EB83007330D3
:103B20001BE60123CDF810B0CDF808B00593FFF7E0
:103B3000ECB901232B609D4E9D4CFFF72AB9039BE6
:103B40001B78FBB19B4B1B88012B00F0C283022B1F
:103B500000F09486032B00F0B587042B01F0BB81A5
:103B6000052B01F05482062B01F00F84072B01F086
:103B7000F984082B01F06486092B01F0DC870A2BFD
:103B800002F00281029B1B88002B00F01E83019B28
:103B90001B783BB9049B1B7823B9039B1B78002B34
:103BA00000F07787844B1B78002B00F02D81834930
:103BB0000B78082B00F2288181483A680068814C14
:103BC0000133DBB25F1E101A44F827000B707E4BE6
:103BD000D6F80080198889F800208845734E7FF751
:103BE00095AA3268794B0892089A714C1A60FFF7CF
:103BF000D0B8049B1B78002BA1D03B68A3F10C002C
:103C00007F2840F31B8368488B3B80FB0320DA1737
:103C1000C2EB600000EB4000A3EB800303F17300F4
:103C2000DFF8BC81C0B298F8001006F021FA019BC1
:103C30001B78002B83D0614C2378002B3FF47FAF9F
:103C4000DFF8A0A14FF0000B0CE003F17300C0B24D
:103C500098F8001006F00CFA23780BF1010B5B4585
:103C60007FF76DAF3B685AF8040F4F4A1844A0F134
:103C70008B0382FB0321DA17C2EB61020C3802EBE3
:103C800042027F28A3EB8203DFDCFCF7FBFCDEE7CC
:103C9000494B1B78002B40F09E824D4B1B78002B2C
:103CA00045D03B68A3F10C007F2840F3D8823E4A00
:103CB0008B3B82FB0321DA17C2EB610202EB42026B
:103CC000A3EB820303F17300C0B298F8001006F072
:103CD000CFF9019B1B7853B3384C23783BB3DFF803
:103CE0000491DFF8C4A04FF0000B0BE003F1730068
:103CF000C0B298F8001006F0BBF923780BF1010B65
:103D00005B4514DD3B6859F8040F1844A0F18B03A0
:103D10008AFB0321DA17C2EB61020C3802EB420284
:103D20007F28A3EB8203E1DCFCF7ACFCE0E7294B46
:103D30001B78FBB11F4B1B88012B00F02684022B44
:103D400000F01D86032B00F0AC87042B01F00C81E2
:103D5000052B01F03B82062B01F03583072B01F088
:103D60005B83082B01F00586092B01F09F860A2B47
:103D700001F0B987029B1B88002B00F04382164B91
:103D80001B78002B40F03982144B3A681A700323D9
:103D90002B60FFF7BBB900BFEC9FFF1FE89FFF1F21
:103DA000249EFF1F489DFF1FABAAAA2A10A1FF1F38
:103DB0005C9FFF1F529FFF1F909FFF1FE089FF1F07
:103DC000789DFF1FBC89FF1F389EFF1FCCA0FF1FDF
:103DD000459DFF1F3A9EFF1F749DFF1F869FFF1F7B
:103DE000C69FFF1FB889FF1FDFF8108398F80030C7
:103DF000002B40F0BC80BC4F3B78002B40F06E8421
:103E0000BA4C3B70FEF7C5BF3A68E0E6DBB2184635
:103E1000137006F0BBF9B649B648B74A00230B70D9
:103E20003B7003701370FFF741B8B44AAE4B127881
:103E30001A70AE4CFEF7ADBF0123FFF776B8FCF762
:103E400033FCFFF759BAFCF785FCFFF75ABAFCF7C9
:103E500019FC35E5AA4B02931B8863BBA64B049360
:103E6000A84B0393A84C23787BB3DFF8AC82DFF830
:103E70009CA24FF0000B09E003F17300C0B206F002
:103E80001BF923780BF1010B5B451EDD58F8043F4D
:103E900099F800001844A0F17F038AFB0321DA1788
:103EA000C2EB610202EB42027F28A3EB8203E3DC58
:103EB000FCF7E8FBE2E7904B0493924B039306F088
:103EC000FBF8019B1B78002BCCD1049B1B78002BAB
:103ED0003FF4B8AC99F80030A3F10C007F2840F310
:103EE000BB818A488B3B80FB0320DA17C2EB600062
:103EF00000EB4000A3EB800303F17300C0B206F0B7
:103F0000DBF8019B1B78002B00F09B817E4C237813
:103F1000002B01F06882DFF80082DFF8F0A14FF09B
:103F2000000B0AE003F17300C0B206F0C5F8237875
:103F30000BF1010B5B457FF785AC58F8043F99F80E
:103F400000001844A0F18B038AFB0321DA17C2EBAF
:103F500061020C3802EB42027F28A3EB8203E1DC12
:103F6000FCF790FBE0E72046FCF78CFB53E4684A43
:103F70001278002A40F0DA825B4F5C4C3B70FEF70F
:103F800008BFFCF77FFBFFF708BA00240C706149FB
:103F900091F800A0BAF1000F3FF46CA855490191C7
:103FA0000978002900F07085019C00212170FFF73D
:103FB00061B8514B1B78002B42D099F80030A3F127
:103FC0000C007F2840F39883504A8B3B82FB0321EF
:103FD000DA17C2EB610202EB4202A3EB820303F1A8
:103FE0007300C0B206F068F8019B1B7843B3464CDF
:103FF00023782BB3484FDFF814814FF0000A09E013
:1040000003F17300C0B206F057F823780AF1010AF1
:10401000534515DD57F8043F99F800001844A0F106
:104020008B0388FB0321DA17C2EB61020C3802EB29
:1040300042027F28A3EB8203E2DCFCF723FBE1E7EB
:10404000304B1B78FBB1354B1B88012B00F0B6863B
:10405000022B00F0B687032B01F01B81042B01F02B
:10406000A581052B01F0D183062B01F0EB84072BF2
:1040700001F09885082B01F00887092B01F069876A
:104080000A2B01F04387029B1B88002B00F00F8353
:10409000174B1B78002B40F00583214B1B78002B1E
:1040A00040F0FB821F4B204A1988D6F80080002080
:1040B000012310602B6090E54B2C40F3D78018341F
:1040C000802CB8F80030194AA8BF8024A3427FF49E
:1040D00052ACFEF78CBF0130C0B2022836D828702F
:1040E0001A46FFF72CBA00BF689DFF1F5C9FFF1F99
:1040F000909FFF1FE49FFF1F459DFF1F6C9DFF1FAB
:10410000B29DFF1F3A9EFF1FE089FF1FABAAAA2A9C
:10411000D29FFF1F36A0FF1FB889FF1F529FFF1FAE
:10412000749DFF1F389EFF1F489DFF1F0CA0FF1F9F
:10413000049B1B78002B7FF4ADAB039B1B78002BFB
:104140007FF4A8AB029B1988FFF7AABB00222A7054
:104150001A46FFF7F4B9A24C2478002C7EF4A1AFE4
:1041600000287EF4B1AFBAF1000F7EF4ADAF002CA1
:104170007EF4AAAF9B49097800297EF4A8AF9A483B
:104180009A4904700C709A4F9A489B493C7004708D
:104190000C70FEF7B0BF243B002BB8F8000040F3D2
:1041A0006D8498423EF4DEAE9BB29448A8F800308D
:1041B00001230370FEF7D6BEDFF84482C0B298F840
:1041C000001005F055FFFFF77FBB8D4B387819784D
:1041D00005F04EFFDBE47F21402005F019FF894AFE
:1041E000894B3968116000221A7056E5C0B298F800
:1041F000001005F03DFFFFF7D7B87F21422005F002
:1042000007FFC1E598F80010387805F031FFB6E5F2
:104210007E4BDFF808E21978FEF7A4BE99F800009B
:1042200005F04AFF2188FFF73BBB794B02931B88BF
:10423000002B41F02A876F4B03934BE6FCF722FAE1
:10424000EEE4039B1B78002B7FF4FFAA049B1B78F2
:10425000002B7FF41FAB75E7FCF714FA4EE6FCF772
:1042600011FA31E5FCF70EFAFFF7FCB9243C002CFB
:10427000B8F8003040F31A86A3423EF4B8AEA4B2B8
:104280005E4BA8F8004001221A70FEF7B0BE421C37
:10429000D2B2022A3FF65AAF2A701A46FFF74FB938
:1042A0001446FFF75DBB7F20FFF7A2BA7F20FFF720
:1042B00040B94FF0000C8EF800C0FEF702BF00219D
:1042C0000170FEF718BF4FF0000E84F800E0FEF713
:1042D000E5BEDFF84CA13868BAF800304D4A4E4CC4
:1042E000C31A82FB031ED917C1EB6E0101EB41011A
:1042F000A3EB810303EB430354F8233018447F28D6
:1043000040F346857F3882FB0032C317C3EB62035C
:1043100003EB4303A0EB83007330DFF8E480DFF8A6
:1043200004B198F80010C0B205F0A2FEBBF800304E
:10433000022B7FF627AC3968BAF80030354ACB1A21
:1043400082FB030ED817C0EB6E0000EB4000A3EB1E
:10435000800303EB430304EB8303586808447F287E
:1043600040F330877F3882FB0032C317C3EB620211
:1043700002EB4202A0EB82007330C0B298F800104A
:1043800005F076FEBBF80030032B7FF6FBAB3968F7
:10439000BAF800301F4ACB1A82FB030ED817C0EBC5
:1043A0006E0000EB4000A3EB800303EB430304EB40
:1043B0008304A06808447F2840F3A8817F3882FBEB
:1043C0000032C317C3EB620202EB4202A0EB820091
:1043D000733098F80010C0B205F04AFEFFF7D2BB68
:1043E00033A0FF1F6C9DFF1F909FFF1FE49FFF1FC7
:1043F000459DFF1F3A9EFF1F749DFF1F759DFF1F68
:10440000C69FFF1F789DFF1FE089FF1F0BA0FF1FA6
:10441000B29DFF1FABAAAA2ABC430100D19DFF1F7A
:104420008C9FFF1FF89FFF1FDFF848A399F800003B
:10443000BAF80030C54AC64CC31A82FB031ED9170E
:10444000C1EB6E0101EB4101A3EB810303EB4303DD
:1044500054F8233018447F2840F39E847F3882FB31
:104460000032C317C3EB620303EB4303A0EB8300EB
:104470007330DFF804B3C0B205F01EFEBBF80030A5
:10448000022B7FF602AA99F80010BAF80030AF4A62
:10449000CB1A82FB030ED817C0EB6E0000EB400076
:1044A000A3EB800303EB430304EB83035868084446
:1044B0007F2840F383867F3882FB0032C317C3EB2B
:1044C000620202EB4202A0EB82007330C0B205F040
:1044D000F3FDBBF80030032B7FF6D7A999F8001045
:1044E000BAF80030994ACB1A82FB030ED817C0EBFA
:1044F0006E0000EB4000A3EB800303EB430304EBEF
:104500008304A06808447F2840F3E5807F3882FB5D
:104510000032C317C3EB620202EB4202A0EB82003F
:104520007330C0B205F0C8FDFFF7AFB9894F3878D6
:1045300002F0A8FD884B1B78002B00F0EA803B8836
:104540007E2B00F2E680854CDFF830922268D9F8A5
:104550000010521A0F2A40F2D380814A013310888A
:1045600099B23980002800F0ED80C9B2C0B205F0E0
:104570004FFD7C4F226898F80030C9F800203B704E
:10458000FEF707BC0120FFF733B9DFF8E8A1386870
:10459000BAF800306D4A6E4CC31A82FB031ED9175D
:1045A000C1EB6E0101EB4101A3EB810303EB43037C
:1045B00054F8233018447F2840F3F2837F3882FB7D
:1045C0000032C317C3EB620303EB4303A0EB83008A
:1045D0007330DFF8A4B198F80010C0B205F048FDC0
:1045E000BBF80030022B7FF6C5AB3968BAF8003053
:1045F000564ACB1A82FB030ED817C0EB6E0000EBB5
:104600004000A3EB800303EB430304EB83035868F0
:1046100008447F2840F39F867F3882FB0032C3170F
:10462000C3EB620202EB4202A0EB82007330C0B225
:1046300098F8001005F01CFDBBF80030032B7FF646
:1046400099AB3868BAF80030404AC31A82FB031E9F
:10465000D917C1EB6E0101EB4101A3EB810303EB21
:10466000430304EB8304A36818447F2841DD7F38AB
:1046700082FB0032C317C3EB620202EB4202A0EBE3
:1046800082007330C0B298F8001005F0F1FCFFF71B
:1046900071BB05F011FDFEF7EEBF0021422005F0D1
:1046A000B7FCFFE40021402005F0B2FCF5E499F8E6
:1046B000000005F001FDEBE40120FEF73ABF2A4BB4
:1046C00002931B88002B3FF4BDA8FFF7F8BB274BD4
:1046D0001A60FEF74BBEFBF7D5FF22E71D4B1F4CC0
:1046E00019886A2005F016FE98F800303B70FEF736
:1046F00050BBFBF7C7FFC5E7FBF7C4FF71E4174CDE
:10470000184F98F800303B70FEF743BBFBF7BAFF39
:104710005FE6174B1B78002BF1D03B880D4F002B29
:10472000EDD00E4CDFF854902268D9F80010521AE0
:104730000F2AE5D90A4A013B108899B2398000282E
:104740007FF413AFC8B205F003FD12E7ABAAAA2AA3
:10475000BC430100A89DFF1F37A0FF1F5C9FFF1FE8
:10476000009EFF1F689DFF1FB29DFF1F489DFF1FFA
:1047700036A0FF1F8C9FFF1FF89FFF1F18A0FF1F71
:10478000DFF834A399F80000BAF80030C64AC74CE5
:10479000C31A82FB031ED917C1EB6E0101EB410165
:1047A000A3EB810303EB430354F8233018447F2821
:1047B00040F3FE837F3882FB0032C317C3EB6203F2
:1047C00003EB4303A0EB83007330DFF8F0B2C0B219
:1047D00005F072FCBBF80030022B7FF656A899F862
:1047E0000010BAF80030B04ACB1A82FB030ED8177B
:1047F000C0EB6E0000EB4000A3EB800303EB430330
:1048000004EB8303586808447F2840F3D8857F3839
:1048100082FB0032C317C3EB620303EB4303A0EB3D
:1048200083007330C0B205F047FCBBF80030032BA7
:104830007FF62BA899F80010BAF800309A4ACB1AE4
:1048400082FB030ED817C0EB6E0000EB4000A3EB19
:10485000800303EB430304EB8304A06808447F2830
:104860007FF739AF7F3882FB0032C317C3EB620397
:1048700003EB4303A0EB8300733052E6DFF838A26A
:104880003868BAF80030884A884CC31A82FB031E85
:10489000D917C1EB6E0101EB4101A3EB810303EBDF
:1048A000430354F8233018447F2840F384837F382F
:1048B00082FB0032C317C3EB620303EB4303A0EB9D
:1048C00083007330DFF8F881DFF8F0B198F800105A
:1048D000C0B205F0CDFBBBF80030022B7FF652A929
:1048E0003968BAF80030704ACB1A82FB030ED81729
:1048F000C0EB6E0000EB4000A3EB800303EB43032F
:1049000004EB8303586808447F2840F364857F38AC
:1049100082FB0032C317C3EB620303EB4303A0EB3C
:1049200083007330C0B298F8001005F0A1FBBBF80B
:104930000030032B7FF626A93868BAF800305A4AAF
:10494000C31A82FB031ED917C1EB6E0101EB4101B3
:10495000A3EB810303EB430304EB8304A368184434
:104960007F287FF7D3AE7F3882FB0032C317C3EBBB
:10497000620303EB4303A0EB8300733029E5DFF808
:1049800038A13868BAF80030474A484CC31A82FB4D
:10499000031ED917C1EB6E0101EB4101A3EB8103AB
:1049A00003EB430354F8233018447F2840F3068375
:1049B0007F3882FB0032C317C3EB620303EB430370
:1049C000A0EB83007330DFF8F4B098F80010C0B2A9
:1049D00005F04EFBBBF80030022B7FF6CBA93968FF
:1049E000BAF80030304ACB1A82FB030ED817C0EB5E
:1049F0006E0000EB4000A3EB800303EB430304EBEA
:104A00008303586808447F2840F3E9847F3882FB99
:104A10000032C317C3EB620303EB4303A0EB830035
:104A20007330C0B298F8001005F022FBBBF80030DC
:104A3000032B7FF69FA93868BAF800301A4AC31AC8
:104A400082FB031ED917C1EB6E0101EB4101A3EB01
:104A5000810303EB430304EB8304A36818447F281A
:104A60007FF747AE7F3882FB0032C317C3EB620388
:104A700003EB4303A0EB8300733003E601283EF40D
:104A800071AA0123FFF791BB094C0A490394FEF771
:104A9000E8BA4FF47A43013BFDD199F8000005F0E4
:104AA0000BFBFFF77FB800BFABAAAA2A584701004B
:104AB0003A9EFF1F909FFF1F8C9FFF1FF89FFF1FB5
:104AC000C69FFF1FDFF8E8A23868BAF80030B64A80
:104AD000B64CC31A82FB031ED917C1EB6E0101EB62
:104AE0004101A3EB810303EB430354F82330184443
:104AF0007F2840F3E7817F3882FB0032C317C3EB86
:104B0000620202EB4202A0EB82007330DFF8A48263
:104B1000DFF8A4B298F80010C0B205F0A9FABBF80B
:104B20000030022B7FF62EA83868BAF800309E4A73
:104B3000C31A82FB0321DA17C2EB610202EB4202C5
:104B4000A3EB820303EB430304EB83035B6818448A
:104B50007F2840F310847F380C2290FBF2F302FB95
:104B600013007330C0B298F8001005F081FABBF85A
:104B70000030032B7FF606A83868BAF800308A4A5E
:104B8000C31A82FB0321DA17C2EB610202EB420275
:104B9000A3EB820303EB430304EB8304A3681844F1
:104BA0007F287FF7B3AD7F380C2290FBF2F302FB36
:104BB000130073300DE4DFF8F8A199F80000BAF89B
:104BC0000030794A794CC31A82FB031ED917C1EB16
:104BD0006E0101EB4101A3EB810303EB430354F8A6
:104BE000233018447F2840F367817F3882FB0032EE
:104BF000C317C3EB620202EB4202A0EB82007330E8
:104C0000DFF8B4B1C0B205F057FABBF80030022BA0
:104C10007EF63BAE99F80000BAF80030624AC31A3B
:104C200082FB0321DA17C2EB610202EB4202A3EB23
:104C3000820303EB430304EB83035B6818447F2880
:104C400040F390837F380C2290FBF2F302FB1300B9
:104C50007330C0B205F030FABBF80030032B7EF69B
:104C600014AE99F80000BAF800304F4AC31A82FB1C
:104C70000321DA17C2EB610202EB4202A3EB8203CB
:104C800003EB430304EB8304A36818447F287FF7F6
:104C900022AD7F380C2290FBF2F302FB130073303D
:104CA0003FE4DFF80CA13868BAF800303E4A3F4CC8
:104CB000C31A82FB031ED917C1EB6E0101EB410140
:104CC000A3EB810303EB430354F8233018447F28FC
:104CD00040F3F5807F3882FB0032C317C3EB6202DA
:104CE00002EB4202A0EB82007330DFF8CCB098F800
:104CF0000010C0B205F0BCF9BBF80030022B7FF603
:104D000039A83868BAF80030274AC31A82FB032151
:104D1000DA17C2EB610202EB4202A3EB820303EB60
:104D2000430304EB83035B6818447F2840F32A8322
:104D30007F380C2290FBF2F302FB13007330C0B2F9
:104D400098F8001005F094F9BBF80030032B7FF6BB
:104D500011A83868BAF80030134AC31A82FB03213D
:104D6000DA17C2EB610202EB4202A3EB820303EB10
:104D7000430304EB8304A36818447F287FF7B9AC8E
:104D80007F380C2290FBF2F302FB1300733079E4BE
:104D9000FBF778FCFFF7C1BAFBF774FCFFF769BBC0
:104DA000FBF770FC15E400BFABAAAA2AE847010094
:104DB0008C9FFF1FC69FFF1FF89FFF1FDFF82CA3CC
:104DC00099F80000BAF80030C34AC44CC31A82FBF9
:104DD0000317D917C1EB670101EB4101A3EB810375
:104DE00003EB430354F8233018447F2870DD7F38E9
:104DF00082FB0032C317C3EB620202EB4202A0EB5C
:104E000082007330DFF8E8B2C0B205F055F9BBF8A4
:104E10000030022B7FF637A999F80000BAF800306D
:104E2000AD4AC31A82FB0321DA17C2EB610202EB1F
:104E30004202A3EB820303EB430304EB83035B68AF
:104E400018447F2840F39B827F380C2290FBF2F3BA
:104E500002FB13007330C0B205F02EF9BBF800302E
:104E6000032B7FF610A999F80000BAF800309A4A8F
:104E7000C31A82FB0321DA17C2EB610202EB420282
:104E8000A3EB820303EB430304EB8304A3681844FE
:104E90007F281ADD7F380C2290FBF2F302FB13000F
:104EA0007330C0B205F008F9FFF7EDB8012B3EF4FE
:104EB0009EA80124FFF7E4B9FBF7E4FBA0E6FBF7AB
:104EC000E1FB12E7FBF7DEFB20E6FBF7DBFBE8E7A5
:104ED000FBF7D8FB96E7DFF814A23868BAF8003081
:104EE0007D4A7F4CC31A82FB031ED917C1EB6E01AA
:104EF00001EB4101A3EB810303EB430354F823309F
:104F000018447F28DEDD7F3882FB0032C317C3EBF5
:104F1000620303EB4303A0EB83007330F6E5DFF895
:104F2000CCA199F80000BAF800306B4A6C4CC31A57
:104F300082FB031ED917C1EB6E0101EB4101A3EB0C
:104F4000810303EB430354F8233018447F28B3DD77
:104F50007F3882FB0032C317C3EB620303EB4303CA
:104F6000A0EB830073304BE6DFF880A13868BAF815
:104F70000030594A5A4CC31A82FB031ED917C1EBA1
:104F80006E0101EB4101A3EB810303EB430354F8F2
:104F9000233018447F2892DD7F3882FB0032C3170C
:104FA000C3EB620303EB4303A0EB830073309CE687
:104FB000FBF768FB09E4FBF765FB83E4FBF762FBA7
:104FC00001E5DFF828A199F80000BAF80030424A5C
:104FD000444CC31A82FB0317D917C1EB670101EBDD
:104FE0004101A3EB810303EB430354F8233018443E
:104FF0007F287FF76DAF7F3882FB0032C317C3EB8A
:10500000620303EB4303A0EB83007330FAE6DFF89F
:10501000DCA03868BAF800302F4A334CC31A82FB40
:105020000321DA17C2EB610202EB4202A3EB820317
:1050300003EB430354F8233018447F2840F398814E
:105040007F380C2290FBF2F302FB13007330DFF881
:10505000A480DFF89CB098F80010C0B205F008F802
:10506000BBF80030022B1AD93868BAF800300C228D
:10507000C11A91FBF2F302FB131302FB03435B68BB
:1050800018447F2840F353847F3890FBF2F302FBEF
:1050900013007330C0B298F8001004F0E9FFBBF8B9
:1050A0000030032B7EF66EADBAF8003038680C2263
:1050B000C11A91FBF2F302FB131302FB0344A36832
:1050C00018447F287FF722AB7F3890FBF2F302FB76
:1050D00013007330FFF77DB9ABAAAA2ABC430100C5
:1050E0009440010058470100E84501008C9FFF1FD4
:1050F000F89FFF1FC69FFF1FDFF814A399F8000059
:10510000BAF80030BD4ABE4CC31A82FB0321DA173D
:10511000C2EB610202EB4202A3EB820303EB430307
:1051200054F8233018447F2840F319817F380C222B
:1051300090FBF2F302FB13007330DFF8D8B2C0B279
:1051400004F0BAFFBBF80030022B19D999F800001F
:10515000BAF800300C22C11A91FBF2F302FB1313D0
:1051600002FB03435B6818447F2840F3E7837F38E2
:1051700090FBF2F302FB13007330C0B204F09CFF0B
:10518000BBF80030032B7EF680ABBAF8003099F8FC
:1051900000000C22C11A91FBF2F302FB131302FB75
:1051A0000344A36818447F287FF795AA7F3890FBB3
:1051B000F2F302FB13007330FFF7B3B9FBF762FAA7
:1051C000FFF784B9FBF75EFAFFF7D7B8DFF840A224
:1051D0003868BAF80030894A894CC31A82FB032127
:1051E000DA17C2EB610202EB4202A3EB820303EB8C
:1051F000430354F8233018447F2840F3B6807F38A7
:105200000C2290FBF2F302FB13007330DFF804B2C0
:1052100098F80010C0B204F02BFFBBF80030022B4E
:105220001AD93868BAF800300C22C11A91FBF2F38F
:1052300002FB131302FB03435B6818447F2840F30F
:105240007A837F3890FBF2F302FB13007330C0B215
:1052500098F8001004F00CFFBBF80030032B7EF62A
:1052600089ADBAF8003038680C22C11A91FBF2F30C
:1052700002FB131302FB0344A36818447F287FF743
:1052800038AA7F3890FBF2F302FB13007330FFF76C
:10529000F9B9DFF87CA199F80000BAF80030574A54
:1052A000584CC31A82FB0321DA17C2EB610202EBEE
:1052B0004202A3EB820303EB430354F82330184468
:1052C0007F2845DD7F380C2290FBF2F302FB1300B0
:1052D0007330DFF840B1C0B204F0EEFEBBF800302E
:1052E000022B18D999F80000BAF800300C22C11A24
:1052F00091FBF2F302FB131302FB03435B681844B8
:105300007F2877DD7F3890FBF2F302FB13007330C8
:10531000C0B204F0D1FEBBF80030032B7EF6B3AE72
:10532000BAF8003099F800000C22C11A91FBF2F390
:1053300002FB131302FB0344A36818447F287FF782
:10534000C4AD7F3890FBF2F302FB13007330A8E585
:10535000FBF798F9BDE7FBF795F9FFF768B9FBF79D
:1053600091F9EAE6FBF78EF973E4FBF78BF94DE769
:10537000FBF788F96BE6FBF785F9FFF7F3BBFBF763
:1053800081F968E5FBF77EF9D9E4DFF884A0386895
:10539000BAF80030194A1C4C40E6DFF874A099F8BE
:1053A0000000BAF80030154A174CADE6DFF860A0EF
:1053B00099F80000BAF80030104A144C71E7FBF776
:1053C00061F9FFF72FBADFF848A03868BAF8003063
:1053D0000A4A0D4C01E7FBF755F9FFF7A3BAFBF7B3
:1053E00051F9FFF71EBB039B1B78002B7EF42DAAFF
:1053F000FEF750BAFBF746F98AE700BFABAAAA2A24
:10540000E8450100E8470100DC4801009440010044
:105410008C9FFF1FF89FFF1FA54C2388002B00F0D7
:105420008783A44ADFF8A0B21288BBF800100332C9
:10543000914228DDA0493868A04A0988B2F800E006
:10544000DFF87CC2411A0C2291FBF2F902FB191120
:105450004FF0900909FB0EFE02FB01E16FF00B0E0D
:105460005CF8011001440EFB03107F2840F33784E1
:105470007F3890FBF2F302FB13007330C0B298F850
:10548000001004F0F5FDBBF8002023881344022B24
:1054900023DD894B894A38681B88B2F800C0DFF8E1
:1054A00020E2C31A0C2193FBF1F201FB123290238C
:1054B00003FB0CF301FB023373445B6818447F2841
:1054C00040F3C3857F3890FBF1F301FB1300733089
:1054D000C0B298F8001004F0CBFDBBF80020238880
:1054E0001344032B23DD744B744A38681B88B2F8CD
:1054F00000C0DFF8CCE1C31A0C2193FBF1F201FBF1
:105500001232902303FB0CF301FB023373449B68BC
:1055100018447F2840F39D857F3890FBF1F301FB11
:1055200013007330C0B298F8001004F0A1FDBBF86E
:10553000002023881344042B7EF71CAC5D4B1B8892
:10554000012B7EF417AC3A68A2F10C007F287FF79C
:10555000D0A88B3A0C2092FBF0F300FB13207330A1
:10556000FFF790B8524C2388002B40F0D682DFF82A
:1055700058B15149514A0988D7F80080B2F800E083
:105580004F48C1EB080C0C229CFBF2F102FB11C14D
:105590004FF0900C0CFB0EFE02FB01E16FF00B0EC6
:1055A000405880440EFB03807F2840F39583A0F190
:1055B0007F0393FBF2F002FB10307330414BC0B21B
:1055C000197804F055FDBBF8002023881344022B02
:1055D00023DD394A394B11883868B3F800C0DFF849
:1055E000E0E0411A0C2291FBF2F302FB131190232D
:1055F00003FB0CF302FB013373445B6818447F2800
:1056000040F374847F3890FBF2F302FB1300733095
:105610002C4BC0B2197804F02BFDBBF80020238876
:105620001344032B23DD244A244B11883868B3F834
:1056300000C0DFF88CE0411A0C2291FBF2F302FB70
:105640001311902303FB0CF302FB013373449B689B
:1056500018447F2840F3E3847F3890FBF2F302FB89
:1056600013007330174BC0B2197804F001FDBBF87A
:10567000002023881344042B7EF784AA0D4B1B883B
:10568000012B7EF47FAA3A68A2F10C007F2840F338
:10569000B7818B3A0C2092FBF0F300FB13207330A0
:1056A000084BC0B2197804F0E3FCFEF76BBA00BFF8
:1056B000149EFF1FA69DFF1F8C9FFF1F3E9FFF1F75
:1056C00024410100C69FFF1FF89FFF1FCE4C238877
:1056D000002B40F0BF81DFF864B3CC49CC4A098885
:1056E00099F80000B2F800E0DFF85483C1EB000C39
:1056F0000C229CFBF2F102FB11C14FF0900C0CFB51
:105700000EFE02FB01E16FF00B0E58F80110084489
:105710000EFB03007F2840F36E83A0F17F0393FB11
:10572000F2F002FB10307330C0B204F0C5FCBBF8DD
:10573000002023881344022B22DDB44AB44B118885
:1057400099F80000B3F800C0DFF8F4E2411A0C2227
:1057500091FBF2F302FB1311902303FB0CF302FB0A
:10576000013373445B6818447F2840F35C847F38BE
:1057700090FBF2F302FB13007330C0B204F09CFC08
:10578000BBF8002023881344032B22DD9F4AA04B43
:10579000118899F80000B3F800C0DFF8A4E2411ABC
:1057A0000C2291FBF2F302FB1311902303FB0CF389
:1057B00002FB013373449B6818447F2840F39D83A8
:1057C0007F3890FBF2F302FB13007330C0B204F099
:1057D00073FCBBF8002023881344042B7EF755A8E4
:1057E0008C4B1B88012B7EF450A899F80020A2F165
:1057F0000C007F287EF76FAF8B3A0C2092FBF0F302
:1058000000FB13207330FEF78CBEDFF800A299F87E
:105810000000BAF80030804CC11A0C2291FBF2F360
:1058200002FB131302FB03F3E35818447F287FF7AE
:105830008FAD7F3890FBF2F302FB1300733048E525
:10584000764B1A88182A13D03B681344A3F118002A
:105850007F2840F34F830C20973B93FBF0F200FB33
:10586000123303F173006E4BC0B2197804F000FCE0
:105870006C4B6D491A78022A94BF013200221A70CB
:105880001A7831F81200182810D10424022A02F1E3
:105890000100C2B288BF002231F81200182804D1DA
:1058A000013CF3D11A70FEF76DB91A703B680344DE
:1058B000A3F118007F2840F3A3800C20973B93FBB3
:1058C000F0F200FB123303F17300E9E6534B1B883F
:1058D000182B12D099F800201344A3F118007F2848
:1058E00040F334830C20973B93FBF0F200FB123320
:1058F00003F17300C0B204F0DFFB4A4A4A4B12784E
:1059000033F81230182B3DF4C0AF99F8002013443F
:10591000A3F118007F287EF7DEAE0C20973B93FBA7
:10592000F0F200FB123303F17300FEF7FABDFAF751
:10593000A9FEFFF7AFBBFAF7A5FE88E4FAF7A2FECF
:105940001BE43A4B1B78002B00F05882384B1B7835
:10595000002B7DF44CAB374B1B78002B3DF447AB51
:10596000B8F8003034490A3BA8F800300A70FDF757
:105970003EBB2A4B1A88182A13D03B681344A3F164
:1059800018007F2840F3BC820C20973B93FBF0F279
:1059900000FB123303F17300C0B298F8001004F05A
:1059A00067FB204B20491A78022A94BF013200225B
:1059B0001A701A7831F81200182810D10424022A1B
:1059C00002F10100C2B288BF002231F8120018288B
:1059D00004D1013CF3D11A70FEF7CCB91A703B68C0
:1059E0000344A3F118007F287EF783AE0C20973B79
:1059F00093FBF0F200FB123303F17300FEF742BE9B
:105A0000FAF740FE4CE600BF149EFF1F8C9FFF1F5D
:105A10003E9FFF1FA69DFF1FE8450100E29FFF1F5D
:105A2000C69FFF1F188AFF1FA89FFF1F33A0FF1FDD
:105A300034A0FF1F35A0FF1F759DFF1FF89FFF1F9C
:105A400024410100DFF828A399F80000BAF80030DB
:105A5000C04CE1E6C04ADFF82CB31288BBF8001056
:105A6000033291427FF763AE37E6BC4B1B88182B9D
:105A700012D099F800201344A3F118007F2840F3B6
:105A800042820C20973B93FBF0F200FB123303F1B0
:105A90007300C0B204F010FBB14AB24B127833F875
:105AA0001230182B7FF431AFFDF7EFBEAB4B1A88E5
:105AB000182A13D03B681344A3F118007F2840F341
:105AC000AB820C20973B93FBF0F200FB123303F107
:105AD0007300C0B298F8001004F0CAFAA04BA149B4
:105AE0001A78022A94BF013200221A701A7831F80B
:105AF000120018287FF473AF0424022A02F1010275
:105B000094BFD2B2002231F8120018287FF466AF99
:105B1000013CF2D11A70FEF72DB98F4ADFF864B25A
:105B20001288BBF80010033291427FF74CAD20E59C
:105B3000DFF850B27EE4894B1A88182A13D03B68EC
:105B40001344A3F118007F2840F323820C20973BD5
:105B500093FBF0F200FB123303F17300824BC0B2EF
:105B6000197804F085FA7E4B7E491A78022A94BF90
:105B7000013200221A701A7831F8120018287FF4C6
:105B800095AE0424022A02F1010294BFD2B200228F
:105B900031F8120018287FF488AE013CF2D11A7057
:105BA000FDF7F0BF714C2388002B40F04382DFF8F3
:105BB000D4B16F4999F800006E4A09881788DFF858
:105BC000B8E1411A0C2291FBF2FC02FB1C114FF0D0
:105BD000900C0CFB07F702FB01716FF00B075EF8EE
:105BE0000110014407FB03107F2840F320827F3817
:105BF00090FBF2F302FB13007330C0B204F05CFAC6
:105C0000BBF8002023881344022B21DD584B594A4E
:105C100099F800001B88B2F800E0574FC31A0C2116
:105C200093FBF1F201FB1232902303FB0EF301FB15
:105C300002333B445B6818447F2840F314827F386A
:105C400090FBF1F301FB13007330C0B204F034FA9F
:105C5000BBF8002023881344032B21DD444B454A25
:105C600099F800001B88B2F800E0434FC31A0C21DA
:105C700093FBF1F201FB1232902303FB0EF301FBC5
:105C800002333B449B6818447F2840F3E6817F3809
:105C900090FBF1F301FB13007330C0B204F00CFA77
:105CA000BBF8002023881344042B7EF7ECA92A4B71
:105CB0001B88012B7EF4E7A999F80020A2F10C00C3
:105CC0007F287FF702A98B3A0C2092FBF0F300FBB0
:105CD00013207330FFF7E5B8FAF7D4FC6EE4FAF757
:105CE000D1FCFFF7CBBB254B1A88182A13D03B6891
:105CF0001344A3F118007F2840F3BE810C20973B8A
:105D000093FBF0F200FB123303F17300C0B298F87A
:105D1000001004F0ADF9124B19491A78022A94BF09
:105D2000013200221A701A7831F8120018287FF414
:105D300056AE0424022A02F1010294BFD2B200221C
:105D400031F8120018287FF449AE013CF2D11A70E4
:105D5000FEF710B8DC480100A69DFF1F9E9DFF1FA7
:105D6000188AFF1F209FFF1FC69FFF1F149EFF1F43
:105D70008C9FFF1F3E9FFF1F24410100A09DFF1F1E
:105D8000289FFF1FF89FFF1FC24B1A88182A13D0A5
:105D90003B681344A3F118007F2840F36A810C206C
:105DA000973B93FBF0F200FB123303F17300BA4B05
:105DB000C0B2197804F05CF9B84BB9491A78022AD4
:105DC00094BF013200221A701A7831F81200182894
:105DD0007FF46CAD0424022A02F1010294BFD2B216
:105DE000002231F8120018287FF45FAD013CF2D197
:105DF0001A70FDF7C7BEFAF745FC95E4A94B1B786E
:105E0000002B7DF4F4A8A84B1B78002B3DF4EFA8E1
:105E1000B8F80030A549013BA8F800300A70FDF73A
:105E2000E6B89C4B1B88182B12D099F8002013441D
:105E3000A3F118007F2840F313810C20973B93FBBC
:105E4000F0F200FB123303F17300C0B204F034F936
:105E5000924A934B127833F81230182B7FF455ADD9
:105E6000FDF713BD8F4B1B78002B7DF495AD8E4B4A
:105E70001B78002B3DF4BBA8B8F800308B490133E8
:105E8000A8F800300A70FDF7B2B8894B1B88182BB0
:105E900012D099F800201344A3F118007F2840F392
:105EA000E5800C20973B93FBF0F200FB123303F1EB
:105EB0007300C0B204F000F9784A7E4B127833F8D0
:105EC0001230182B3EF4DFA899F800201344A3F1F8
:105ED00018007F287EF7F9AF0C20973B93FBF0F278
:105EE00000FB123303F17300FEF7DBBFFAF7CAFBC6
:105EF000FFF78EBBFAF7C6FBB5E4FAF7C3FB65E420
:105F0000FAF7C0FB48E5FAF7BDFBC2E5614B1B8819
:105F1000182B12D099F800201344A3F118007F2801
:105F200040F3AD800C20973B93FBF0F200FB123363
:105F300003F17300C0B204F0BFF8584A584B12780E
:105F400033F81230182BBFD1FEF79DB8FAF79AFB41
:105F5000D0E4594B1B88182B12D099F80020134419
:105F6000A3F118007F2840F38D800C20973B93FB12
:105F7000F0F200FB123303F17300C0B204F09CF89E
:105F8000464A4E4B127833F81230182B9CD1FEF74C
:105F90007AB8FAF777FBE1E5494B00227F21072029
:105FA0001A8004F035F87F210B2004F031F8FDF75A
:105FB00026BD444B01227F2107201A8004F028F8D7
:105FC0007F210B2004F024F8FDF711BD3E4B042285
:105FD0007F2107201A8004F01BF800210B2004F019
:105FE00017F8FDF7FDBC384B02227F2107201A80ED
:105FF00004F00EF87F210B2004F00AF8FDF7EBBC4B
:10600000314B002107201C8004F002F87F210B2077
:1060100003F0FEFFFDF7DABCFAF734FB59E5FAF7B7
:1060200031FBFFF71FBBFAF72DFBFFF7A6BBFAF713
:1060300029FBE2E5254ADFF89CB01288BBF8001086
:10604000033291427FF7DCADB3E5FAF71BFBFFF7B4
:106050003FBAFAF717FBFFF765BAFAF713FB1CE62E
:10606000FAF710FBF1E6FAF70DFBEEE5FAF70AFB9B
:106070001FE7FAF707FB9AE6FAF704FB46E6FAF79A
:1060800001FB57E7FAF7FEFA77E7114B0393FDF7A9
:1060900016BF00BFA09DFF1FC69FFF1F188AFF1FCE
:1060A000289FFF1F34A0FF1F35A0FF1F759DFF1FF6
:1060B000E29FFF1FA89FFF1F9E9DFF1F209FFF1FA6
:1060C0006A9DFF1F2A9EFF1F849FFF1FA69DFF1F23
:1060D0003A9EFF1FF89FFF1F38B508F017FB0E48C8
:1060E00005F016FF0D4805F013FF0D4805F010FFF1
:1060F00000234FF07E5201210A48FAF7B7F90A4B04
:106100000A4A0B49802400251C7118461D60BDE811
:1061100038400BF013BE00BF889DFF1FBC9DFF1FC2
:10612000309EFF1F609FFF1FF09FFF1F1C89FF1FF6
:106130002906000010B50446A4206368198804F0FD
:10614000E9F8E368A6201988BDE8104004F0E2B839
:1061500043682A20198804F0DDB800BF10B5044652
:1061600022206368198804F0D5F8E3682420198890
:10617000BDE8104004F0CEB810B504460A206368AC
:10618000198804F0C7F8E3680C201988BDE81040AE
:1061900004F0C0B810B5044606206368198804F0FE
:1061A000B9F8E36808201988BDE8104004F0B2B8D7
:1061B00010B5044602206368198804F0ABF8E36860
:1061C00004201988BDE8104004F0A4B870B50E4C46
:1061D00084B0122504220123064603900293204630
:1061E0008DE824001423102107F03CFD062209232A
:1061F000029303960195204600921423102107F084
:1062000031FD04B070BD00BF64A0FF1FF8B5B04CF5
:10621000B4F90030032B00F01281002B6AD0022B5E
:1062200000F08A80052B00F0B580012B00F0DD80A6
:10623000042B00D0F8BDA74FA74E00254FF4AF7434
:10624000E9B2A64805F08EFE57F8043BC3F59673F5
:1062500000FB03F086FB0023C017C0EB63108442F1
:1062600005F10105A8BF0446062DE9D19C4F9A4EC1
:106270000025E9B29B4805F075FE57F8043BC3F5CD
:10628000967300FB03F086FB0023C017C0EB63107E
:10629000844205F10105A8BF04460C2DE9D1924FB7
:1062A0008D4E0025E9B2914805F05CFE57F8043B9D
:1062B000894AC3F5967300FB03F086FB0013C017F1
:1062C000C0EB6310844205F10105A8BF04460C2D04
:1062D000E8D1A4F11401312900F3A38040F26C72DB
:1062E00032218348834B01801A602A20BDE8F840A0
:1062F00004F010B80E2008F06DF940F6FF71C830B8
:106300008842A8BF084620EAE07000F2DC5283B25F
:106310008A42794D794EA8BF0A4602201946338039
:106320002A8003F0F7FF2988042003F0F3FFB4F973
:106330000030022B7FF476AF012009F0E7FC054620
:10634000002009F0E3FCA842B8BF284600F1C801CC
:10635000B1F5FA7FC0F2B480B1F57A6FA8BF4FF4FF
:106360007A6101F54873B3F57A6FA8BF4FF47A6389
:106370009BB289B2624A634D11800A202B8003F0E0
:10638000C9FF29880C2003F0C5FFB4F90030052BA4
:106390007FF44BAF0F2009F0B9FCC0F53F63043325
:1063A000B3F5AF6FC0F28980B3F5FA6FA8BF4FF4B1
:1063B000FA6399B2544BC0F54360B0F5AF6F1980E2
:1063C00061DBB0F5FA6FA8BF4FF4FA6083B24F4DAE
:1063D000A4202B8003F09EFF2988A62003F09AFFBB
:1063E000B4F90030012B7FF423AF152008F0F2F848
:1063F00000F59671B1F52F7F4DDB41F25C23994298
:1064000063DC434A00F5617089B2B0F52F7F1180DB
:10641000B8BF4FF42F7344DB8342A8BF03469BB23F
:106420003FE040F23A73A4F5B97403FB04F482FB35
:106430000432E417A4EB621289B2323251E7102021
:1064400009F064FCC830B0F5FA7F1FDBB0F57A6F55
:106450000146A8BF4FF47A6101F51673B3F57A6F60
:10646000A8BF4FF47A639BB289B22A4A2A4D1180A1
:1064700022202B8003F04EFF2988242003F04AFFBE
:10648000B4F90030C9E64FF4AF63A0E740F24C43E3
:106490004FF4FA71E9E740F214534FF42F711C4A9C
:1064A00011801E4D06202B8003F034FF2988082020
:1064B00003F030FFB4F90030BAE64FF4AF6179E78A
:1064C00040F214534FF4FA7154E71946E7E700BF5E
:1064D00042A0FF1F688AFF1FB5814E1B889DFF1FCA
:1064E000388AFF1FBC9DFF1F4089FF1F309EFF1F82
:1064F000FA9FFF1F248AFF1F5C9DFF1F389EFF1F0E
:10650000989FFF1F9C9DFF1F3C9EFF1FB89FFF1F72
:10651000DC9DFF1F4C9FFF1F489FFF1FCC9FFF1F4D
:106520002DE9F041224D82B0012602B284B20092E0
:10653000284601967823192107F0DAFA04F10C02B3
:1065400012B28DE844002846A7197823192104F1D6
:10655000020807F0CDFA3FB20FFA88F819233A463D
:10656000284619460196CDF8008007F0C1FA782335
:106570003A4628461946CDF80080019604F10A07EC
:106580000B3407F0B5FA3FB224B278233A462846D6
:1065900019468DE8500007F0ABFA192300943A46EB
:1065A00001962846194607F0A3FA02B0BDE8F0812B
:1065B00064A0FF1F30B583B000230C4605B20093E2
:1065C00026225B231C210C4806F0E2FF294601230A
:1065D0002622094806F0F8FA002C24B205DB2146F1
:1065E00001232622044806F0EFFA044A044B1580E2
:1065F0001C8003B030BD00BF64A0FF1F828AFF1F54
:10660000848AFF1F2DE9F041BB4C237882B01BB177
:10661000BA4B4FF6FF721A80B94BB3F90030CBB9C1
:10662000B84AB64B1068B3F9002080F30C005B2326
:1066300003FB00F000131C3082424BD04FF0FF31BF
:10664000FFF7B8FFB04807F007F80023237002B047
:10665000BDE8F081012B1BD0022B5AD0032B3FD079
:10666000042B00F09980052BEFD10F2009F04EFB91
:10667000C0F53B600830B0F5AF6F48DBB0F5FA6F9E
:10668000A8BF4FF4FA60A0F5AF625B239F4835E0E6
:106690009F4B1B78002B75D0152007F09BFF9D4B5F
:1066A0001860B0F52F7F32DB41F25C239842A8BF1F
:1066B0001846A0F52F735B22974802FB03F380FB7B
:1066C0000320DB17C3EBA0201C308C4BB3F9003048
:1066D0008342B3D1914BB3F900300133AED1B4E76B
:1066E0008F4B1B68B3F5FA7F11DBB3F57A6FA8BF48
:1066F0004FF47A638B48A3F5FA725B2303FB02F332
:1067000080FB0320DB17C3EB20201C30DDE71C20BF
:10671000DBE7854B1B68B3F5FA7F3BDBB3F57A6F9C
:10672000A8BF4FF47A63A3F5FA727E485B2303FB9C
:1067300002F380FB0320DB17C3EB20201C307B4BD4
:106740001B68B3F5FA7F23DBB3F57A6FA8BF4FF46C
:106750007A63A3F5FA7273495B2303FB02F381FBAF
:106760000321DB17C3EB21211C31644BB3F900304B
:1067700083427FF465AF694BB3F900308B427FF4FD
:106780005FAF62E7112009F0C1FA624B186088E739
:106790001C21EAE71C20D2E7252200258DE82400F1
:1067A00076231C215848624E624FDFF8A08107F023
:1067B0009FF916E0B0F5AF7FA8BF4FF4AF70323845
:1067C00002FB00F088FB0031C017C0EB61111C31E7
:1067D00009B201231D4425224B4806F0F5F90C2D82
:1067E00014D0E9B2544805F0BDFB56F8043BC3F59C
:1067F000967300FB03F087FB0013C017C0EB631018
:1068000031284FF05B02D5DC1C21E2E7262200256F
:106810008DE8240076231C213B48484E454FDFF885
:106820002C8107F065F916E0B0F5AF7FA8BF4FF4F3
:10683000AF70323802FB00F088FB0031C017C0EBAC
:1068400061111C3109B201231D4426222E4806F095
:10685000BBF90C2D14D0E9B2394805F083FB56F88A
:10686000043BC3F5967300FB03F087FB0013C017CE
:10687000C0EB631031284FF05B02D5DC1C21E2E74E
:10688000272200258DE8240076231C211E482D4E4A
:10689000284FDFF8B88007F02BF917E0B0F5AF7F8D
:1068A000A8BF4FF4AF70323802FB00F088FB003114
:1068B000C017C0EB61111C3109B201231D4427220E
:1068C000114806F081F9062D3FF4BCAEE9B21E482E
:1068D00005F048FB56F8043BC3F5967300FB03F044
:1068E00087FB0013C017C0EB631031284FF05B0229
:1068F000D4DC1C21E1E700BF3CA0FF1F828AFF1F00
:1069000042A0FF1F9C9FFF1F64A0FF1F37800B6DDD
:10691000549FFF1F549DFF1FD3058541848AFF1F8D
:10692000AC9DFF1F011FB812B89DFF1F7C9DFF1F6C
:10693000388AFF1FB5814E1BBC9DFF1F4089FF1F7A
:10694000309EFF1F688AFF1F889DFF1F4B48371B23
:106950002DE9F043754C054683B02046D5F80080FC
:10696000EE6806F06DFD1120FFF7DAFD012719230F
:106970004FF028091946204601972422CDF80090AF
:1069800007F0B6F878231946242201972046CDF85F
:10699000009007F0ADF83946204607F033FC02239B
:1069A000192240462382E2810CF08AFF41460246CA
:1069B00020460AF055FE20460AF068FE0027142300
:1069C00003225B4923822046E7810AF049FE2046E4
:1069D0000AF05CFE2323204603225649E7812382E6
:1069E0000AF03EFE20460AF051FE6EB12F20FFF75E
:1069F00097FD322303225049E781204623820AF083
:106A00002FFE20460AF042FE01234C4A184613701E
:106A1000FFF7DCFB29896A896B68521A1B885C2A9C
:106A2000A3EB010357DD03EB43030132C3EB431335
:106A300093FBF2F303F11B023C4FDFF80CE113B2BE
:106A40001A214FF001088DE802013846AEF8002007
:106A50001946142207F04CF8002E4ED0298A6B8A72
:106A6000EA685B1A5C2B12883DDC511A5C2202FB3F
:106A700001F292FBF3F31B33314A2C4813800126B9
:106A80001BB2382219468DE84400322207F030F854
:106A90000022402309218DE806002448194606F00B
:106AA000F5FF3146214807F0ADFB6B681F48022215
:106AB00044212282E18119880AF038FE32462149B8
:106AC0001A480AF0CDFDEB681848198803B0BDE8F4
:106AD000F0430AF02BBE5C2101FB03F393FBF2F3BE
:106AE00003F11B02A8E7521A02EB4202C2EB421268
:106AF000434492FBF3F31B33BEE7402309213246A4
:106B0000009138461946019606F0C0FF41463846C6
:106B100007F078FB6B6868210222F9813A821988B4
:106B2000384603B0BDE8F0430AF000BE64A0FF1F82
:106B3000444A0100484A01004C4A0100F1A0FF1FED
:106B400040A0FF1F504A01003EA0FF1F2DE9F04F5B
:106B50001F4685B01446002A4ED0052A0646D0F8B6
:106B60000C8000F0AB800F9B8C4A00EBC305012C1E
:106B7000B5F80AE029896868C1EB0E0382FB03C2FD
:106B80001A444FEAE373C3EBA213028851D0042CDA
:106B900000F08D80824D00220921402328468DE897
:106BA0000600194606F072FF2846012107F02AFB6D
:106BB000B8F1000F00F0E8807368022244212A82B5
:106BC000E981198828460AF0B1FD76490122284654
:106BD0000AF046FDF368284619880AF0A7FD724BB3
:106BE000022CB3F9001000F0AD80082C00F0C98031
:106BF000012005B0BDE8F08F6C4E6D4A3368126815
:106C0000CB1A93420D4655D96A4A3B88117864489D
:106C1000012918BF012414700E9A06321BB212B259
:106C20008DE814001946BDF9382006F061FF356083
:106C3000DEE79BB2D31A994203DC9E457146A8BF9A
:106C400019460E9A0180B7F90030BDF938A05448B2
:106C500002F106094FF0000E0FFA89F91946524663
:106C6000CDF80090CDF804E006F042FF29896A894A
:106C70006868521A03885C2AA3EB01037ADD03EBF0
:106C800043030132C3EB431393FBF2F303F11B0203
:106C900013B201203A80194652460190CDF8009077
:106CA0003F4806F025FF434B00221A7072E712FAA4
:106CB00083F3C0E7204605B0BDE8F08F384D4FF0B4
:106CC000070A4FF0000B28465A2323228DE8000CB8
:106CD0001A2106F0DBFE2846012107F093FA4FF057
:106CE00001094FF0350E2323A5F80EE052462B8202
:106CF0003149A5F814902846A5F8129003930AF09C
:106D0000AFFC28460AF0C2FC284606F0A5FC4FF46A
:106D1000FA6008F0E9F8FFF779FA039B1A211A469E
:106D200028465A238DE8000C06F0B0FE284606F0EF
:106D300093FC3046FFF70CFE204B83F80090FFF7E2
:106D400061FC27E74A1C12B21A8091423FF450AF0F
:106D50000E9AB7F9003012480632012412B200929E
:106D600019460194BDF9382006F0C2FE204605B050
:106D7000BDE8F08F5C2101FB03F393FBF2F21B32C1
:106D800086E700221A80E0E7736868210222E98121
:106D90002A82198828460AF0C9FC20E7C94216B29F
:106DA00064A0FF1F504A010046A0FF1FCCA0FF1F98
:106DB000385B0100F1A0FF1F544A01003CA0FF1FF7
:106DC0002DE9F04F5A4E5B4DB6F900704C7855F8EE
:106DD000277085B08146984604B10C78DFF874A11D
:106DE0001AB99AF80030002B39D0534D0023384699
:106DF0002B808AF80030FFF7ABFD504A504BB5F9B5
:106E00000000012111704FF6FF721A8060B3012853
:106E10005ED0012032232246019000934946494B1F
:106E20003846FFF793FE00240346B5F90020022AF6
:106E300039DD00222A80B6F900203D49002A3BDBDB
:106E4000052AC4BF00220A80B8F1000F39D1002CF6
:106E50000CBF18464FF0FF3005B0BDE8F08F364D3F
:106E6000B5F900000028D2D1DFF8ECB0364ADBF8E3
:106E700000301268C3EB0903934227D9334B1A78C9
:106E8000012A18BF01201870FFF7A0F90123CBF8E1
:106E90000090012C2AD0042C35D0022C3AD0082C9A
:106EA0003ED00024C1E7C6D1FA68002AC1D0B6F9A5
:106EB00000201F49002AC3DA05220A80B8F1000F1A
:106EC000C5D00393FFF79EFB039BC0E70346E0E7B3
:106ED0004FF0000E142322468DE8084049461C4B13
:106EE00038467446FFF732FE03469EE732888AF83A
:106EF0000040013232807A6982B10024384603931F
:106F00009047039B91E732880121013A32808AF849
:106F10000010F0E701222A8000248CE7144684E761
:106F20007A69002129804FF0FF34002AE6D182E7F8
:106F300042A0FF1F888AFF1F46A0FF1F3CA0FF1F23
:106F4000828AFF1F40A0FF1F385B0100F1A0FF1FD6
:106F50003EA0FF1F44A0FF1FCCA0FF1F01210D205A
:106F600007F086BF00210D2007F082BF01460D20EB
:106F700007F07EBF08B50D2007F080FFB0FA80F162
:106F800049090D20BDE8084007F072BF10B5002187
:106F900044080D2007F06CFF204607F0A5FF0D20E8
:106FA000012107F065FF2046BDE8104007F09CBFB7
:106FB0002D4A2E4B10881B68984210B549DA2C4A8E
:106FC0001288141A9A42A8BF1A46B4F5157F36DA09
:106FD000121A40F2532303FB02F393FBF4F1053141
:106FE0000A2007F0B5FD234B1978C9B3224B23497A
:106FF0001B6840F2271283F3070302FB03F381FBB4
:1070000003211944DB17C3EBA1110531092007F057
:107010009FFD1B4B1968F1B181F3070140F2271264
:10702000164802FB01F380FB03211944DB17C3EB75
:10703000A11105311620BDE8104007F089BD131AD3
:107040004FF41572611C02FB03F393FBF1F1053160
:10705000C6E70021C4E71620BDE8104007F078BD60
:10706000092007F075FDD4E7389EFF1F489DFF1FDC
:107070005C9DFF1FE19DFF1FE89FFF1F0904028128
:10708000B49FFF1F7F2838B5A8BF7F200F4C4FF457
:10709000167202FB00F284FB02311144D21705463E
:1070A000C2EBA1110A2007F053FD7F3D4FF4967308
:1070B00003FB05F384FB03211944DB17A3EBA111A8
:1070C0000920BDE8384007F043BD00BF0904028134
:1070D000C368B3F9003030B583EAE374A4EBE3741A
:1070E000002BA0B218DB012300E0134603EB830260
:1070F00052009442F9DA0A4D90FBF3F285FB03E467
:1071000003FB1200DB173032D3EBA40380B201F88B
:10711000012BF1D10B7030BD2D230B700131E2E753
:107120006766666638B5094D4624204603F00CF9BB
:1071300035F8021B00B28842204601D003F0EAF87D
:107140000234A4B24E2CF0D138BD00BFA89FFF1F5F
:10715000024B4420198803F0DDB800BFE29FFF1FF7
:1071600038B5094D7824204603F0EEF835F8021BB7
:1071700000B28842204601D003F0CCF80234A4B219
:10718000802CF0D138BD00BF209FFF1F024B76201E
:10719000198803F0BFB800BF9E9DFF1F38B5094D89
:1071A0008224204603F0D0F835F8021B00B2884252
:1071B000204601D003F0AEF80234A4B28A2CF0D1FC
:1071C00038BD00BF289FFF1F024B8020198803F0A5
:1071D000A1B800BFA09DFF1F024B4E20198803F0ED
:1071E00099B800BFB29DFF1F024B9A20198803F087
:1071F00091B800BF149EFF1F024B9820198803F01E
:1072000089B800BFA69DFF1F024B8C20198803F090
:1072100081B800BF3E9FFF1F024B9C20198803F0DE
:1072200079B800BFF89FFF1F024BA020198803F018
:1072300071B800BFB09FFF1F024B9620198803F062
:1072400069B800BF8C9FFF1F024B8A20198803F08A
:1072500061B800BF529FFF1F024B1020198803F036
:1072600059B800BF509FFF1F024B0E20198803F032
:1072700051B800BF649DFF1F024B2C20198803F0FA
:1072800049B800BF869DFF1F024B1E20198803F0DE
:1072900041B800BFA49DFF1F024B2820198803F0AE
:1072A00039B800BFA69FFF1F024B6420198803F066
:1072B00031B800BFA09FFF1F024BB420198803F014
:1072C00029B800BFE89DFF1F024BB620198803F0C4
:1072D00021B800BF24A0FF1F024B5A20198803F0D9
:1072E00019B800BF5E9DFF1F024B1620198803F0DE
:1072F00011B800BF6A9DFF1F024B2E20198803F0B2
:1073000009B800BF1C9EFF1F024B3020198803F0F4
:1073100001B800BF509DFF1F024B9E20198802F04C
:10732000F9BF00BF208AFF1F024BAC20198802F072
:10733000F1BF00BFA29FFF1F024BAE20198802F0D1
:10734000E9BF00BFB09DFF1F024BB020198802F0BB
:10735000E1BF00BF349FFF1F024BB220198802F02B
:10736000D9BF00BFD29DFF1F024B1820198802F021
:10737000D1BF00BF3E9EFF1F024BA220198802F022
:10738000C9BF00BFD49FFF1F024B1A20198802F00B
:10739000C1BF00BFC09DFF1F024B1C20198802F017
:1073A000B9BF00BFB49DFF1F024B6620198802F0D1
:1073B000B1BF00BFE09FFF1F024B7220198802F08F
:1073C000A9BF00BF08A0FF1F024B2020198802F0B0
:1073D000A1BF00BFDE9FFF1F024B3220198802F0C1
:1073E00099BF00BFCE9FFF1F024B6820198802F093
:1073F00091BF00BF009EFF1F024B6C20198802F056
:1074000089BF00BF4C9DFF1F024BBA20198802F0B4
:1074100081BF00BF1E9FFF1F024B6E20198802F024
:1074200079BF00BF3AA0FF1F024B5220198802F01B
:1074300071BF00BF7889FF1F024B5020198802F0EE
:1074400069BF00BF3689FF1F024B5420198802F024
:1074500061BF00BF348AFF1F024B5C20198802F015
:1074600059BF00BF808AFF1F024B5E20198802F0BF
:1074700051BF00BF7089FF1F024B5620198802F0D0
:1074800049BF00BF0E9EFF1F244B1B880B2B43D808
:10749000DFE803F00B10151A1F24292E33383D06A0
:1074A000084604221E490CF0C9BA084604221D49A8
:1074B0000CF0C4BA084604221B490CF0BFBA0846B7
:1074C00004221A490CF0BABA0846042218490CF0F2
:1074D000B5BA0846042217490CF0B0BA084604228F
:1074E00015490CF0ABBA0846042214490CF0A6BAB0
:1074F0000846042212490CF0A1BA08460422114998
:107500000CF09CBA084604220F490CF097BA0846C2
:1075100004220E490CF092BA704700BF8C9FFF1FE7
:10752000CC570100E858010008530100A85401009D
:107530000C53010034590100105301001453010091
:107540006456010018530100D85701001C53010074
:10755000064B074A10B41C88064B0846002C14BF83
:1075600011461946042210BC0CF068BAD89DFF1FC2
:107570002053010024530100064B074A10B41C8815
:10758000064B0846002C14BF11461946042210BCB5
:107590000CF054BA209EFF1F205301002453010019
:1075A000064B074A10B41C88064B0846002C14BF33
:1075B00011461946042210BC0CF040BA469FFF1F2A
:1075C0002053010024530100064B074A10B41C88C5
:1075D000064B0846002C14BF11461946042210BC65
:1075E0000CF02CBA8E9FFF1F205301002453010082
:1075F000064B074A10B41C88064B0846002C14BFE3
:1076000011461946042210BC0CF018BA2A9EFF1F1E
:1076100020530100245301001B4B1B880A2B0AD85E
:10762000DFE803F00A0E12161A1E22262A2E060082
:10763000164B186808607047154B1868086070474B
:10764000144B186808607047134B1868086070473F
:10765000124B186808607047114B18680860704733
:10766000104B1868086070470F4B18680860704727
:107670000E4B1868086070470D4B1868086070471B
:107680000C4B186808607047529FFF1F4C53010055
:1076900024530100285301002C53010030530100F2
:1076A00034530100385301003C53010040530100A2
:1076B0004453010048530100424B1B88182B0ED83D
:1076C000DFE803F07B77726E6964605B57524E4966
:1076D00045413C38332E2A25211C18130E007047D3
:1076E0000846042238490CF0A9B908460422374953
:1076F0000CF0A4B9364B186808607047084604229D
:1077000034490CF09BB9344B186808607047084640
:10771000042232490CF092B9314B18680860704766
:10772000084604222F490CF089B9084604222E4944
:107730000CF084B92D4B1868086070470846042285
:107740002B490CF07BB92B4B1868086070472A4B0B
:107750001868086070470846042228490CF06EB982
:10776000274B1868086070470846042225490CF02A
:1077700065B9254B186808607047084604222349FC
:107780000CF05CB9224B1868086070470846042268
:1077900020490CF053B9084604221F490CF04EB999
:1077A0001E4B186808607047084604221C490CF0FC
:1077B00045B91C4B186808607047084604221A49EE
:1077C0000CF03CB9649DFF1FB0530100AC530100A5
:1077D000A8530100A4530100A05301009C530100D1
:1077E0009853010094530100905301008C53010001
:1077F0008853010084530100805301007C53010031
:107800007853010074530100705301006C53010060
:107810006853010064530100605301005C53010090
:10782000585301005453010050530100F0B52B4E42
:107830002B4FDFF8C4E005460FCE87B06C460FC46F
:1078400096E803003B68274A274F44F8040B40F6AC
:10785000CC308342C8BF3A46BEF800602180012E7A
:1078600011889278ADF80D108DF80F202AD032D300
:1078700040F6CA02022E18BF00229A4226DAA3F668
:1078800098031A491A4AC3EB031381FB03011944F5
:10789000DB17C3EB6123243382FB0321DA17C2EB2E
:1078A000A10202EB8201A3EB4103303330328DF8A9
:1078B00013308DF811206946284616220CF0BEF8C8
:1078C00007B0F0BD40F698029A42D8DB094B186821
:1078D000CDF81100EFE740F6FC02CEE7C4530100FB
:1078E000949FFF1FB8530100B45301003B773B98AE
:1078F00067666666BC530100309FFF1FF8B5174CE2
:10790000174E2278174D33782F888E46003218BFD5
:10791000012201467046FFF753FA00239842337064
:10792000237015DB14BF012000202B889F420ED04E
:1079300040F23A72A3F5AF730B490C4C02FB03F310
:1079400081FB0312DB17A3EB621332332360F8BD14
:107950000749012218460A702270E6E70C8BFF1FC8
:1079600059A0FF1FFA9FFF1FB5814E1B248AFF1FDE
:10797000E4A0FF1F014B187802F03CBCC8A0FF1F19
:10798000014B187802F050BC1891FF1F134BB3F94C
:10799000003030B583EAE374A4EBE374002BA0B2AB
:1079A00018DB012300E0134603EB830252009442EC
:1079B000F9DA0B4D90FBF3F285FB03E403FB1200B5
:1079C000DB173032D3EBA40380B201F8012BF1D1E5
:1079D0000B7030BD2D230B700131E2E71891FF1FB2
:1079E00067666666144BB3F9003070B583EAE375D9
:1079F000A5EBE375002BACB21ADB012300E00346D4
:107A000003EB830040008542F9DA0C4E94FBF3F05F
:107A100086FB03E503FB1044DB173030D3EBA503F3
:107A2000A4B201F8010BF1D105480B70106070BDD4
:107A30002D230B700131E0E75E9DFF1F67666666D0
:107A4000DC530100134BB3F9003030B583EAE37423
:107A5000A4EBE374002BA0B218DB012300E0134673
:107A600003EB830252009442F9DA0B4D90FBF3F2E0
:107A700085FB03E403FB1200DB173032D3EBA403D6
:107A800080B201F8012BF1D10B7030BD2D230B70AA
:107A90000131E2E7208AFF1F67666666134BB3F980
:107AA000003030B583EAE374A4EBE374002BA0B29A
:107AB00018DB012300E0134603EB830252009442DB
:107AC000F9DA0B4D90FBF3F285FB03E403FB1200A4
:107AD000DB173032D3EBA40380B201F8012BF1D1D4
:107AE0000B7030BD2D230B700131E2E7B09DFF1FFD
:107AF00067666666134BB3F9003030B583EAE3740A
:107B0000A4EBE374002BA0B218DB012300E01346C2
:107B100003EB830252009442F9DA0B4D90FBF3F22F
:107B200085FB03E403FB1200DB173032D3EBA40325
:107B300080B201F8012BF1D10B7030BD2D230B70F9
:107B40000131E2E7D29DFF1F67666666134BB3F90A
:107B5000003030B583EAE374A4EBE374002BA0B2E9
:107B600018DB012300E0134603EB8302520094422A
:107B7000F9DA0B4D90FBF3F285FB03E403FB1200F3
:107B8000DB173032D3EBA40380B201F8012BF1D123
:107B90000B7030BD2D230B700131E2E7D49FFF1F26
:107BA00067666666144B1B8801331BB230B583EAE7
:107BB000E374A4EBE374002BA0B218DB012300E014
:107BC000134603EB830252009442F9DA0B4D90FB0B
:107BD000F3F285FB03E403FB1200DB173032D3EB37
:107BE000A40380B201F8012BF1D10B7030BD2D231D
:107BF0000B700131E2E700BF1E9FFF1F67666666DC
:107C0000134BB3F9003030B583EAE374A4EBE374AB
:107C1000002BA0B218DB012300E0134603EB830224
:107C200052009442F9DA0B4D90FBF3F285FB03E42A
:107C300003FB1200DB173032D3EBA40380B201F850
:107C4000012BF1D10B7030BD2D230B700131E2E718
:107C50007889FF1F67666666134BB3F9003030B54D
:107C600083EAE374A4EBE374002BA0B218DB0123D6
:107C700000E0134603EB830252009442F9DA0B4D05
:107C800090FBF3F285FB03E403FB1200DB173032B9
:107C9000D3EBA40380B201F8012BF1D10B7030BDFE
:107CA0002D230B700131E2E73689FF1F6766666698
:107CB000134BB3F9003030B583EAE374A4EBE374FB
:107CC000002BA0B218DB012300E0134603EB830274
:107CD00052009442F9DA0B4D90FBF3F285FB03E47A
:107CE00003FB1200DB173032D3EBA40380B201F8A0
:107CF000012BF1D10B7030BD2D230B700131E2E768
:107D0000348AFF1F67666666134BB3F9003030B5DF
:107D100083EAE374A4EBE374002BA0B218DB012325
:107D200000E0134603EB830252009442F9DA0B4D54
:107D300090FBF3F285FB03E403FB1200DB17303208
:107D4000D3EBA40380B201F8012BF1D10B7030BD4D
:107D50002D230B700131E2E7808AFF1F676666669C
:107D6000134BB3F9003030B583EAE374A4EBE3744A
:107D7000002BA0B218DB012300E0134603EB8302C3
:107D800052009442F9DA0B4D90FBF3F285FB03E4C9
:107D900003FB1200DB173032D3EBA40380B201F8EF
:107DA000012BF1D10B7030BD2D230B700131E2E7B7
:107DB0007089FF1F6766666608B5B82002F0C4FACE
:107DC000044B1988884204D0B820BDE8084002F06E
:107DD000A1BA08BD669DFF1F08B5702002F0B4FA75
:107DE000044B1988884204D07020BDE8084002F096
:107DF00091BA08BD309FFF1F08B5742002F0A4FAA5
:107E0000044B1988884204D07420BDE8084002F071
:107E100081BA08BDC49FFF1F054B1B88084604227A
:107E200013B904490BF00ABE03490BF007BE00BFAB
:107E3000B29DFF1FE4530100E05301000E4B1B886D
:107E4000032B17D8DFE803F0110C070208460422C1
:107E50000A490BF0F3BD0846042209490BF0EEBDB8
:107E60000846042207490BF0E9BD084604220649EA
:107E70000BF0E4BD704700BF3E9FFF1FF4530100AD
:107E8000F0530100EC530100E853010010B40A4B19
:107E90000A4C0A4693E8030083B0238802AC04E945
:107EA000030004EB8303104653F8081C052203B0BB
:107EB00010BC0BF0C3BD00BFD44A0100A09FFF1F40
:107EC00030B40A4B0A4D0C4693E8070084B02B8867
:107ED00004AD05E9070005EB8303204653F80C1CAD
:107EE000042204B030BC0BF0A9BD00BFDC4A010085
:107EF000309FFF1FF0B40C4D0C4F0E460FCD8CB0D1
:107F000001AC0FC40FCD0FC495E807003B8884E88F
:107F100007000CAA02EB8303304653F82C1C042202
:107F20000CB0F0BC0BF08ABDE84A0100849FFF1F33
:107F300030B50A4B0A4D0C460FCB85B00DF1100E33
:107F40000EE90F002B880EEB8303204653F8101C1C
:107F5000042205B0BDE830400BF070BD244B010099
:107F6000A29FFF1F30B50A4B0A4D0C460FCB85B0C0
:107F70000DF1100E0EE90F002B880EEB8303204647
:107F800053F8101C042205B0BDE830400BF056BD7C
:107F9000244B0100349FFF1FF0B40B4D0B4F0E46D6
:107FA0000FCD86B06C460FC495E803003B8884E88B
:107FB000030006AA02EB8303304653F8181C042280
:107FC00006B0F0BC0BF03ABD344B01003E9EFF1FE3
:107FD000F0B40A4D0A4F0E460FCD86B001AC0FC467
:107FE0002A683B88226006AA02EB8303304653F8D6
:107FF000141C0C2206B0F0BC0BF020BD4C4B010051
:10800000B49DFF1FF0B40B4D0B4F0E460FCD88B043
:108010006C460FC495E80F0084E80F003B8808AA5F
:1080200002EB8303304653F8201C042208B0F0BC56
:108030000BF004BD604B0100C49FFF1F164B1B8853
:108040000BB31BB283EAE370A0EBE370002B30B5F7
:1080500084B21DDB012300E0134603EB83025200D0
:108060009042F9DA0D4894FBF3F280FB03E503FB41
:108070001244DB173032D3EBA503A4B201F8012B75
:10808000F1D10B7030BD0846042205490BF0D6BC77
:108090002D230B700131DDE7009EFF1F67666666CA
:1080A000F8530100F0B40A4D0A4F0E460FCD86B0CA
:1080B00001AC0FC42A683B88226006AA02EB830346
:1080C000304653F8141C042206B0F0BC0BF0B6BCCA
:1080D000804B01004C9DFF1F054B1B881BB9054BB6
:1080E0001868086070470846042203490BF0A6BCD4
:1080F000149EFF1F2453010020530100164B1B88C0
:108100000BB31BB230B583EAE374A4EBE374002B2A
:10811000A0B21CDB012300E0134603EB83025200F4
:108120009442F9DA0D4D90FBF3F285FB03E403FB77
:108130001200DB173032D3EBA40380B201F8012B1D
:10814000F1D10B7030BD064B1868086070472D23C5
:108150000B700131DEE700BFA49DFF1F67666666F6
:1081600024530100164B1B880BB31BB230B583EAB6
:10817000E374A4EBE374002BA0B21CDB012300E04A
:10818000134603EB830252009442F9DA0D4D90FB43
:10819000F3F285FB03E403FB1200DB173032D3EB71
:1081A000A40380B201F8012BF1D10B7030BD064B56
:1081B0001868086070472D230B700131DEE700BF9F
:1081C000669DFF1F6766666624530100164B1B8879
:1081D0000BB31BB230B583EAE374A4EBE374002B5A
:1081E000A0B21CDB012300E0134603EB8302520024
:1081F0009442F9DA0D4D90FBF3F285FB03E403FBA7
:108200001200DB173032D3EBA40380B201F8012B4C
:10821000F1D10B7030BD064B1868086070472D23F4
:108220000B700131DEE700BF929FFF1F6766666635
:1082300024530100164B1B880BB31BB230B583EAE5
:10824000E374A4EBE374002BA0B21CDB012300E079
:10825000134603EB830252009442F9DA0D4D90FB72
:10826000F3F285FB03E403FB1200DB173032D3EBA0
:10827000A40380B201F8012BF1D10B7030BD064B85
:108280001868086070472D230B700131DEE700BFCE
:108290006A9DFF1F67666666FC530100174B1B88CB
:1082A0001BB31BB270B583EAE375A5EBE375002B36
:1082B000ACB21EDB012300E0034603EB8300400069
:1082C0008542F9DA0E4E94FBF3F086FB03E503FBDF
:1082D0001044DB173030D3EBA503A4B201F8010B37
:1082E000F1D108480B70106070BD074B186808602A
:1082F00070472D230B700131DCE700BF1C9EFF1F70
:10830000676666660054010024530100164B1B8803
:108310000BB31BB230B583EAE374A4EBE374002B18
:10832000A0B21CDB012300E0134603EB83025200E2
:108330009442F9DA0D4D90FBF3F285FB03E403FB65
:108340001200DB173032D3EBA40380B201F8012B0B
:10835000F1D10B7030BD064B1868086070472D23B3
:108360000B700131DEE700BF509DFF1F6766666638
:1083700024530100164B1B880BB31BB230B583EAA4
:10838000E374A4EBE374002BA0B21CDB012300E038
:10839000134603EB830252009442F9DA0D4D90FB31
:1083A000F3F285FB03E403FB1200DB173032D3EB5F
:1083B000A40380B201F8012BF1D10B7030BD064B44
:1083C0001868086070472D230B700131DEE700BF8D
:1083D000E09FFF1F6766666624530100164B1B88EB
:1083E0000BB31BB230B583EAE374A4EBE374002B48
:1083F000A0B21CDB012300E0134603EB8302520012
:108400009442F9DA0D4D90FBF3F285FB03E403FB94
:108410001200DB173032D3EBA40380B201F8012B3A
:10842000F1D10B7030BD064B1868086070472D23E2
:108430000B700131DEE700BF08A0FF1F67666666AC
:1084400024530100174B1B881BB31BB270B583EA82
:10845000E375A5EBE375002BACB21EDB012300E056
:10846000034603EB830040008542F9DA0E4E94FB8D
:10847000F3F086FB03E503FB1044DB173030D3EB4E
:10848000A503A4B201F8010BF1D108480B701060EC
:1084900070BD074B1868086070472D230B700131C1
:1084A000DCE700BFDE9FFF1F6766666600540100C1
:1084B00024530100054B1B881BB1054B186808604D
:1084C0007047044B18680860704700BF0E9EFF1F7E
:1084D000145401001054010070B5F9F7B9FE164BA1
:1084E0001B7813B1154C237833B9154B102019881C
:1084F00001F010FF012070BD124D134E2B78328811
:10850000B3FA83F382F008025B09114642202B7014
:10851000328001F0FFFE23780BB12B782BB90021BC
:10852000212006F0A5FC002070BD0121212006F0CD
:108530009FFC002070BD00BF6C9DFF1F369FFF1F7A
:10854000509FFF1F4E9FFF1F02A0FF1F184B1A884E
:1085500052B3184A128830B50A80B3F90030002BA4
:1085600083EAE374A4EBE374BCBF2D238B70A0B249
:10857000ACBF02310331012300E0134603EB830259
:1085800052009442F9DA0C4D90FBF3F285FB03E4C0
:1085900003FB1200DB173032D3EBA40380B201F8E7
:1085A000012BF1D10B7030BD044B18680860704787
:1085B000C09DFF1F185401006766666624530100C2
:1085C00070B53C4D2B780646002B35D11C46737890
:1085D0000BB9204670BDF9F73BFE374A374B384898
:1085E000127831781B78007802EB43034A1E03EBC4
:1085F00080030E2AEDD801A050F822F06586000015
:1086000087860000D385000065860000D3850000C2
:10861000D3850000D385000053860000D385000079
:10862000D3850000D3850000D3850000D3850000EA
:10863000D38500004F860000AE21224804F0B4FC30
:10864000204804F0FDFE00232B700124BFE707F053
:108650007DFCAF211B4804F0A7FC1B4A01231370CB
:108660002B70B6E783B91948038804294FF6FF71C8
:1086700003F1FF320CBF01230B46134403F07F03C9
:10868000013303800FE073B1013B114A32F813301C
:108690004BB10E4E0F481049104A3380012300267B
:1086A00006700B701370084A0221012311702B70A1
:1086B000204670BD0C8BFF1FE59FFF1FE69FFF1F2D
:1086C000E79FFF1F64A0FF1FE4A0FF1F0CA0FF1F78
:1086D000109FFF1FF89DFF1F759DFF1FF3A0FF1F39
:1086E00010B5064B064C1A882046012101F000FE09
:1086F00021884220BDE8104001F00CBED89DFF1F2C
:1087000002A0FF1F10B5064B064C1A882046022116
:1087100001F0EEFD21884220BDE8104001F0FABDD5
:10872000209EFF1F02A0FF1F10B5064B064C1A88A3
:108730002046042101F0DCFD21884220BDE81040E4
:1087400001F0E8BD469FFF1F02A0FF1F10B5064BBA
:10875000064C1A882046002101F0CAFD21884220DB
:10876000BDE8104001F0D6BD8E9FFF1F02A0FF1F85
:1087700008B5122001F0E8FD054B1988884206D0A3
:10878000122001F0C7FDBDE8084001F065BC08BD3E
:10879000849FFF1F08B5582001F0D6FD054B1988AE
:1087A000884206D0582001F0B5FDBDE8084001F030
:1087B00053BC08BD929FFF1F08B5142001F0C4FDF3
:1087C000054B1988884206D0142001F0A3FDBDE8AE
:1087D000084001F041BC08BD2A9EFF1FF0B480EAAA
:1087E000E075A5EBE0750028ACB21FDB1DBF2B23A5
:1087F0000B704E1C0E46012300E0134603EB830270
:1088000052009542F9DA0B4F94FBF3F287FB030514
:1088100003FB1244DB173032D3EBA503A4B206F8F6
:10882000012BF1D133700846F0BC70472D230B703B
:108830004E1CE0E767666666084B188828B10D286D
:1088400007D00D3800B2FFF7C9BF054A10680860AD
:108850007047044A10680860704700BF3AA0FF1FC5
:10886000245301001C5401001A4B18880C2815D001
:10887000192817D01A2819D01B281BD01C281DD046
:108880001D281FD01E2821D01F2803D00C3800B26D
:10889000FFF7A4BF104A1068086070470F4A1068BD
:1088A000086070470E4A1068086070470D4A1068EB
:1088B000086070470C4A1068086070470B4A1068DF
:1088C000086070470A4A106808607047094A1068D3
:1088D00008607047CE9FFF1F3C54010020540100E8
:1088E00024540100285401002C540100305401008C
:1088F0003454010038540100034B1888A0EB800069
:10890000400000B2FFF76ABFC8A0FF1F024B1888E3
:10891000643800B2FFF762BF24A0FF1F024B188823
:10892000643800B2FFF75ABFE89DFF1F024B18885A
:10893000033800B2FFF752BFA69FFF1F024B1888F3
:10894000183800B2FFF74ABFA09DFF1F024B1888DE
:10895000183800B2FFF742BF9E9DFF1F024B1888D8
:10896000183800B2FFF73ABFE29FFF1FC3681888AC
:10897000183800B2FFF732BF054B1B881BB9054BF7
:108980001868086070470846042203490BF056B87F
:10899000B09FFF1F2453010020530100054B1B888B
:1089A0001BB9054B18680860704708460422034944
:1089B0000BF044B8A69DFF1F245301002053010073
:1089C00030B5154C85B001252B463C2202212046AE
:1089D000009504F05FFB204604F032FD00224021A8
:1089E000802320460191009311460C4B029505F01F
:1089F000D5F9204604F030FE09480A490A4A002306
:108A00000360436003720B604B600B721360536032
:108A1000137205B030BD00BF64A0FF1F8C4E010073
:108A200048A0FF1FE8A0FF1FD0A0FF1F10B500EB5C
:108A3000C00000F10F02D2B293B284B09C1E981C09
:108A40003D2303918DE819003921024805F00AF908
:108A500004B010BD64A0FF1F014B01221A707047C3
:108A600059A0FF1FF0B5784B784C794F794E7A4D6D
:108A700085B004228DE80C0002932046774B4022FB
:108A8000802104F00FF92046754A7649764C09F0AA
:108A900055F9764B76489F61764FDF61764FB76127
:108AA000764FF761764FAF61764FEF61764FA761F2
:108AB000764FE761764F87617649774FC761774F89
:108AC0008F61774A774FCF61774F9761774B784FB8
:108AD000D761784F9F61784E784FDF61784FB761EB
:108AE000784D794FF761794F794CAF61794FEF61EC
:108AF000794F7A48A7617A4FE7617A4F7A4987615F
:108B00007A4FC7617A4F7B4A8F617B4FCF617B4F32
:108B10007B4B97617B4FD7617B4F7C4E9F617C4F36
:108B2000DF617C4F7C4DB7617C4FF7617C4FAF615B
:108B30007C4C7D4FEF617D4FA7617D487D4FE761A4
:108B40007D4F87617D497E4FC7617E4F8F617E4A31
:108B50007E4FCF617E4F97617E4B7F4FD7617F4FB6
:108B60009F617F4E7F4FDF617F4FB7617F4D804FA9
:108B7000F761804FAF61804C804FEF61804FA761FC
:108B80008048814FE761814F87618149814FC7618B
:108B9000814F824A8F61824FCF61824F824B9761B2
:108BA000824FD761824F834E9F61834FDF61834F36
:108BB000834DB761834FF761834F844CAF61844F1E
:108BC000EF61844F8448A761844FE761844F8549F2
:108BD0008761854FC761854F8F61854A854FCF611A
:108BE000854F9761854B864FD761864F9F61864E33
:108BF000864FDF61864F874DB761874FF761874F9B
:108C0000874CAF61874F88488849EF61884F894D0D
:108C1000A761E561884F894D894CDFF848E2894AB0
:108C2000894B8761C5618C61884E894F894D8A4C1B
:108C3000C1F81CE089488A499761D5619C61D86177
:108C4000B16005B0F0BD00BF40420F0064A0FF1F3F
:108C50002D890000308FFF1FE08CFF1F0092FF1F47
:108C60001C89FF1FFDCC0000F88FFF1FD48FFF1F52
:108C7000248EFF1F9972000051750000E1860000EC
:108C80007975000005870000A175000029870000A4
:108C90008D7E00004C8DFF1FA9720000C975000079
:108CA000488EFF1F4D8700001D8900008891FF1F1F
:108CB000B97200000D8900006491FF1FC9720000A5
:108CC00065810000008EFF1FB97D0000F98800005B
:108CD000DC8DFF1F757900008D790000708DFF1FFE
:108CE00081790000C17E0000608CFF1FD97D0000EB
:108CF000F57E00006490FF1F71870000CD810000A9
:108D0000288DFF1F95870000E5790000208CFF1F4C
:108D1000D9720000F1750000F490FF1FB9870000C0
:108D200035820000048DFF1FE97200009D82000063
:108D3000908EFF1FF97200000D830000A88CFF1FAA
:108D400009730000457A0000A08BFF1F1973000013
:108D5000317F0000AC90FF1F297300009D7A000056
:108D6000788FFF1F39730000657F00007C8BFF1F29
:108D700049730000F57A00006C8EFF1F59730000E4
:108D8000997F0000C48AFF1F697300004D7B0000BB
:108D9000948DFF1F797300004D8500009C8FFF1F8D
:108DA00089730000D17F0000DC91FF1F99730000E0
:108DB000758300000C8FFF1FA9730000DD83000086
:108DC000588BFF1FB9730000058000008890FF1FBB
:108DD000F97D000045840000548FFF1FC973000017
:108DE00069880000348BFF1FD97300003D800000AC
:108DF000108BFF1FE9730000A5800000D88BFF1FB8
:108E0000F9730000A57B0000A08AFF1F0974000011
:108E100039880000B88DFF1F19740000017C000024
:108E2000848CFF1F29740000E88AFF1FFC8BFF1F42
:108E3000597C000039740000B17C000049740000C6
:108E4000097D00001C90FF1FB891FF1FAC91FF1F10
:108E5000617D000069740000B58400007974000031
:108E60002194000059740000F0B5461C83B00D46F3
:108E70000127032336B22AB2044631468DE8880022
:108E80002348ADB204F084FE0C23AA1C12B2009356
:108E90000197052321B21E4804F07AFE1D4A1E4B9D
:108EA00012881B68BA422AD023D3022A10D11B4C45
:108EB000A3F6CA0384FB03241C44DB17C3EB24146E
:108EC0000A2CA8BF0A2424EAE474A2B223B202E066
:108ED00000231A461C460D35AA1A01200093019062
:108EE00012B2314603230A4804F0D0FD204603B0F5
:108EF000F0BD0B4CA3F6FC0384FB0324DDE7094C17
:108F0000A3F6980384FB0324DB17C3EBA404D7E781
:108F100064A0FF1F309FFF1F949FFF1F09CB3D8D53
:108F20001F85EB51398EE3382DE9F0438FB283B0C2
:108F3000DFF84C80BD1D461D2DB204B236B24FF095
:108F400001090AB22346314640460095CDF8049007
:108F500004F0CEFD2A463346214640468DE82002E5
:108F600004F0C6FD07F10C020095334612B221460B
:108F7000CDF80490404604F0BBFD03B0BDE8F0839B
:108F800064A0FF1F2DE9F04F804685B0002959D11C
:108F90000121314805F036F9304998F8062098F853
:108FA000083011F80290994525DADFF8ACB04FEAA5
:108FB00089064D460C244FF0000AD8F80C309B5916
:108FC0005F68ABF810403846ABF80EA00AF078FCAA
:108FD00039460246204808F043FB1F4808F056FB7C
:108FE00098F8083001350934AB42A4B206F1040602
:108FF00001DD422CE1D1B9F1000F13D109F10609CD
:1090000099450CDA3C2301213B2203910293009302
:10901000019239233F223A210F4804F023FE05B084
:10902000BDE8F08F0F2301213B22039102930093AF
:10903000019239230C223A21074804F013FE98F8D4
:109040000830DBE700213423009301913F230C22F9
:10905000014804F01BFD9BE764A0FF1FE8A0FF1F71
:1090600038B50F4C012320461946A382638255254B
:1090700005F0C8F83423204602220A492382E581FC
:1090800008F0EEFA20460522074908F0E9FA2046E2
:1090900008F0FCFA2046BDE8384004F0DDBA00BF15
:1090A00064A0FF1F885401008C540100F8B50F46DE
:1090B00006460AF005FC00EB40008400AFB33846DA
:1090C0000AF0FEFB00EB4000400023185B10194D36
:1090D00003F16002121A4FF0280E01212846C3F155
:1090E0006004EA81A5F810E005F08CF838460AF033
:1090F000E7FB39460246284608F0B2FA284608F04F
:10910000C5FA02210B4805F07DF8212330462B8259
:10911000EC810AF0D5FB31460246064808F0A0FA79
:109120000448BDE8F84008F0B1BA6410C4F1600426
:10913000004DE6E764A0FF1F10B50D4B1B5C51F816
:109140002340237884B013B1012004B010BD04AAD9
:1091500001A942F8103D2046A3699847A38A9B07BE
:10916000F2D401A80099FFF7A1FF012004B010BDBF
:1091700048A0FF1F2DE9F04F304DDFF8D0B0DFF8E9
:10918000C8A00FCD91B003AC0FC40FCD0FC40FCD4D
:109190000FC42B6823600025A8462F462E4600E00A
:1091A0009846BAF8003026495BF82320DFF8A090F3
:1091B00011232846F7F716FB00EBC00300EB8300F2
:1091C000204B83FB00340444C017C0EB6434C4F16B
:1091D0003C00C6F13C0207F14101012600B208F152
:1091E000410300901BB2019612B209B2484604F046
:1091F0007FFC08EB060305F211153C2B2646ADB2A9
:109200004746CDD16B22342300214846A9F80E20D1
:10921000A9F8103004F0F6FF0B4B1B8810AA02EBE4
:10922000830353F8344C20460AF04AFB2146024699
:10923000484611B0BDE8F04F08F012BA944B010057
:109240000045010009000280869DFF1F6443010064
:1092500064A0FF1F234B70B5B3F9003083EAE374B9
:10926000A4EBE374002B82B0A1B234DB68466D46F8
:10927000012300E0134603EB830252009442F9DA23
:10928000194E91FBF3F286FB03E403FB1211DB178B
:109290003032D3EBA40389B205F8012BF1D1194682
:1092A0002B70FFF703FF114B1B7813B1104B1B788A
:1092B0000BB902B070BD0F4C0121204604F0A2FF93
:1092C00064253323204604220B49E581238208F0DC
:1092D000C7F902B070BD2D238DF800300DF10105E6
:1092E0006846C5E7509FFF1F67666666369FFF1F8B
:1092F0004E9FFF1F64A0FF1F9454010070B5404EA5
:10930000404D82B0304604F09BF82B78D3B93C4CEA
:109310000621204604F076FF2B78012B38D9022B4A
:109320004FF003024FF00A030CBF37493749E3817E
:109330002046238208F094F9204602B0BDE8704030
:1093400008F0A4B9324B1A7801210523002A33D141
:10935000019100931146304604F01AFC2D4B1A7807
:10936000002A34D0052301220192009300220A2111
:10937000234804F08BFB284B1A78002A33D10121B3
:1093800005230191009314211D4804F001FCBEE760
:10939000224B1988092930D963298CBF0A221F2240
:1093A0000A231748F281338208F0C0F9144802B04A
:1093B000BDE8704008F06AB900220191009311469F
:1093C000304604F063FB134B1A78002ACAD10523F8
:1093D0000121019100930A21094804F0D9FB0E4BA9
:1093E0001A78002ACBD00122052301920093002293
:1093F0001421034804F04AFB89E73022D0E700BF7C
:1094000064A0FF1FF3A0FF1F9C540100A0540100A3
:10941000E59FFF1FE69FFF1FE79FFF1F0CA0FF1F99
:109420002DE9F047714E307848B9714B1B6899426D
:109430005FD3704A012313703370BDE8F0876E4D1F
:109440006B4F0C46284603F0FBFF04F6AC53312467
:109450000022EC810124114628462A82AC826C82CB
:109460003B60327004F0CEFE05226449644E28460B
:1094700008F0F6F8102728464FF00C0808F006F917
:109480000B226049EF812846A5F8108008F0E8F823
:109490005D490522284608F0E3F8284608F0F6F86A
:1094A0005A4BEF811A68A2F69803C3EB031386FBAD
:1094B00003161E44DB17C3EB662640F6CC3320218F
:1094C0009A42298206F124064FF022014FF004004F
:1094D00011DCFFF7C9FC4E4BB3F800908246B9F19E
:1094E000000F30D0B9F1010F4DD0B9F1020F47D0C4
:1094F0002046BDE8F087FFF717FD464909222846B8
:1095000008F0AEF84449EF8181FB0637F317C3EB4F
:10951000A7072A23394628462B8208F007F9224656
:109520003E49284608F09CF807EB8701A6EB41016D
:10953000284608F0FBF822462846394908F090F8FA
:109540002046BDE8F08737493A46284608F088F8B3
:10955000284608F09BF82A232B825146EF812846A3
:109560002D4F08F0E3F807222F49284608F078F835
:10957000F31787FB0627C3EBA70739462846CCE736
:1095800042462A49E1E742462949234C284608F049
:1095900067F8284608F07AF82A232B825146284695
:1095A000EF8108F0C3F807221F49284608F058F851
:1095B000F31784FB0624C3EBA4042146284608F0D5
:1095C000B5F84A461549284608F04AF804EB8401E4
:1095D000A6EB4101284608F0A9F84A46284610495A
:1095E00008F03EF84846BDE8F08700BF0C8BFF1F2F
:1095F00060A0FF1FE4A0FF1F64A0FF1FA454010090
:109600003B773B98AC5401008C540100949FFF1FA2
:10961000309FFF1FB854010067666666F85C010062
:10962000685C0100C4540100D8540100F0540100EA
:10963000E05401002DE9F041744C2278002A0546DF
:109640000F4614BF4FF001084FF000084ED1704E86
:109650003368CB1AB3F5FA6F04D86B78A3B94046D8
:10966000BDE8F0816B4B6C486C49DFF8CCE11A70B7
:10967000012303700988237026208EF8002000F053
:1096800049FE6B78002BEAD03760F8F7E1FD644AB9
:10969000644B6549127828781B78097802EB4303FC
:1096A000421E03EB81030E2AD9D801A151F822F002
:1096B0009D970000699700005F9600009D9700004D
:1096C0005F9600005F9600005F96000051970000D3
:1096D0005F960000079700005F9600005F9600000D
:1096E0005F9600005F96000003970000AF214F488F
:1096F000474E03F059FCFFF701FE0023376023704B
:10970000ABE706F023FC494C204603F099FE2046C7
:10971000022104F077FD23250F23238205224449EB
:10972000E581204607F09CFF204607F0AFFF1E238F
:109730000522404923822046E58107F091FF20461B
:1097400007F0A4FF204603F087FF00F0D5FC86E772
:10975000394D2B78012B50D9304B2620198800F039
:10976000D9FD00232B707AE7002B3FF478AF013B43
:10977000324A32F81330002B3FF471AF274C304897
:1097800025492D4A23804FF001080023037081F8FA
:10979000008082F80080FFF7B1FD60E793B1013BE4
:1097A000264A32F8131019B31C4B254D1A4C224A85
:1097B00019800026012326202E702370137000F0DC
:1097C000A9FD15E0154C1E4922880B7004284FF6A0
:1097D000FF7002F1FF310CBF012202460A440E4E17
:1097E000154D02F07F0201320121228031702B7071
:1097F000FFF784FD4FF0010831E70649064A0123CF
:109800000020087013702370A6E700BF0C8BFF1FA9
:10981000E0A0FF1FE4A0FF1F759DFF1F0CA0FF1F0E
:10982000E59FFF1FE69FFF1FE79FFF1F64A0FF1F2D
:109830000055010008550100F3A0FF1F109FFF1FF6
:10984000F89DFF1F2DE9F04FAE4E4FF00109A6F82D
:109850001490A6F81290838813EA09048BB0054689
:109860000F46934640F0AB80DFF8C48298F8003092
:10987000002B7BD1AA79A44CA35CA3B9DFF8B4A2D6
:1098800079781AF8029039B33B78013B072B00F244
:10989000B280DFE813F0EF005101B0006B01B000BF
:1098A000B000B000E7007E78002E00F0C580013BDC
:1098B000E868397850F82360F0684B1E0788072B5A
:1098C00000F2A380DFE813F070015901A1006A01E2
:1098D000A100A100A1009B008C4E3368C3EB0B03D9
:1098E000B3F5967F72D98A4B187801281ABF0120E8
:1098F00018701970874B18BF0146985CC0EB0900BF
:10990000C0B2FFF793F80124C6F800B0AB889B07FC
:109910006DD57B78002B6AD0F8F79AFC7E4B7F4A96
:109920007F481B78127839780078022515FB0233BE
:109930000A2903EB800300F049810C2957D1002B41
:1099400055D003F11900774E774A013B00214000C2
:1099500080B226F813100123157088F8003000F04B
:10996000D9FC724B032220461A702CE0304603F0DB
:1099700067FD3046494604F045FCF4813482AB88EB
:10998000580725D42C68204609F09AFF2146024644
:10999000304607F065FE304607F078FE09220123C5
:1099A0008DE80C0000217F23564804F0A1F8002127
:1099B0002846FFF7E7FA002388F800305AE7836863
:1099C0001146384698470BB0BDE8F08F0846FAE7D5
:1099D0002B6804A8984704A809F072FF04A902465E
:1099E000304607F03DFE304607F050FED6E72046F1
:1099F0000BB0BDE8F08F00240AF8029086E7002340
:109A0000A3543046F3699847F06807800024252264
:109A10003C238DE81400412118223A4804F036F81E
:109A2000E968A879FFF788FB394A384B1470C3F806
:109A300000B00BB0BDE8F08F34490B68C3EB0B03EB
:109A4000B3F5967F40F2E080314FC1F800B03C782A
:109A5000012C00F0AF800123E9683B701046FFF74E
:109A60006BFBB0E7304BE9791970012388F80030BF
:109A70000024C1E72B7A013B4B45BCDD09F1010411
:109A8000E4B2A145B7D0234E16F802B0CBEB0900E3
:109A9000C0B20021FEF7CAFF2B7A052BD9461BD98D
:109AA000CBEB0402042A40F3A980A4F1040BBBF120
:109AB000000FC0F2AD80063B5B45A8BF5B465FFA76
:109AC00083F9AA791348B15C994205D000F8029055
:109AD00001212846FFF756FAC9EB0400C0B2012164
:109AE0000B4EFEF7A3FF00213423019100930B22BC
:109AF0003170044840233F21A14603F0C7FF0124F1
:109B0000AA7979E764A0FF1FD0A0FF1FCCA0FF1F98
:109B1000F1A0FF1FE8A0FF1FE59FFF1FE69FFF1FAB
:109B2000E79FFF1F109FFF1FE4A0FF1FF3A0FF1F71
:109B30000C8BFF1F48A0FF1F0FFA89F3E9685D48EF
:109B400051F823B0036804935B499BF800300498F4
:109B50000860002B6CD0012B7FF44DAF57499BF868
:109B6000080088F800300870002445E7B9F1000FBC
:109B70004CD009F1FF34E4B283E7B38A03F0040365
:109B80009BB2002B3FF43CAF336A984700283FF468
:109B90003BAFAB79F0680022E25436E7738ABB42F0
:109BA00040D90137BFB230E7338ABB4234D2013FDC
:109BB000BFB22AE725238DE8480041483E703C2388
:109BC0001822412103F062FF2046FCE6002B3FF4FF
:109BD0000EAF3C4A3C4E1188384A03F11900013B54
:109BE000400080B226F81310012388F80030157069
:109BF00000F090FB354B20461D70E4E6002A3FF74D
:109C00005AAF04F1FF3B52E73046DCE64C46F3E640
:109C10004FF000094B4654E7B38AD9077FF5F5AEFC
:109C2000778AF2E6B38ADA077FF5EFAE378AECE699
:109C300027490393885CC0EB090009F1010EC0B20B
:109C4000012104F802E0FEF7F1FE039BDBF808B007
:109C5000019334231A4800930B2240233F2103F041
:109C600015FF012434230B228DE818003F214023E7
:109C7000134803F08DFF2146114804F0C3FA5846FB
:109C800009F01EFEA0EB800000F15F030F22F381BC
:109C90003282584609F014FE59460246084807F039
:109CA000DFFC074807F0F2FCE968A879FFF744FAFF
:109CB000AA79A1E610A1FF1FCCA0FF1FE4A0FF1FFF
:109CC00064A0FF1F0CA0FF1F109FFF1FF3A0FF1F2A
:109CD000E8A0FF1F2DE9F047DFF85C927F4B99F871
:109CE00000601B68DFF854A282B0003601934FF089
:109CF000030018BF0126019F9AF8008005F0BEF806
:109D00000546042005F0BAF80446052005F0B6F82B
:109D1000800040EA4404062005F0B0F82C4364B209
:109D20006F4944EAC0000A7880F00F03DBB29A4220
:109D30006C4A48D0176000226B480B7003788DF88E
:109D400000808DF80120002B35D0684A12684EF64D
:109D50006021BA1A8A4223D8022B65D0012B6BD01E
:109D6000062B54D0032B6FD0042B75D0052B00F09D
:109D70008B80072B00F09080082B00F09580092B3A
:109D800072D00A2B00F098800B2B00F09D800C2BDA
:109D900072D016B1564803F05FFC02B0BDE8F08700
:109DA000544A554C00230121237003701360536003
:109DB000137289F800103A4669465048FFF742FD91
:109DC0003043C6B2E5E71268BA1A1E2A40F2848010
:109DD0009AF80020934222D0444C49488AF8003037
:109DE000012B276082EA030207609846A4D0042B67
:109DF000A2D143480068381AB0F5C87F9CD9414CBD
:109E00002068381A322897D927601A4694E73A46CC
:109E100069463D48FFF716FD3043C6B2B9E7012B4E
:109E20004FF00002E3D1E4E73A4669463748FFF7CE
:109E300009FD3043C6B2ACE73A4669463448FFF7FD
:109E400001FD3043C6B2A4E73A4669463148FFF700
:109E5000F9FC3043C6B29CE73A4669462E48FFF704
:109E6000F1FC3043C6B294E73A4669462B48FFF707
:109E7000E9FC3043C6B28CE73A4669462848FFF70A
:109E8000E1FC3043C6B284E73A4669462548FFF70D
:109E9000D9FC3043C6B27CE73A4669462248FFF710
:109EA000D1FC3043C6B274E73A4669461F48FFF713
:109EB000C9FC3043C6B26CE73A4669461C48FFF716
:109EC000C1FC3043C6B264E73A4669461948FFF719
:109ED000B9FC3043C6B25CE700222DE710A1FF1F9A
:109EE000F4A0FF1F54A0FF1FE4A0FF1FDCA0FF1F72
:109EF00064A0FF1FD0A0FF1FF2A0FF1F5C4E010057
:109F0000F8A0FF1F5CA0FF1F8C520100D84D01007C
:109F10007C4C0100084C0100845B01006C4C01008A
:109F2000144C0100F84C0100E85B0100AC91FF1FEC
:109F3000804D0100F84B01000C8BFF1F58A0FF1F44
:109F400028B11028044BA8BF102018607047024B9E
:109F500001201860704700BFFCA0FF1F08B500205B
:109F600006F0ECFE0028FAD108BD00BF70B50D4622
:109F70001446064605F0B2FD284605F0AFFD204622
:109F800005F0ACFD084B1B7813B1084B1B7803B9E7
:109F900070BD304605F030FA284605F02DFA20460F
:109FA000BDE8704005F028BA369FFF1F4E9FFF1F87
:109FB00038B5164D2B78044641F6FF72A0F50050D7
:109FC000824203F1FF33A8BF02461B0202F5005292
:109FD00003F47063100443F4604343F00E0300F491
:109FE000FE005204184302F0FE42104306F0DCFD6E
:109FF0002868013860F01F00C4F3C61204F07F0126
:10A00000C0B2BDE83840FFF7B1BF00BFFCA0FF1FE2
:10A0100070B5104E3378013B1B0203F470630446A5
:10A0200043F430430806220400F0FE4043F00B03E3
:10A03000034302F4FE0018430D4606F0B5FD3068F8
:10A04000013860F04F002A462146C0B2BDE870409A
:10A05000FFF78CBFFCA0FF1F08B564210720FFF7A6
:10A06000D7FF7F210B20BDE80840FFF7D1BF00BF1D
:10A0700070B5104E3378013B1B0203F47063044645
:10A0800043F410430806220400F0FE4043F00903A5
:10A09000034302F4FE0018430D4606F085FD3068C8
:10A0A000013860F06F002A462146C0B2BDE870401A
:10A0B000FFF75CBFFCA0FF1F38B50E4D2B78013BAE
:10A0C0001B0203F47063044643F41043000443F09E
:10A0D000090300F4FE00184306F066FD2868013805
:10A0E00060F06F002146C0B20022BDE83840FFF7A3
:10A0F0003DBF00BFFCA0FF1F10B500217B20FFF774
:10A1000087FF0024E0B2FFF7D7FF0134022004F0FC
:10A11000EBFE802CF6D110BD38B50C46054605F097
:10A12000DDFC204605F0DAFC074B1B7813B1074B2A
:10A130001B7803B938BD284605F05EF92046BDE816
:10A14000384005F059B900BF369FFF1F4E9FFF1FD3
:10A1500038B50D4D2B78013B1B0203F470630446A8
:10A1600043F45043000443F00D0300F4FE00184391
:10A1700006F01AFD2868013860F02F002146C0B2B1
:10A18000BDE83840FFF7C8BFFCA0FF1F38B50E4D33
:10A190002B78013B01381B02C4B203F47063200426
:10A1A00043F4404343F00C0300F4FE00184306F070
:10A1B000FBFC2868013860F03F002146C0B2BDE8D2
:10A1C0003840FFF7A9BF00BFFCA0FF1F38B5044609
:10A1D0000D46F02005F082FC35B1254414F8010B42
:10A1E00005F07CFCAC42F9D1F720BDE8384005F021
:10A1F00075BC00BF00B50B4B83B002469988186848
:10A200000090032AADF8041002D903B05DF804FBF6
:10A21000684606218DF80520FFF7D8FF03B05DF8EA
:10A2200004FB00BF285C010000B50B4B024683B065
:10A23000186899880090131F4C2BADF8041002D9B0
:10A2400003B05DF804FB684606218DF80520FFF792
:10A25000BDFF03B05DF804FB305C0100030203F4B2
:10A26000FE43C0F3C6101843704700BF0378407820
:10A27000DB0103F47E5300F07F001843704700BFFA
:10A2800082B002AA114642F8040D002012F8013BE8
:10A2900003F07F03914243EA0020F7D102B07047F8
:10A2A00010B547F6122104460D4807F093F805F063
:10A2B00035FC0C4B1B7833B974B1102C0A4BA8BF7A
:10A2C00010241C6010BD47F61221084806F0D2FF8A
:10A2D00005F04EF9002CF0D1034B01241C6010BD99
:10A2E000DC93FF1F369FFF1FFCA0FF1FC893FF1FBB
:10A2F000003210B403884FF0010404FA01F418BFCF
:10A30000012202FA01F123EA04020A43028010BC8E
:10A31000704700BF70B5CEB20C46054604F03EFA59
:10A32000864203D03146284604F052FA01352846C9
:10A3300004F034FA240A844205D021462846BDE8B8
:10A34000704004F045BA70BD38B5054604F026FAF1
:10A350004FF0000460F30704681C04F01FFA60F378
:10A360000F24A0B238BD00BFF8B504460020FFF7A7
:10A37000EBFF002C00F0DD854FF4AF610220FFF70A
:10A38000C9FF4FF47A610420FFF7C4FF4FF49661D0
:10A390000620FFF7BFFF4FF4FA610820FFF7BAFF6E
:10A3A0004FF4FA610A20FFF7B5FF40F6B8310C20F0
:10A3B000FFF7B0FF4FF42F612220FFF7ABFF40F60D
:10A3C000AC512420FFF7A6FF7D212A20FFF7A2FF32
:10A3D0000C210E20FFF79EFF01211020FFF79AFFAE
:10A3E00002211220FFF796FF00211420FFF792FFB1
:10A3F00000211620FFF78EFF02211820FFF78AFFA9
:10A4000001211A20FFF786FF01211C20FFF782FFA0
:10A4100004211E20FFF77EFF14212020FFF77AFF82
:10A4200001212620FFF776FF03212820FFF772FF86
:10A4300004212C20FFF76EFF14212E20FFF76AFF66
:10A4400000213020FFF766FF0C213220FFF762FF6A
:10A4500000213420FFF75EFF00213620FFF75AFF6E
:10A4600000213820FFF756FF00213A20FFF752FF66
:10A4700000213C20FFF74EFF00213E20FFF74AFF5E
:10A4800000214020FFF746FF00214220FFF742FF56
:10A490001F214420FFF73EFF13214620FFF73AFF1C
:10A4A0000E214820FFF736FF11214A20FFF732FF27
:10A4B0000A214C20FFF72EFF00214E20FFF72AFF34
:10A4C00006215020FFF726FF02215220FFF722FF2E
:10A4D0000C215420FFF71EFF00215620FFF71AFF22
:10A4E00000215820FFF716FF01215A20FFF712FF25
:10A4F00008215C20FFF70EFF0F215E20FFF70AFF07
:10A5000000216020FFF706FF04216220FFF702FF11
:10A5100001216420FFF7FEFE00216620FFF7FAFE0E
:10A520000B216820FFF7F6FE7F216A20FFF7F2FE7D
:10A5300000216C20FFF7EEFE00216E20FFF7EAFEFF
:10A5400000217020FFF7E6FE00217220FFF7E2FEF7
:10A5500000217420FFF7DEFE1F217620FFF7DAFED0
:10A5600013217820FFF7D6FE0E217A20FFF7D2FEC6
:10A5700011217C20FFF7CEFE0A217E20FFF7CAFEC4
:10A580001F218020FFF7C6FE13218220FFF7C2FEA5
:10A590000E218420FFF7BEFE11218620FFF7BAFEB0
:10A5A0000A218820FFF7B6FE00218A20FFF7B2FEBD
:10A5B00000218C20FFF7AEFE00219620FFF7AAFEB7
:10A5C00000219820FFF7A6FE00219A20FFF7A2FEA7
:10A5D00005219C20FFF79EFE06219E20FFF79AFE94
:10A5E0000021A020FFF796FE7F21A220FFF792FE18
:10A5F00040F2A461A420FFF78DFE4FF4E161A62094
:10A60000FFF788FE0021A820FFF784FE0021AA2082
:10A61000FFF780FE0221AC20FFF77CFE0121AE2077
:10A62000FFF778FE0121B020FFF774FE0B21B22066
:10A63000FFF770FE6421B420FFF76CFE6421B620A2
:10A64000FFF768FE0321B820FFF764FE0121BA205E
:10A65000FFF760FE2D210020FFF75CFE0220FFF7D0
:10A6600073FEB0F5805F034680F04986D24A04202D
:10A670001380FFF769FEB0F5805F034680F03686F1
:10A68000CE4A06201380FFF75FFEA0F52F739BB222
:10A69000B3F57A6F024606D940F628210620FFF767
:10A6A00039FE40F62822C64B08201A80FFF74CFEE0
:10A6B000A0F52F739BB2B3F57A6F024606D940F628
:10A6C000E4410820FFF726FE40F6E442BD4B0A2095
:10A6D0001A80FFF739FEA0F5FA739BB240F6AC5131
:10A6E0008B42024606D94FF4FA610A20FFF712FEA8
:10A6F0004FF4FA62B44B0C201A80FFF725FEA0F548
:10A70000FA739BB240F6AC518B42024606D940F632
:10A71000B8310C20FFF7FEFD40F6B832AB4B0E20EF
:10A720001A80FFF711FE1828034600F2D885A84AC0
:10A7300010201380FFF708FE431E9BB20F2B02462A
:10A7400004D901211020FFF7E5FD0122A14B1220C1
:10A750001A80FFF7F9FD0A28034600F2B9859E4AE0
:10A7600014201380FFF7F0FD0128034604D90021CF
:10A770001420FFF7CFFD0023984A16201380FFF71F
:10A78000E3FD7F28034600F29C85954A182013803C
:10A79000FFF7DAFD0528034600F28C85914A1A205E
:10A7A0001380FFF7D1FD0C28034600F27C858E4A0A
:10A7B0001C201380FFF7C8FD0428034600F26C85B7
:10A7C0008A4A1E201380FFF7BFFD0928034600F2C6
:10A7D0005C85874A20201380FFF7B6FD4628034694
:10A7E00000F24C85834A22201380FFF7ADFDA0F5CF
:10A7F000FA739BB240F6AC518B42024606D94FF435
:10A800002F612220FFF786FD4FF42F627A4B242020
:10A810001A80FFF799FDA0F5FA739BB240F6AC548D
:10A82000A342024604D921462420FFF773FD2246A5
:10A83000724B26201A80FFF787FD7F28034600F21F
:10A8400016856F4A28201380FFF77EFD06280346F1
:10A8500000F206856B4A2A201380FFF775FDA0F1F0
:10A8600032039BB2B3F5967F024604D97D212A209C
:10A87000FFF750FD7D22644B2C201A80FFF764FD0A
:10A880000C28034600F2E584604A2E201380FFF76F
:10A890005BFD1E28034600F2D5845D4A30201380FC
:10A8A000FFF752FD0928034600F2C584594A3220B9
:10A8B0001380FFF749FD1F28034600F2B584564A6E
:10A8C00034201380FFF740FD7F28034600F2A58463
:10A8D000524C36202380FFF737FD7F28034600F2D5
:10A8E000958438206380FFF72FFD7F28034600F210
:10A8F00086843A20A380FFF727FD7F28034600F2D5
:10A9000077843C20E380FFF71FFD7F28034600F299
:10A9100068843E202381FFF717FD7F28034600F25D
:10A92000598440206381FFF70FFD7F28034600F222
:10A930004A844220A381FFF707FD394D2880442037
:10A94000FFF702FD3028034600F23684354A4620E0
:10A950001380FFF7F9FC3028034600F22684324CBE
:10A9600048202380FFF7F0FC3028034600F21684CD
:10A970004A206380FFF7E8FC3028034600F2E283B8
:10A980004C20A380FFF7E0FC3028034600F2D4837C
:10A990004E20E380FFF7D8FC0128034604D90021AC
:10A9A0004E20FFF7B7FC0023204A50201380FFF70A
:10A9B000CBFC431E3CE000BF389EFF1F5C9DFF1F89
:10A9C000DC9DFF1FCC9FFF1F989FFF1F9C9DFF1FBB
:10A9D000649DFF1F509FFF1F849FFF1F2A9EFF1F24
:10A9E0006A9DFF1F3E9EFF1FC09DFF1FB49DFF1F5E
:10A9F000A49DFF1FDE9FFF1F4C9FFF1F489FFF1F4F
:10AA00000CA0FF1FA69FFF1FFA9FFF1F869DFF1F21
:10AA10001C9EFF1F509DFF1FCE9FFF1F109FFF1FFB
:10AA200002A0FF1FE29FFF1FA89FFF1FB29DFF1FF5
:10AA30009BB20B2B024604D906215020FFF76AFC7B
:10AA40000622CF4B52201A80FFF77EFC04280346D3
:10AA500000F26C83CB4A54201380FFF775FC431E31
:10AA60009BB21D2B024604D90C215420FFF752FC47
:10AA70000C22C54B56201A80FFF766FC01280346BE
:10AA800004D900215620FFF745FC0023BF4A582077
:10AA90001380FFF759FC7F28034600F24183BC4A2C
:10AAA0005A201380FFF750FC431E9BB2092B02462D
:10AAB00004D901215A20FFF72DFC0122B54B5C205F
:10AAC0001A80FFF741FC431E9BB2102B024604D9AB
:10AAD00008215C20FFF71EFC0822AF4B5E201A8085
:10AAE000FFF732FC431E9BB21D2B024604D90F21F7
:10AAF0005E20FFF70FFC0F22A84B60201A80FFF7A3
:10AB000023FC0228034600F20583A54A6420138033
:10AB1000FFF71AFC0128034604D901216420FFF73E
:10AB2000F9FB01239F4A62201380FFF70DFCC31E2F
:10AB30009BB2012B024604D904216220FFF7EAFBF5
:10AB40000422994B66201A80FFF7FEFB7F280346FC
:10AB500000F2DA82954A68201380FFF7F5FB7F2820
:10AB6000034600F2CB82924A6A201380FFF7ECFB87
:10AB70007F28034600F2BC828E4A6C201380FFF7C8
:10AB8000E3FB0428034600F2AD828B4A6E2013805B
:10AB9000FFF7DAFB1928034600F29E82874A7020ED
:10ABA0001380FFF7D1FB0228034600F28F82844A0C
:10ABB00072201380FFF7C8FB0628034600F280824C
:10ABC000804A74201380FFF7BFFB0728034600F27A
:10ABD00071827D4A8A201380FFF7B6FB0A2803465C
:10ABE00000F26282794A8C201380FFF7ADFB0428C3
:10ABF000034600F25382764A98201380FFF7A4FBA5
:10AC00000128034604D900219820FFF783FB002385
:10AC1000704A9A201380FFF797FB0128034604D956
:10AC200000219A20FFF776FB00236B4A96201380C1
:10AC3000FFF78AFB0B28034600F22A82674A9C2012
:10AC40001380FFF781FB831E9BB2032B024604D9BE
:10AC500005219C20FFF75EFB0522614B76201A80C0
:10AC6000FFF772FB3028034600F20C825D4A782021
:10AC70001380FFF769FB3028034600F2FD815A4C30
:10AC80007A202380FFF760FB3028034600F2EE8134
:10AC90007C206380FFF758FB3028034600F2E081F8
:10ACA0007E20A380FFF750FB3028034600F2D281BC
:10ACB0008020E380FFF748FB3028034600F2C48180
:10ACC0004A4A82201380FFF73FFB3028034600F2F8
:10ACD000B581474C84202380FFF736FB302803469C
:10ACE00000F2A68186206380FFF72EFB3028034602
:10ACF00000F298818820A380FFF726FB30280346C6
:10AD000000F28A81A020E380FFF71EFB01280346A2
:10AD100004D90021A020FFF7FDFA0023354A9E2028
:10AD20001380FFF711FBC31E9BB20C2B024604D904
:10AD300006219E20FFF7EEFA06222F4BA2201A8052
:10AD4000FFF702FB431E9BB27E2B024604D97F21F4
:10AD5000A220FFF7DFFA7F22284BA4201A80FFF7FA
:10AD6000F3FAA0F5AF639BB2B3F5167F024647D95D
:10AD700040F2A461A420FFF7CDFA40F2A4623FE0C4
:10AD80003689FF1F7889FF1F348AFF1F0E9EFF1F21
:10AD9000929FFF1F5E9DFF1F808AFF1F7089FF1F0C
:10ADA000449FFF1FA09FFF1FC89DFF1FE09FFF1F25
:10ADB000009EFF1FA89DFF1F4C9DFF1F3AA0FF1F75
:10ADC000309FFF1F08A0FF1FC49FFF1F529FFF1F40
:10ADD0003E9FFF1FA69DFF1F149EFF1F8C9FFF1FFE
:10ADE000F89FFF1F9E9DFF1F209FFF1FA09DFF1F1D
:10ADF000289FFF1FB09FFF1F208AFF1FD49FFF1FA8
:10AE0000D34BA6201A80FFF79FFAA0F5AF639BB241
:10AE1000B3F5167F024606D94FF4E161A620FFF78D
:10AE200079FA4FF4E162CB4BA8201A80FFF78CFA35
:10AE30000628034600F2EA80C74AAA201380FFF7DB
:10AE400083FA0328034600F2DB80C44AAC20138057
:10AE5000FFF77AFA0328034600F2CC80C04AB020FC
:10AE60001380FFF771FA0328034600F2BD80BD4A44
:10AE7000AE201380FFF768FA7F28034600F2AE8009
:10AE8000B94AB2201380FFF75FFA7F28034600F229
:10AE90009F80B64AB4201380FFF756FA431E9BB238
:10AEA000C62B024604D96421B420FFF733FA64228A
:10AEB000AF4BB6201A80FFF747FA431E9BB2C62B52
:10AEC000024604D96421B620FFF724FA6422A94B74
:10AED000B8201A80FFF738FA0828034672D8A64A25
:10AEE000BA201380FFF730FA032865D82B88DFF8E3
:10AEF000A8E2A24FA24AA34DA34EA44CA44903F03A
:10AF0000010CAEF800C0C3F3400EA7F800E0C3F395
:10AF100080071780C3F3C0079E4A2F70C3F3001742
:10AF2000C3F34015C3F38013378025800B80108056
:10AF3000F8BD4FF6FF7398423FF41EAA2D283FF448
:10AF40008DAB17287FF618AA19287FF681AA1B282F
:10AF50007FF69EAA1C283FF4B3AA1E287FF6B8AA43
:10AF60001F283FF4BDAA20283FF4D6AA21283FF489
:10AF7000DFAA22283FF4E4AA23283FF4EDAA2428DC
:10AF80003FF41EAB25283FF423AB26283FF424AB27
:10AF900027283FF429AB28283FF434AB29283FF475
:10AFA00039AB2A283FF446AB2B283FF44BAB2C2877
:10AFB0007FF450ABFFF74ABBBA200121FFF7AAF993
:10AFC000012093E70321B820FFF7A4F9032386E7C4
:10AFD0000B21B220FFF79EF90B235AE70121AE2087
:10AFE000FFF798F901234BE70121B020FFF792F911
:10AFF00001233CE70221AC20FFF78CF902232DE767
:10B000000021AA20FFF786F900231EE70021A820CF
:10B01000FFF780F900230FE70A218820FFF77AF96C
:10B020000A236FE611218620FFF774F9112361E6E8
:10B030000E218420FFF76EF90E2353E613218220A0
:10B04000FFF768F9132344E61F218020FFF762F918
:10B050001F2335E60A217E20FFF75CF90A2327E645
:10B0600011217C20FFF756F9112319E60E217A20D1
:10B07000FFF750F90E230BE613217820FFF74AF96A
:10B080001323FCE51F217620FFF744F91F23EDE58C
:10B0900000219620FFF73EF90023CFE500218C2008
:10B0A000FFF738F90023A6E500218A20FFF732F9DF
:10B0B000002397E500217420FFF72CF9002388E591
:10B0C00000217220FFF726F9002379E50021702086
:10B0D000FFF720F900236AE500216E20FFF71AF937
:10B0E00000235BE500216C20FFF714F900234CE5F9
:10B0F0007F216A20FFF70EF97F233DE50B216820B1
:10B10000FFF708F90B232EE500216620FFF702F96F
:10B1100000231FE500216020FFF7FCF80023F4E482
:10B1200000215820FFF7F6F80023B8E4022152204E
:10B13000FFF7F0F802238DE40A214C20FFF7EAF82C
:10B140000A2325E411214A20FFF7E4F8112317E42C
:10B150003C9EFF1FB89FFF1F609DFF1FE29DFF1FCA
:10B16000A29FFF1F349FFF1FB09DFF1FD29DFF1F97
:10B17000E89DFF1F24A0FF1F669DFF1FD89DFF1F96
:10B18000209EFF1F4E9FFF1F469FFF1FDA9DFF1F40
:10B19000569FFF1F1E9FFF1F8E9FFF1F0E214820DF
:10B1A000FFF7B8F80E23FFF7E3BB13214620FFF7A4
:10B1B000B1F81323FFF7D3BB1F214420FFF7AAF8F0
:10B1C0001F23FFF7C3BB00214020FFF7A3F8002394
:10B1D000FFF7AFBB00213E20FFF79CF80023FFF7ED
:10B1E000A0BB00213C20FFF795F80023FFF791BB9F
:10B1F00000213A20FFF78EF80023FFF782BB0021E1
:10B200003820FFF787F80023FFF773BB00213620B3
:10B21000FFF780F80023FFF764BB00213420FFF71D
:10B2200079F80023FFF754BB0C213220FFF772F8A6
:10B230000C23FFF744BB00213020FFF76BF80023FD
:10B24000FFF734BB14212E20FFF764F81423FFF717
:10B2500024BB04212C20FFF75DF80423FFF714BB67
:10B2600003212820FFF756F80323FFF7F3BA012143
:10B270002620FFF74FF80123FFF7E3BA142120201F
:10B28000FFF748F81423FFF7ADBA04211E20FFF79B
:10B2900041F80423FFF79DBA01211C20FFF73AF87B
:10B2A0000123FFF78DBA01211A20FFF733F801239C
:10B2B000FFF77DBA02211820FFF72CF80223FFF7D1
:10B2C0006DBA00211620FFF725F80023FFF75DBABD
:10B2D00002211220FFF71EF80223FFF740BA0C21CB
:10B2E0000E20FFF717F80C23FFF721BA4FF47A610D
:10B2F0000420FFF70FF84FF47A63FFF7C1B94FF45A
:10B30000AF610220FFF706F84FF4AF63FFF7AEB965
:10B31000F8B5CD2007F030FD204B214A054603CB80
:10B320001368C5F803001A0CBC20C5F807102B8061
:10B33000AA70FEF793FF2E46002426F80B0FA0B24A
:10B34000FFF702F8FEF78AFF0234BC2C26F8020F42
:10B35000F5D16C1E05F1C8064FF0FF3014F8013F1F
:10B36000082758400F4B40F300017A1E0B4012F0A3
:10B37000FF0783EA5000F5D1B442EFD1C043FEF796
:10B380007FFF3A46C5F8C900CD21284605F05AFC92
:10B390002846BDE8F84007F0F7BC00BF3C5C010060
:10B3A000385C01002083B8EDF0B50E4B0E4C05461D
:10B3B00093E8070085B024682E88AD7801AB83E858
:10B3C0000700270C184600220B21ADF804408DF829
:10B3D0000670ADF80C608DF80E5005F033FC05B02A
:10B3E000F0BD00BF485C0100385C0100F0B5124BB5
:10B3F000124D1E68124F0FCD87B06C460FC495E8F2
:10B40000030044F8040B38683B79CDF80D00320C8A
:10B410002D2021808DF802208DF81130ADF80060CC
:10B42000FEF71CFF0022ADF80B001221684605F064
:10B4300009FC07B0F0BD00BF385C0100545C01009E
:10B440008C540100002005F079BC00BF03F05EB908
:10B4500070B5104C82B00025402306462946204690
:10B46000009301958023202202F010FB012320226B
:10B4700030462282A3826382E58108F021FA3146B8
:10B480000246204606F0ECF8204602B0BDE87040C7
:10B4900002F0E2B864A0FF1FF0B5CC2983B075D9E3
:10B4A0000546441E00F1C8064FF0FF3014F8012F86
:10B4B00008275040404A40F300017B1E0A4013F029
:10B4C000FF0782EA5000F5D1B442EFD1C043FEF746
:10B4D000D7FE0146D5F8C9000190019A914202D0E9
:10B4E000B2F17F2F0BD105F10B00FEF7BFFEBC2898
:10B4F0000BD03248FFF7ACFF002003B0F0BD30485E
:10B50000FFF7A6FF384603B0F0BD05F10D00FEF7CA
:10B51000ADFE2D2840D1002440F6AC5613E004289F
:10B520001AD0062821D008281FD00A2828D00C2895
:10B5300022D1A1F5FA7292B2B24201D8FEF7EAFE28
:10B540000234BC2C0ED004F10D002844FEF78EFE10
:10B55000022C0146A0B2E2D1B1F5805FEED30234F5
:10B56000BC2CF0D1012003B0F0BDA1F52F7292B236
:10B57000B2F57A6FE4D8E1E7222801D0242811D16E
:10B58000A1F5FA7292B2B242DAD8D7E70D48FFF7C6
:10B590005FFF002003B0F0BD0B48FFF759FF00200C
:10B5A00003B0F0BD2A28C9D1A1F1320292B2B2F59E
:10B5B000967FC5D8C2E700BF2083B8ED985C010034
:10B5C000845C01006C5C0100AC5C010003290CD9B7
:10B5D00070B5461C82B005460C46304603222A4907
:10B5E00008F0DCF910B102B070BD70470B2C05D922
:10B5F00005222649281D08F0D1F940B12448FFF75B
:10B6000027FF244802B0BDE87040FFF7CDBE05F12A
:10B610000901032201A808F011FA01A803221E491A
:10B6200008F0BCF9D8B103221C4901A808F0B6F90A
:10B6300008B301A803221A4908F0B0F9B0B91948B3
:10B64000FFF706FFA11E89B23046FFF725FF00284D
:10B65000C9D0154802B0BDE87040FFF7F9BE1348E5
:10B66000FFF7F6FEFFF754FE1148F3E71148FFF726
:10B67000EFFE1148C6E71148FFF7EAFE02B0BDE849
:10B680007040FFF7B3BE00BF385C0100C45C01002E
:10B69000CC5C0100E05C0100E45C01000C5D010099
:10B6A000245D0100285D01003C5D0100E85C0100B3
:10B6B000FC5C0100505D0100645D0100105D010053
:10B6C0002DE9F043174D2B6883B081460F46904615
:10B6D000F3B1154E34880A1992B2184611463280D9
:10B6E00007F0C8FE28603A464946204402F092FD21
:10B6F000B8F1000F09D031882868FFF767FF286884
:10B7000007F042FB00232B60338003B0BDE8F083D9
:10B71000054E01930846318007F02EFB019B2860FF
:10B720001C46E0E704A1FF1F00A1FF1F10B51D4C40
:10B730004FF4FA70FBF72AFC204601F081FE00234B
:10B74000194601222046E3812382A282628202F00E
:10B7500059FD0B221449204605F082FF204605F0D2
:10B7600095FF0F221149204605F07AFF204605F08B
:10B770008DFF0F490722204605F072FF204605F095
:10B7800085FF204601F068FF0A4B0B4A1A604FF410
:10B79000FA70FBF7FBFBFFF729FE0848BDE81040F5
:10B7A000FFF756BE64A0FF1F685D0100745D0100D5
:10B7B000845D010018A3FF1FC1B600008C5D01006D
:10B7C0000020704790F8392090F83800101A704720
:10B7D00090F8383090F839209A4205D95A1C034421
:10B7E00080F83820187E70474FF0FF30704700BF58
:10B7F00090F8383090F839209A4286BF1B18187E8E
:10B800004FF0FF30704700BF704700BF38B50546A6
:10B81000B0F85E0090B195F85D301446C3F1210296
:10B8200094420CD805F13B001844224602F0F2FC89
:10B8300095F85D30234485F85D30204638BD012001
:10B8400014462871EEE700BFB0F85E306BB190F897
:10B850005D30202B07D8C218013380F85D300120FD
:10B8600082F83B107047012303710020704700BF2E
:10B870000023426980F8383080F8393080F85C3035
:10B8800080F85D3080F85E3080F85F3006CA30B4F2
:10B890000D68046943662A4383660A60A37042699F
:10B8A00090F861301649146813441D7A5B7B01EBF4
:10B8B000C5051B026D6803F4E06343F064032B606D
:10B8C00090F8623013449D7CDB7D01EBC5011B02C7
:10B8D000496803F4E06343F064030B602168536834
:10B8E000194205D0036927225A70036904229A710C
:10B8F000036920225A71036980229A7030BC704714
:10B90000B068010043690CCB12681A420CD0094B95
:10B9100099420AD9084B9942036994BF1A220D2211
:10B920005A70036904229A717047036927225A707A
:10B93000F7E700BF7F1A06003F420F0010B502690B
:10B94000D378DBB2D90604463DD510215806D17014
:10B9500038D503F0040303F0FF02002B51D03D491A
:10B96000626E00230B7084F85D30002A5BD0904734
:10B9700094F85D30002B56D02369D0229A70236949
:10B9800094F83B201A712369012284F85C2002227A
:10B99000DA7010BD304B84F860009C424AD02F4BC7
:10B9A0009C4252D094F8391013791F29DBB207D882
:10B9B0002848007820B16018013184F839100376E6
:10B9C0000223D37010BD5906C3D4917801F0100141
:10B9D00001F0FF000029DDD013F001031ED194F81F
:10B9E0005C1094F85D00884281BF4B1C091984F8F3
:10B9F0005C3091F83B3013712369D0229A70226930
:10BA0000DEE7236984F83920C0229A702369114A3D
:10BA10001979012111700222DA7010BDC0239370D0
:10BA200022691379CCE70122002384F85D2084F891
:10BA30003B30A1E7626994F861300949134403225D
:10BA4000187A02F0B3FF2269ACE7626994F86130BA
:10BA50000449F3E708A1FF1F0092FF1F6C92FF1F2C
:10BA6000C5BA0000D1BA00000369DB7803F02003F7
:10BA700073B190F860300133DBB2012B80F8603095
:10BA80001AD9426990F861301344187A03F00AB861
:10BA900070B5426903F0FF0590F861301344044625
:10BAA000187A02F0FFFFA36E5BB184F8385094F867
:10BAB0003900BDE87040184790F85F30002BE0D0A7
:10BAC000704770BD0148FFF7CFBF00BF0092FF1F56
:10BAD0000148FFF7C9BF00BF6C92FF1F2DE9F04777
:10BAE000374FDFF8E0903B68026982B0064600936A
:10BAF000DDF800800021A025D3789B065BD53B684C
:10BB00000193019BC8EB03030F2BF5D949B1102B0F
:10BB1000F2D000209070336980229A7002B0BDE8A4
:10BB2000F087726996F8613013440521187A03F0A2
:10BB3000B3F9726996F861301344012193F812A0A9
:10BB4000504603F0A9F909240021504603F090F96A
:10BB50002B46013BFDD10121504603F089F92B46CC
:10BB6000013BFDD1013CEFD1706996F861100144B1
:10BB70004FF4A0720C7A4B7B09EBC4011B0249689D
:10BB800003F4E06343F064030B6096F8623003440F
:10BB9000997CDB7D09EBC1011B02496803F4E0637A
:10BBA00043F064030B60013AFDD13269D3789B0600
:10BBB0004FF00101A3D4012002B0BDE8F08700BF1F
:10BBC00010A1FF1FB0680100F0B503691222DA70FE
:10BBD0000269937803F0200385B004460D46002BDC
:10BBE0005ED0B42393703C4922690B680093009E99
:10BBF00005E00B680193019B9B1B042B42D8D37873
:10BC000003F0200303F0FF00002BF2D094F85D3026
:10BC1000002B31D04FF0000E4FF0020C04EB0E035E
:10BC200093F83B3013710B680393039F206907E07F
:10BC30009B060DD50B680293029BDB1B052B28D8B6
:10BC4000C378DBB203F0020202F0FF06002AEFD055
:10BC500080F803C02669F378DBB2DF0632462DD4C4
:10BC60009F062BD5DB0731D40EF1010E94F85D3021
:10BC70005FFA8EFE7345D1D800201DBB002384F8E7
:10BC80005E3004E09070236980229A70042005B031
:10BC9000F0BD86702369802204209A7005B0F0BD43
:10BCA00003F0FF06FFF71AFF10B9042005B0F0BD3E
:10BCB000236984F85F60B0229A7094E78023B370A0
:10BCC0000420DAE726698023B370D7E7BEF1000FBE
:10BCD0000CBF02200320F6E710A1FF1F2DE9F04161
:10BCE00006690025122780F8385080F83950F7701F
:10BCF000D0F810C09CF802E00EF0200E88B0044688
:10BD0000884615461E46BEF1000F49D0B4238CF874
:10BD10000230784B21691A680092DDF800E006E0F5
:10BD20001A6801920198CEEB0000042830D8C87838
:10BD300000F0200000F0FF070028F1D04FEA480291
:10BD400042F00102D2B20A711A680292DDF808E0EC
:10BD5000206906E01A6803920399CEEB01010529D8
:10BD60002AD8C17801F0020101F0FF070029F1D0C3
:10BD70004FF0020C80F803C02269D17811F011074E
:10BD800022D12DBB002E0CBFA0238023937003E093
:10BD90008F70236980229A70384608B0BDE8F08120
:10BDA0000EF0FF07FFF79AFE0028F5D0236984F80C
:10BDB0005F70B0229A70ACE78770236980223846A2
:10BDC0009A7008B0BDE8F081802393700027E3E704
:10BDD000012D75D0A021917021690A79BE46674670
:10BDE0004FF0A80C1A680492049805E01A680592AE
:10BDF000059A121A052A4AD8CA7802F0020202F0FD
:10BE0000FF08002AF2D0CF702169CA78D2B212F0AE
:10BE1000100F08465AD1920658D5013DEDB2012DBA
:10BE200049D0BEF11F0F3BD90A79012DDAD11A682A
:10BE30000692069D05E01A680792079A521B052A8A
:10BE400046D8C27802F0020202F0FF01002AF2D0C6
:10BE50000223C3702269D378DBB2D9063AD49B0699
:10BE600034D5B023BEF11F0F93703FD8226904EB85
:10BE70000E0312791A760EF1010E5FFA8EFE16B1DC
:10BE8000236980229A7084F839E0774684E781F844
:10BE90000280236980229A70774684F839E07BE734
:10BEA00004EB0E0291F8048082F818800EF1010E66
:10BEB0005FFA8EFEB9E781F802C021690846B0E753
:10BEC000A82191702069BE460279B0E7774663E702
:10BED0008170DEE71021A023D170013BFDD12269E2
:10BEE000937803F0F7037746937055E723691B793E
:10BEF000C5E700BF10A1FF1F0148FFF71FBD00BF2E
:10BF00000092FF1F0148FFF719BD00BF6C92FF1F91
:10BF100000220260704700BF30B5056889B0012378
:10BF200000240A460193294602A8009400F006F96D
:10BF300002A800F0ADF9C0B209B030BD30B5056857
:10BF400089B0012400230A468DE8180029460223FF
:10BF500002A800F0F3F802A800F09AF980B209B044
:10BF600030BD00BF0C2901D90020704702314900C3
:10BF700001F0FE01FFF7E2BF2DE9F04303688FB047
:10BF8000012600240D4607461946904633465E2298
:10BF900002A80196009400F0D1F802A800F078F908
:10BFA0005E2D03D0A5F17303072B10D801230024C5
:10BFB000396801932A4608A8009400F0BFF8224689
:10BFC000414608A800F006F90FB0BDE8F0838146AD
:10BFD0002246214602A800F0FDF8396833462A4679
:10BFE0008DE8500008A800F0A9F82246414608A8AC
:10BFF00000F0F0F822465FFA89F102A800F0EAF8B2
:10C000000FB0BDE8F08300BFF8B505460F461646F1
:10C01000412421463A462846FFF7AEFF611C023410
:10C02000C9B232462846E4B2FFF7A6FF592CF0D138
:10C03000F8BD00BF2DE9F843044600689DF8209044
:10C040000E461746984610B1102105F081FB1020CE
:10C0500005F07CFB3A460546314600F057F925606D
:10C060002846012100F078F9054618B90025284630
:10C07000BDE8F883632280212046FFF77DFF012081
:10C0800002F032FF00225E212046FFF775FF5D219E
:10C090002046FFF741FF2428E8D14A464146204682
:10C0A000FFF7B2FF204601222B21FFF765FF204654
:10C0B00001222C21FFF760FF20460E222D21FFF7E1
:10C0C0005BFF204600222E21FFF756FF204601226B
:10C0D0002F21FFF751FF204605223021FFF74CFFAB
:10C0E000204601223121FFF747FF2046002232215E
:10C0F000FFF742FF204600223321FFF73DFF204695
:10C1000000223421FFF738FF204600223521FFF7B7
:10C1100033FF204600225B21FFF72EFF204610222E
:10C120005C21FFF729FF204620225D21FFF724FF35
:10C1300020468C225E21FFF71FFF98E770B49DF820
:10C1400010609DF80C500160002146738573428198
:10C1500003734161416070BC704700BFF0B5438913
:10C16000056885B0DCB21B128DF80C408DF80D30DF
:10C170004DB1437B019303AB00932846012300F0AC
:10C18000FBF805B0F0BD43680BB31746027A0E46C4
:10C190006AB904F07F048DF80C40427B009231466E
:10C1A0003A46184603AB00F055FA05B0F0BD022A36
:10C1B00004D164F07F048DF80C40EEE7012AECD145
:10C1C00004F07F0444F040048DF80C40E5E7184685
:10C1D000D7E700BF02B9027B042A1AD8F0B4416144
:10C1E00000F10F077AB102F10E03867B3C4603444F
:10C1F00000F10E055EB92170013BAB424FEA1121FF
:10C2000004F10104F6D13946F0BCFFF7A7BF19705D
:10C21000F2E70020704700BF70B54489066884B01B
:10C22000E5B224128DF80C508DF80D405EB1437BC1
:10C23000009200241A4630460B46019403A900F0F0
:10C240000BF904B070BD4468FCB1037A7BB965F0AA
:10C250007F058DF80C50437B0092FF251A4620463F
:10C260000B46019503A900F08BFA04B070BD022BB8
:10C2700004D105F07F058DF80C50ECE7012B04BFCD
:10C2800065F03F058DF80C50E5E72046D9E700BF83
:10C2900038B500F10F042146027B0546FFF7BCFFCD
:10C2A00010B94FF0FF3038BD287B0028FBD00E308E
:10C2B0002B18AA7B21460E35002007E01C78013B95
:10C2C000AB4240EA040001F101010AD00002002A59
:10C2D000F4D00C78013BAB4240EA040001F10101CB
:10C2E000F4D138BD70B5044640681E4603685B68EB
:10C2F00015469847854201D0002070BD31466068E0
:10C30000FFF762FCB0FA80F0400970BD30B4002540
:10C3100020240572C4600170426030BC704700BFC9
:10C32000037A10B5044683B1227863680121520074
:10C3300083F83B2083F85E1083F85D106068FFF798
:10C3400043FCB0FA80F0400910BD012100F004F870
:10C350000028E9D110BD00BF38B5044640680D463D
:10C36000FFF786FA0120207205B938BD2046BDE8E6
:10C370003840FFF7D5BF00BF2DE9F041079EC468E4
:10C38000DDF818E09519A54219D8154602789846A7
:10C3900043680F4652000121044683F83B2083F88E
:10C3A0005E1083F85D106EB1BEF1000F0AD04068D8
:10C3B000036871465B6832469847864202D0002087
:10C3C000BDE8F08143462A4639462046BDE8F041A3
:10C3D000FFF788BF2DE9F843C468A24202D90020C4
:10C3E000BDE8F88316468846074601784068D2B211
:10C3F000FFF774FC8642F2D136B30023DFF8549085
:10C400001C4612E090F8383090F839209A4203F137
:10C41000010E00EB03011AD980F838E0087E28707D
:10C420000134A4B2A64223460ED978680268526944
:10C430004A4508EB0305E5D090470134A4B2C0B2E9
:10C44000A64228702346F0D80120BDE8F883FF20DB
:10C45000E5E700BFD1B700002DE9F041C568069FB0
:10C460009DF81C60AA4202D90020BDE8F08190F836
:10C4700000C0D0F804E04FF001084FEA4C0C1D4614
:10C480008EF83BC033468EF85E808EF85D800446A1
:10C49000FFF728FF0028E7D043463A4629462046C2
:10C4A000BDE8F041FFF796BF2DE9F0470468134659
:10C4B0000A4624B12046BDE8F04700F035BB057BB5
:10C4C0000C7886686249B1FBF6F1002D0CBF4FF085
:10C4D00001094FF0800919EA040F0CBF4FF0010C5D
:10C4E0004FF0000CCDB2002B00F0AF804F0107F4ED
:10C4F000FF57114602EB030811F801EB4B460026EB
:10C50000002D50D0002F4ED03A46013AFDD1427B4B
:10C5100012F0F70F40F08D8090F91020013212D008
:10C520001EEA030214BF0124002464450BD0002A34
:10C530006CD0446990F8242094F800C04CEA0202C0
:10C5400022704FF0010C846990F8262094F800A026
:10C550004AEA020222701DB117B13A46013AFDD1F2
:10C5600090F91120013206D0C26990F82540127866
:10C57000224218BF1E43826990F826A0147824EA4C
:10C580000A04147090F91120013201D001F8016CF5
:10C59000027B002A35D15B00DBB2002BB0D188458D
:10C5A000AAD1BDE8F087427B12F0F70FB4D08469BE
:10C5B00090F8262094F800A04AEA0202227090F92E
:10C5C000102001320AD01EEA030F44692AD090F8E5
:10C5D000242094F800A04AEA02022270846990F8AC
:10C5E00026A0227822EA0A02227090F91120013254
:10C5F000CED0C26990F825401278224218BF1E435F
:10C60000C4E75B08002B7FF47BAFC8E7D0F814A029
:10C6100090F824C09AF8004024EA0C048AF80040FC
:10C62000944690E790F824A0227822EA0A02227029
:10C63000D4E7846990F8262094F800A04AEA020220
:10C6400022703A46013AFDD1B9E7BDE8F08700BF54
:10C6500020A107002DE9F0430C4683B001680A9F32
:10C66000064690461D4681B14268CB7A1268002B7F
:10C670004ED10B68D968914207D0394818603949C2
:10C68000DA6042F08040186119600021B07B02F04E
:10C69000EFFB77B105EB07090DF1070715F8013B33
:10C6A0008DF80730012239463046FFF7FDFEA945D7
:10C6B000F4D1B8F1000F0ED004EB08050DF1070717
:10C6C00014F8013B8DF80730012239463046FFF758
:10C6D000EBFEA542F4D10121B07B02F0C9FB336827
:10C6E00093B1DA7A82B1D00703D51F4A99691160F4
:10C6F000DA7A910703D51D4AD9691160DA7A5207AF
:10C7000002D51B4A1B6A1360012003B0BDE8F08309
:10C7100072B6CB7AD80709D5DFF858E0C868DEF8DA
:10C72000003003408B61CEF80030CB7A980709D5F2
:10C73000DFF844E00869DEF800300340CB61CEF852
:10C740000030CB7A5B0708D5DFF830E04869DEF8C7
:10C75000003003400B62CEF8003062B689E700BFBC
:10C7600001403F0000003F8000E100E004E100E004
:10C7700008E100E080E100E084E100E088E100E021
:10C780002DE9F0470D4682B00168DDF828909DF84C
:10C790002C80064617461C4681B14268CB7A126847
:10C7A000002B4FD10B68D968914207D039481860E7
:10C7B0003949DA6042F08040186119600021B07B8D
:10C7C00002F056FB77B105EB070A0DF1070715F8E4
:10C7D000013B8DF80730012239463046FFF764FEF1
:10C7E000AA45F4D1B9F1000F0FD0A1440DF107070C
:10C7F0000122394630468DF80780FFF755FE9DF837
:10C80000073004F8013BA145F2D10121B07B02F0D1
:10C810002FFB336893B1DA7A82B1D00703D51F4A70
:10C8200099691160DA7A910703D51D4AD9691160B7
:10C83000DA7A520702D51B4A1B6A1360012002B044
:10C84000BDE8F08772B6CB7AD80709D5DFF858E093
:10C85000C868DEF8003003408B61CEF80030CB7A38
:10C86000980709D5DFF844E00869DEF80030034096
:10C87000CB61CEF80030CB7A5B0708D5DFF830E02B
:10C880004869DEF8003003400B62CEF8003062B633
:10C8900088E700BF01403F0000003F8000E100E06A
:10C8A00004E100E008E100E080E100E084E100E074
:10C8B00088E100E02DE9F0410468E56815F0807F2B
:10C8C000794D256052D1DF0740F1B380002900F097
:10C8D000E3800D78012B18BF45F0004565630131F9
:10C8E00090F8248003F1FF3C48EA0828BCF1000FCF
:10C8F00000F0A88021B14D7811F8028B45EA082894
:10C9000045682E7ABCF1020F06F1FF364FEA063673
:10C910000CBF48F0805548F01045B6B26563ACF1E5
:10C92000020C08E00AB114700132013B05F47045B5
:10C93000B54216D90468E56A15F0F00FF6D0A46B7D
:10C9400013F0010F17464FEA242EEBD11AB107F866
:10C9500002EB54703A4605F47045B542A3F1020368
:10C96000E8D8BCF1000F6DD00468C3E7DD074CD5F3
:10C97000002900F089800D78012B18BF45F0004593
:10C980006563013103F1FF3E90F824C0BEF1000F52
:10C9900041D029B191F801C00D78023145EA0C2C43
:10C9A00045682E7ABEF1020F06F1FF364FEA0636D1
:10C9B0000CBF4CF080554CF01045B6B26563AEF13B
:10C9C000020E08E00AB114700132013B05F4704513
:10C9D000B54215D90468E56A15F0F00FF6D013F0EA
:10C9E000010F1746A46BEDD122B107F8024B2412B8
:10C9F00054703A4605F47045B542A3F10203E9D8F4
:10CA0000BEF1000F07D00468C3E79E4690F824C02B
:10CA1000BEF1000FBDD11BB30468E16A11F0F00F45
:10CA2000FBD0A16BDC071DD50AB111700132013BAF
:10CA3000F1E790F824809C4648EA0828BCF1000FF2
:10CA40007FF458AF63B10468E16A11F0F00FFBD0D6
:10CA5000DE07A16B0FD50AB111700132013BF1E77E
:10CA6000BDE8F0812AB114460D1204F8021B55707E
:10CA70002246023BCFE72AB114460D1204F8025BAE
:10CA800051702246023BDDE790F82450012B18BF7D
:10CA900045F00045656375E790F82450012B18BFF9
:10CAA00045F0004565631BE700041F8090E80C001B
:10CAB000F0B41C6859682568164F174E2943216049
:10CAC000164D17491760D66015611160417A154AF5
:10CAD0005C180A3194F8244053F8215002EBC40149
:10CAE00049680D60017A5C1803EB8101247ECD69F1
:10CAF00002EBC40149680D60817A581803EB810389
:10CB000090F83000596B02EBC002F0BC536819601A
:10CB1000704700BF01401F0001100038011000786D
:10CB200000001F80B06801000BB1FFF7C3BE704763
:10CB3000704700BFF0B50C1EBDF8146034DBB0F9CF
:10CB400006701919B942C4BF3B1B1BB2002BA64685
:10CB50001CDD002A1146B8BFD11D02F00705CC101C
:10CB6000826A012007FB04E1A840012E0A44C0B2FA
:10CB70001ED00CD3022E09D1013B12FA83F3013AE5
:10CB800012F8011F41409A421170F9D1F0BDC04323
:10CB9000013B12FA83F3C0B2013A12F8011F0140BF
:10CBA00093421170F9D1F0BD23441BB20024C6E7B3
:10CBB000013B12FA83F3013A12F8011F01439A4232
:10CBC0001170F9D1F0BD00BF00291EDB30B4B0F9FF
:10CBD0000A408C4218DD002A16DBB0F90C40944262
:10CBE00012DD047E022C54D0032C4CD0012C06D133
:10CBF0005140C4884A405140013C611A09B2012B9E
:10CC00002DD017D3022B01D030BC7047002AB0F9C9
:10CC10000630856A1446B8BFD41D44F3CF0404FB24
:10CC2000031102F007026B5C012000FA02F25A4085
:10CC30006A54E9E7002AB0F90630856A1446B8BF9D
:10CC4000D41D44F3CF0404FB031102F007026B5C14
:10CC5000012000FA02F223EA02026A54D4E7002A11
:10CC6000B0F90630856A1446B8BFD41D44F3CF042A
:10CC700004FB031102F007026B5C012000FA02F2D0
:10CC80001A436A54C0E70489013C641A114622B26F
:10CC9000B5E7C5880489013D013C691AA21A09B2A9
:10CCA00012B2ACE72DE9F041079E9DF91880089D6E
:10CCB00004461F4600F0BCFF0D4B0E480E4984F899
:10CCC0003380FF22002F08BF1F4684F82F20002347
:10CCD00084F8302084F8312084F8322020606665A2
:10CCE000A565676221662362A3622046BDE8F081E4
:10CCF0000092FF1F185E01000110013810B50446B4
:10CD0000806A034B236008B106F03EF8204610BD50
:10CD1000185E0100F8B5436ADBB190F82C200125BC
:10CD2000AA4083F83B2083F85E5083F85D500446A8
:10CD3000406A03680E461B6800219847606A0368D2
:10CD400031461B6898472946606ABDE8F840FEF7FF
:10CD50003BBFC26BC56C1368046A23EA050313600A
:10CD60004CB122684FF00043D3625163D36A002B69
:10CD7000FCDA936BF8BD836B466B0825802410E0CA
:10CD80003768426C3A4332601F68826C3A431A60DB
:10CD90001A68876C013D22EA07024FEA54041A60C0
:10CDA00007D02142ECD13268476C22EA0702326098
:10CDB000EAE7F8BD70B50446406A0D4600282BD05E
:10CDC000616DFEF79FFD002D20460CBFA621A72117
:10CDD000FFF7A0FF606A20B1A16DBDE87040FEF7CB
:10CDE00091BD216C226D0868236A02430A6093B1E9
:10CDF000DA7A82B1D00703D5224A99691160DA7ACA
:10CE0000910703D5204AD9691160DA7A520702D511
:10CE10001E4A1B6A136070BD236A002B2BD0D97A7F
:10CE2000226EE1B172B6D97ACE0706D51848D96814
:10CE30000668314099610160D97A880706D515489E
:10CE4000196906683140D9610160D97A4E0705D564
:10CE500011485969066831401962016062B61B6861
:10CE6000D968914207D00D4818600D49DA6042F048
:10CE7000804018611960226C216D136823EA010358
:10CE80001360A0E700E100E004E100E008E100E059
:10CE900080E100E084E100E088E100E001403F0043
:10CEA00000003F80436A2DE9F04105460E4690465A
:10CEB000002B3ED090F82C100124A14083F83B10A9
:10CEC00083F85E4083F85D40406A036800211B6878
:10CED00008F1FF379847FFB2B8F1000F23D037446D
:10CEE000A046013E686A16F8011F03681B68984750
:10CEF0000134B742A4B216D01F2CF3D90121686ABD
:10CF0000FEF762FE95F82C206B6A520083F83B20F6
:10CF100083F85E8083F85D80686A036800211B687F
:10CF200098470124DEE7686A0121BDE8F041FEF779
:10CF30004BBEC26BC16C136823EA010306EB080405
:10CF400013604FF00048A6420ED02B6A16F801EB92
:10CF500063B11A68C2F82C80C2F834E0D36A002B9F
:10CF6000FCDAA642936BF0D1BDE8F081AB6BD5F84B
:10CF700034C008208021DCF800206F6C1EEA010F0D
:10CF800014BF3A43BA43CCF800201A68AF6C3A4356
:10CF90001A601A68AF6C013822EA07024FEA5101A1
:10CFA0001A60E8D1CFE700BF70B50446406A0D466D
:10CFB000002828D0616DFEF7A5FC20462946FFF722
:10CFC000A9FE606A20B1A16DBDE87040FEF79ABC71
:10CFD000216C226D0868236A02430A6093B1DA7AF1
:10CFE00082B1D00703D5234A99691160DA7A910793
:10CFF00003D5214AD9691160DA7A520702D51F4A4E
:10D000001B6A136070BD236A002B2BD0D97A226E65
:10D01000E1B172B6D97ACE0706D51948D968066843
:10D02000314099610160D97A880706D51548196998
:10D0300006683140D9610160D97A4E0705D512489A
:10D040005969066831401962016062B61B68D96887
:10D05000914207D00D4818600D49DA6042F08040D7
:10D0600018611960226C216D136823EA01031360B3
:10D07000A3E700BF00E100E004E100E008E100E018
:10D0800080E100E084E100E088E100E001403F0051
:10D0900000003F802DE9F041044686B0806A9DF88B
:10D0A00030801E460F461546B4F90830002800F0BF
:10D0B0004B81DA1D48BF03F10E02B4F90630D210DD
:10D0C00003FB02F2002106F083F9B4F90820202ABC
:10D0D00000F3A780B4F90610A74B0120203A73395A
:10D0E00002EBD27201EBD1714FF0200E029073204F
:10D0F0008DE8014042F34F0241F34F01204600F01A
:10D100004DFE606A84F82D70002800F05181002DDA
:10D1100040F09F80B4F90830202B14BF3D253C25FA
:10D1200084F82C50B8F1000F40F09A8006B394F9BF
:10D130003300002818DBC0B2012101F0ADFE01214F
:10D1400094F8330001F094FE012001F0CDFE00219F
:10D1500094F8330001F08CFE0A2001F0C5FE012195
:10D1600094F8330001F084FE606A002800F0988093
:10D17000616DFEF7C7FB042280492046FFF792FE4F
:10D18000217A0139C9B22046FFF7C4FD7C49042247
:10D190002046FFF787FE94F92D30012B14BF142190
:10D1A00010212046FFF7B6FD042276492046FFF7FE
:10D1B00079FEB4F906308F22802B84F85C2000F0D1
:10D1C000A580602B00F0B1800225DA212046FFF710
:10D1D000A1FD29462046FFF79DFD81212046FFF74E
:10D1E00099FD94F85C102046FFF794FDD921204664
:10D1F000FFF790FD94F92D30012B14BFF12122216E
:10D200002046FFF787FD204606225F49FFF74AFECA
:10D21000606A58B3A16DFEF775FB012006B0BDE84A
:10D22000F081B4F90610594B0120403A52394FF0C1
:10D23000400E029002EBD272522001EBD1718DE8C8
:10D24000014042F34F0241F34F01204600F0A6FD9A
:10D2500057E76DB284F82C50B8F1000F3FF466AF79
:10D26000FEF706FB002E3FF47FAF60E7216C226DD6
:10D270000868236A02430A6073B1DA7A62B1D007A0
:10D2800003D5434A99691160DA7A91076FD452073E
:10D2900002D5404A1B6A1360012006B0BDE8F08148
:10D2A000236A002B2BD0D97A226EE1B172B6D97ADB
:10D2B000CF0706D53848D9680568294099610160CB
:10D2C000D97A8E0706D53548196905682940D9618C
:10D2D0000160D97A4D0705D531485969056829405B
:10D2E0001962016062B61B68D968914207D02D4867
:10D2F00018602D49DA6042F0804018611960226C94
:10D30000216D136823EA0103136034E7B4F9083090
:10D31000402B7FF459AF94F92D30012B14BFCF234C
:10D320009F2384F85C3012254FE7B4F90830102BA6
:10D330007FF44AAF94F92D30012B14BFAF23102393
:10D3400084F85C30022540E7DA1D48BF03F10E0285
:10D35000B4F90630D21003FB02F21046059205F034
:10D360000BFDA06200283FF459AF059AAAE60F4AC8
:10D37000D9691160DA7A8AE7685E010048600100C5
:10D380004C60010050600100546001005C600100CD
:10D3900000E100E008E100E080E100E084E100E07D
:10D3A00088E100E001403F0000003F8004E100E030
:10D3B000012194F83100214F01F06EFD94F8320004
:10D3C000012101F069FD94F9312094F9323057F8C8
:10D3D0003220E26357F83330206A23640125E56484
:10D3E00025651A682A431A6048B1B8F1000F3FF466
:10D3F00039AFFFF75BFB002E3FF4B6AE97E6294648
:10D4000094F82F0001F048FD294694F8300001F00F
:10D4100043FD94F92F2094F9303057F8322062639D
:10D4200057F833306564A5641A68A36322F00102DB
:10D430001A60002E3FF498AE79E600BFB068010094
:10D44000B0F90820D31D48BF02F10E03B0F9062041
:10D45000806ADB1002FB03F2002105F0B9BF00BFB8
:10D46000F0B50029BDF814502EDBB0F90660B142CA
:10D470002ADA002A59DBB0F9087014461C44BC4271
:10D48000C4BFBB1A1BB2002B1EDDD2B2D408D0F829
:10D4900028E016FB041112F00702DBB20EEB0104C8
:10D4A00021D0C2F10807FAB2374F9342BF5C0CD2C9
:10D4B000C3EB020CFF2646FA0CF6012D07EA06071D
:10D4C0003FD005D3022D36D0F0BD012D39D030D25A
:10D4D0001EF8016026EA07070EF801709342F3D3A5
:10D4E000B0F906100C449A1AD2B2072A10D9022DAC
:10D4F00036D0002D14BFFF26002613462670083BA9
:10D50000B0F90610DBB2072B0C44F7D802F0070283
:10D51000002AD9D01D4B012D9B5C1DD017D3022DA5
:10D52000D2D1227853402370F0BD13441BB20022A5
:10D53000A1E7022D25D11EF8016077400EF8017099
:10D54000CCE71EF8016037430EF80170C6E7227879
:10D5500022EA03032370F0BD227813432370F0BD49
:10D5600011462378DB4323700839B0F90630C9B27D
:10D5700007291C44F5D812F00702A5D0034B9B5C89
:10D58000CFE73444AFE700BF085E0100F85D01005B
:10D5900070B4047EBDF80C50022C18D0032C1FD0A0
:10D5A000012C0BD0002A03DBB0F90840944201DCC7
:10D5B00070BC7047039570BCFFF7BCBAC488039574
:10D5C000013CA41A0A4621B270BCFFF749BF068984
:10D5D000C488013E641AB21AE41A12B221B2E1E719
:10D5E00004890395E41A641A114622B270BCFFF74D
:10D5F00037BF00BF70B4057EBDF80C60022D1AD095
:10D60000032D12D0012D03D0039670BCFFF728BF65
:10D61000C488E41AA41A0A4621B2002A03DBB0F92E
:10D620000840944213DC70BC70470489013C641AC2
:10D63000114622B2F1E7C48805890396013CAD1A70
:10D64000ED1A621A11B22AB270BCFFF709BF039635
:10D6500070BCFFF76FBA00BF2DE9F8430446406A7B
:10D66000002863D0616DFEF74DF90522744920460C
:10D67000FFF718FCA1790139C9B22046FFF74AFB30
:10D68000B4F90820E588A66AD31D48BF02F10E034D
:10D69000DB10626A15FB03F51FFA85F8002A7BD0C0
:10D6A00094F82C300125AB4082F83B3082F85E5074
:10D6B00082F85D50606A036840211B6808F1FF37FB
:10D6C0009847BFB2B8F1000F23D03744A846013EB7
:10D6D000606A16F8011F03681B6898470135B74256
:10D6E000ADB216D01F2DF3D90121606AFEF76CFA96
:10D6F00094F82C20636A520083F83B2083F85E8004
:10D7000083F85D80606A036840211B6898470125A3
:10D71000DEE70121606AFEF757FA606A002800F030
:10D720008D80A16DBDE8F843FEF7ECB8236A002BAD
:10D730002BD0D97A226EE1B172B6D97ACE0706D54E
:10D740004048D9680568294099610160D97A8D07F8
:10D7500006D53D48196905682940D9610160D97A23
:10D76000480705D53948596905682940196201609B
:10D7700062B61B68D968914207D0354818603549B0
:10D78000DA6042F0804018611960226C216D1368E4
:10D7900023EA0103136068E7E26BE36C1168276A10
:10D7A0000B4306EB080913604FF0004E4E450DD0B9
:10D7B00016F801CB2FB33A68C2F82CE0C2F834C097
:10D7C000D36A002BFCDA4E45936BF1D1226C236DAA
:10D7D00011680B43136097B1FB7A83B1D90703D566
:10D7E0001D4BBA691A60FB7A9A0703D51B4BFA697D
:10D7F0001A60FB7A5B0702D5194B3A6A1A60BDE8DA
:10D80000F883A36BD4F8348008208021D8F8002056
:10D81000656C1CEA010F14BF2A43AA43C8F8002014
:10D820001A68A56C2A431A601A68A56C013822EAA6
:10D8300005024FEA51011A60E8D1B7E7276AC5E748
:10D84000005E010080E100E084E100E088E100E0AA
:10D8500001403F0000003F8000E100E004E100E003
:10D8600008E100E02DE9F04F85B09946BDF9387028
:10D87000BDF83CA0BB1AC1EB090B002BB8BF5B4243
:10D88000BBF1000FB8BFCBF1000B5B450D46164650
:10D890000093804648DC4D453A4633464CDC1946F9
:10D8A00013460A46C5EB09019B1A89B2002B0CB23C
:10D8B000B8BF5B4204EBD474BE42ACBF4FF0FF3242
:10D8C00001224D45039102924FEA640429DC9BB288
:10D8D00001930DE0D8F80070BF69B847019BE41AC6
:10D8E000A3B21CB20135002C2DB211DBA94518DB07
:10D8F000009B5B452A46534631464046EADCD8F851
:10D90000002053469769294632464046B847E5E726
:10D91000029A1644039AA94502EB030436B224B2D4
:10D92000E6DA05B0BDE8F08F4A462B46B9463546E3
:10D930004D4517461E46B2DD304629463E464D4609
:10D9400007468946AEE700BF10B404682469A446C0
:10D9500010BC604730B40468BDF808500295A46B51
:10D96000A44630BC604700BF30B40468BDF808501E
:10D970000295E46BA44630BC604700BF70B40468F5
:10D98000BDF90C60BDF8105003960495246CA446B4
:10D9900070BC6047704700BF10B582B0B0F90C2072
:10D9A00001910168009200220C6CB0F90A30114616
:10D9B000A04702B010BD00BF704700BF01F00301D7
:10D9C0000129017606D0032904D0C2880389428147
:10D9D000838170470289C38842818381704700BF79
:10D9E0002DE9F0410568134E6F6986B0B7420446D1
:10D9F000BDF8308010D1013B13441BB20093CDF829
:10DA000004800B46AD6A2046A8472368DB6AB34210
:10DA10000AD106B0BDE8F081059304920391B8479E
:10DA200003A925680EC9E6E7204606B0BDE8F04127
:10DA3000184700BF95D900002DE9F0410568124E46
:10DA40006F6986B0B7420446BDF830800FD1013B04
:10DA5000CDF804800B4400921BB2AD6A2046A84763
:10DA60002368DB6AB3420AD106B0BDE8F0810593B2
:10DA700004920391B84703A925680EC9E7E7204639
:10DA800006B0BDE8F041184795D900002DE9F04FE8
:10DA90000568DFF858B06F6985B05F450646BDF987
:10DAA0003890BDF83CA00C46904615D11F19BC42D9
:10DAB0000CDACDF800A0214601342D6A4B464246CF
:10DAC000304624B2A847BC423568F2DBEB6A5B45BE
:10DAD00007D105B0BDE8F08F0393B8473568039BC5
:10DAE000E4E7304605B0BDE8F04F184795D900008F
:10DAF0002DE9F04387B099420546BDF93840BDF89D
:10DB00003C6025D0A24212D00768DFF88080D7F8A9
:10DB10001490C14532D18DE850002846BC6AA04718
:10DB20002B68DB6A434524D107B0BDE8F0839942F6
:10DB300002DD08461946034628680E96C46B013379
:10DB40005B1A1BB22846A44607B0BDE8F043604705
:10DB5000A24202DD134622461C4628680E96631C2C
:10DB6000846B9B1A1BB22846A44607B0BDE8F0435D
:10DB70006047284607B0BDE8F04318470593049274
:10DB80000391C84703A92F680EC9C4E795D90000BF
:10DB90002DE9F04FD0F800E0DFF89090DEF814B0F7
:10DBA00083B0CB450446BDF93080BDF834A00D46A6
:10DBB00017461E4631D1CDF800A0DEF824B0294624
:10DBC00033463A462046D8472368CDF800A008F1EE
:10DBD000FF323A44D3F824B0294612B233462046E5
:10DBE000D8472368CDF800A02946D3F820B03A469C
:10DBF00043462046D8472068CDF800A0711E29442E
:10DC00004346056A09B23A462046A8472368DB6ABC
:10DC10004B4506D103B0BDE8F08FD847D4F800E0FB
:10DC2000C9E7204603B0BDE8F04F184795D900007A
:10DC3000F0B4002401254FF6FF76094F0760047108
:10DC40000476C48104828476C461C5758575457681
:10DC500086824682C180028141818281F0BC704708
:10DC6000246301002DE9F04F85B00668BDF84450EB
:10DC7000BDF93880CDF8008004460195D6F848B04B
:10DC80000392BDF93C60BDF9407089469A46D84779
:10DC900023680195009742465146D3F848802046B4
:10DCA0003346C0472068039B0E930F95856C4B4607
:10DCB0003A4631462046AC4605B0BDE8F04F6047D5
:10DCC0002DE9F04F87B01746BDF940400091254639
:10DCD000E91D059344BF2B4603F10E010268BDF810
:10DCE000486053690294C91003912B49BDF944401F
:10DCF00001968B42824645D1002C3CDD029B3C4480
:10DD00005E1EB6B24FF0000923B2049301364D46B1
:10DD1000029B002B28DD059B002403EB090806E08D
:10DD2000EDB22B0604F1010411D4A6421CD0A1B21D
:10DD300011F0070F23B24FEA4505F1D1002BB8BF10
:10DD40000733DB10013418F803502B06EDD5009B88
:10DD5000D2F818B019443A4609B2019B5046D84748
:10DD6000A642DAF80020E2D1039B01379944049BD4
:10DD70003FB2BB42CCD1D36A074A934206D107B027
:10DD8000BDE8F08F9847DAF80020B5E7504607B0B5
:10DD9000BDE8F04F184700BF95D9000070B4BDF939
:10DDA0000C60BDF91050BDF814400396049505941D
:10DDB00070BCFFF785BF00BF2DE9F04F91B08346DF
:10DDC0000591C169BDF8680006909DF87400BDF822
:10DDD0006C709DF870A0039002929946002900F0A3
:10DDE000CC800B7A48680A68C3EB0903DBB215469E
:10DDF00000EBC30230F83360D3780993BAF1010F16
:10DE000092F9053092F802800E9392F9064079D982
:10DE1000BDF93830089323B20B93A94BDBF80020EF
:10DE20000F93194653698B4240F0A280099B002B47
:10DE300053D0BDF808300C930021234407910D9373
:10DE40000F460C46A946B8F1000F3FD0BDF81C1094
:10DE50000B9BBDF80C000297CB1813FB00F30C983A
:10DE600003440D981BB2014404930BB20A9300259E
:10DE700005E00135EBB264009845E4B223D9029B7A
:10DE80002B44590703D1731C19F806409EB2230690
:10DE9000EFD5089BE918059B11FB0AF1BAF1010FB8
:10DEA000194402D1039B012B1ED0069B0193039BB7
:10DEB0000093D369049A1F4609B253465846B8479F
:10DEC000DBF80020D5E7029F4744FFB2079B099982
:10DED00001330793DBB29942B5D8D36A0F9A9342C4
:10DEE00041D111B0BDE8F08F0E9B05995918936987
:10DEF0000A9A29441F4609B2069B5846B847DBF8E0
:10DF00000020B6E7039B012B82D800230B930893D4
:10DF100083E70799099A0131013A49B212F0FF02E9
:10DF20000791099260D1069A4A454F4617D0BAF137
:10DF3000010F03D1039A012A00F0B5800A9A0898CC
:10DF400002EB8201039AD2008DE88400084401B2FA
:10DF5000DC69029A53465846A047DBF80030DB6A7A
:10DF60000F9A9342BDD0584611B0BDE8F04F184704
:10DF700058469847DBF8002058E7BBF90A30059966
:10DF80008B42AEDDBBF90C3002988342A9DD06233B
:10DF900013FB0A13002BA4DD039B00EBC303002B30
:10DFA0009FDD9BF81A3033B9B9F1AF0F84BF09F187
:10DFB00001035FFA83F9424ADBF800300F92114601
:10DFC0005A698A426AD1BDF8142008920522099242
:10DFD000002207921FFA8AF20A92CDF830900FFAC7
:10DFE0008AF2B946039F05920799BDF83040089D13
:10DFF0000522104610FB04120A98324C06460846C9
:10E0000001FB0651A65C15FA80F209B212B2049126
:10E010000B92082400251CE0BAF1010F01D1012F59
:10E0200024D0069A0192029A009705FB0722D3F8A2
:10E030001C800499059B12B25846C047DBF800309B
:10E04000013C013514F0FF046DB24FEA56063FF46F
:10E0500060AFF007E0D4069A4A45F1D0BAF1010F5B
:10E0600001D1012F0ED0CDF80490DCE7029AD3F84D
:10E0700018800B99069BAA1812B25846C047DBF8C5
:10E080000030DDE7029AD3F818800B99AA184B46A6
:10E0900012B25846C047DBF80030D1E758469047E7
:10E0A000DBF800308FE70899CDF8009005311C6A45
:10E0B000029A082309B25846A047DBF800304EE721
:10E0C00095D9000074630100F0B5C36985B00446BA
:10E0D0003BB30A296FD00D294FD01A7A91424CD305
:10E0E000987A884249D38A1A5D68D2B205EBC20594
:10E0F000AA78002A56D0E878002853D0607E0028FD
:10E100003ED095F905E0B4F90E00A67DB4F90A7089
:10E11000724406FB0202BA4269DCE77DB4F91020C2
:10E1200034E00A295CD00D2927D0427E002A50D045
:10E13000B0F90E00A57DB4F90A60062212FB0502B3
:10E14000B242E67D42DD228AE38102EBC60212B2D0
:10E1500018462282B4F814E0678A03960B460295AB
:10E1600001468DE880402046FFF726FEA37DE28928
:10E1700003EB430302EB4303E381012005B0F0BD51
:10E18000A67DE77DB4F90E00B4F91020B4F814E0D0
:10E190000397678A02960B468DE880400146204629
:10E1A000FFF70AFE2979E389A27D012001FB0233F2
:10E1B000E38105B0F0BD0022C2811A7BC17D038AD4
:10E1C00001FB02330382012005B0F0BDB4F9102039
:10E1D000C0E7857DC67DB4F91020B0F90E00B9E71F
:10E1E000028AC17DC38102EBC1030382C5E700201F
:10E1F000E0811B7B228AE77D03FB072212B2228289
:10E20000C4E700BF11B18175C175704701218175E7
:10E21000C1757047844641EA000313F003036DD1D2
:10E22000403A41D351F8043B40F8043B51F8043BD9
:10E2300040F8043B51F8043B40F8043B51F8043BE0
:10E2400040F8043B51F8043B40F8043B51F8043BD0
:10E2500040F8043B51F8043B40F8043B51F8043BC0
:10E2600040F8043B51F8043B40F8043B51F8043BB0
:10E2700040F8043B51F8043B40F8043B51F8043BA0
:10E2800040F8043B51F8043B40F8043B51F8043B90
:10E2900040F8043B51F8043B40F8043B51F8043B80
:10E2A00040F8043B403ABDD2303211D351F8043B20
:10E2B00040F8043B51F8043B40F8043B51F8043B60
:10E2C00040F8043B51F8043B40F8043B103AEDD2CF
:10E2D0000C3205D351F8043B40F8043B043AF9D220
:10E2E000043208D0D2071CBF11F8013B00F8013BF3
:10E2F00001D30B8803806046704700BF082A13D300
:10E300008B078DD010F003038AD0C3F10403D21A17
:10E31000DB071CBF11F8013B00F8013B80D331F84B
:10E32000023B20F8023B7BE7043AD9D3013A11F8CB
:10E33000013B00F8013BF9D20B7803704B78437036
:10E340008B78837060467047374A384913681B06DC
:10E35000FCD40B6813F08003F8D172B634490A7804
:10E36000002A5FD0334A3448F0B4344C176806684A
:10E370002568D4680C303E44143200681268304F6F
:10E3800035442C4420440244C2F34E022D4E2E4804
:10E390002E4D2F4C42F400423A60376806682D68D3
:10E3A0002C4A24680C303E44006812682A4F3544D9
:10E3B0002C4420440244C2F34E02284E2848294DE2
:10E3C000294C42F400423A60376806682D68274AB3
:10E3D00024680C303E4400681268254F35442C44B4
:10E3E00020440244C2F34E02224E2348234D244CC3
:10E3F00042F400423A60376806682D68214A246872
:10E400000C303E440068126835442C4420440244D9
:10E41000C2F34E021C4842F4004202600B7062B626
:10E42000F0BC704762B6704724B0034024B00B4084
:10E430000AA1FF1F38B003403CB0034040B0034086
:10E440002CB0034058B003405CB0034060B00340C0
:10E4500064B003406CB0034030B0034038B00B40B0
:10E460003CB00B4040B00B4044B00B404CB00B40B4
:10E470002CB00B4058B00B405CB00B4060B00B4070
:10E4800064B00B406CB00B4030B00B4030B4294846
:10E49000294A2A4B2A4D6024E121047011701B780F
:10E4A000284C082B30D00A2B2748284937D00C2B72
:10E4B0000CBF35223D2212232A60236002600B60CC
:10E4C000234B24491B78244ABBB101230B60136002
:10E4D000224B23491B78234A012B26D9042B0FD921
:10E4E000082B1ED9102B94BF862387230B60136043
:10E4F0001D4B01221A7030BC70470B601360E7E7B8
:10E5000084230B601360F3E700F58E200F49083079
:10E51000012213232A60236002600B60D0E73922B6
:10E52000F7E785230B601360E2E780230B6013603D
:10E53000DEE700BF0040074001400740D892FF1FC0
:10E5400008B003400CB0034008B00B400CB00B40C7
:10E550000DA1FF1F20B0034020B00B40D992FF1F38
:10E5600024B0034024B00B400AA1FF1F0C2830B494
:10E5700017D91023984228BF18461C46104A114D3F
:10E580001178181A8C42287018D00F4913700B7824
:10E5900023B10E490E4A00230B60136030BCFFF715
:10E5A00075BF0A2802D90C231C46E7E7082802D9C0
:10E5B0000A231C46E2E708231C46DFE730BC70470D
:10E5C000D892FF1F09A1FF1F0AA1FF1F24B003401B
:10E5D00024B00B4028282FD8334B2DE9F0411E5C86
:10E5E000FF2E2BD0314B1B78002B2AD132062CD496
:10E5F00072B62F4D2F4C2F46012326602B7062B62A
:10E6000072B623681B060CD43B781BB9F4E72B7851
:10E61000002BF1D062B603F0A1F872B62368180699
:10E62000F5D5254B1B6800222A7062B6234A107864
:10E6300043FA00F0BDE8F081002070470020BDE8FB
:10E64000F081FFF781FE3206D2D572B61C4DDFF89D
:10E650007C801C4C06F04007FFB206F03F06D8F85D
:10E660000030DFB123F01003C8F80030012326602A
:10E67000134A2B7062B672B6236819060CD413784D
:10E680001BB9ECE72B78002BE9D062B603F066F8F3
:10E6900072B623681B06F5D50B4BC3E743F0100396
:10E6A000C8F80030E2E700BF746801000AA1FF1F4C
:10E6B0000CA1FF1F00B0034010B0034009A1FF1FD1
:10E6C0000BA1FF1F00B00B4010B00B400CB00B4073
:10E6D0000A4A0B49136843F4805313600B7843B91B
:10E6E000084BC0221A70084B80F30C0000B218804F
:10E6F0007047044B80221A70F5E700BF2C8004405D
:10E700000DA1FF1F21C00C4000C00C40F0B51B4BF9
:10E710001B4E596818689A68DB6885B06C460FC450
:10E72000337899071DD5174A174C1378174913F0FA
:10E73000700318BF1370164A164B802717700026F7
:10E740003320032226706D4608701A7072B6043C9E
:10E7500045F001052046A84762B6237813F0700300
:10E7600009D10D4B064901E0013B02D00A78D207DE
:10E77000FAD505B0F0BD237005B0F0BDA06801006A
:10E780000100024000000240040002400B00024071
:10E79000070002400A000240410D0300B0F5006F7F
:10E7A0000AD210B5094B1B78DB07044606D504F1E5
:10E7B000A0500078C0B210BD00207047FFF7A6FF40
:10E7C00004F1A0500078C0B210BD00BF01000240AB
:10E7D000B0F5006F17D238B50F4B1B78DA070D462E
:10E7E000044611D504F1A0500378AB420AD00B4A7D
:10E7F000137813F0700318BF1370074A057013786D
:10E80000DB07FCD538BD7047FFF780FF04F1A0504F
:10E810000378AB42EBD1F5E7010002400000024073
:10E8200008B5104C08E0236859050DD423681A0573
:10E830000FD42368DB0411D423685803F3D501F007
:10E8400087FB23685905F1D500F00EF823681A05F7
:10E85000EFD500F02DFF2368DB04EDD501F0EAF9D8
:10E86000EAE700BF3480044008B5FFF7D9FF00BFD6
:10E87000014B10221A80704700200540704700BFEE
:10E88000094908B50B6830B16A461844A2F58052B0
:10E89000904202D20860184608BD04F03FFA0C23EB
:10E8A00003604FF0FF3008BDDC92FF1FFEE700BFA2
:10E8B000EFF3138070B9EFF310836BB9EFF30582B8
:10E8C0005AB94FF48070EFF311832BB1984228BFEF
:10E8D000184670474FF0FF3070470F2A01D818468E
:10E8E000F1E7014BD05CEEE7F0E300E0704700BFDA
:10E8F00010B40F4B53F8302092F880422CB1012312
:10E9000069B182F8803010BC704703EBC0035B68CC
:10E910001A6841B922F002021A6010BC704782F8EE
:10E92000003110BC704742F003021A6010BC7047FF
:10E93000B06801001C4A02EBC00301295B6811D0DA
:10E9400004291BD052F83000002280F8802229B11F
:10E95000022920D0032922D01A6070474FF4807218
:10E960001A60704752F830004FF4A27280F880129B
:10E970001A601A6822F020021A60704752F83010AC
:10E980004FF4A272012081F880021A601A6842F0E6
:10E9900020021A60704740F203121A6070474FF469
:10E9A00081721A60704700BFB0680100212848D802
:10E9B000F8B5042A44D8DFE802F0484B4E0345007E
:10E9C0004FF410262B4B03EBC0030D465C68216807
:10E9D00011F4E06148D0284B284A2949C3F89C210A
:10E9E00004F140422748C3F8A411A2F59221264F12
:10E9F000C3F8A0017C292548C3F8A871C3F8AC016D
:10EA00002CD9A2F594237C2B2AD9A2F596237C2B12
:10EA100028D9A2F598237C2B29D9A2F59A227C2A01
:10EA200027D81B4872B6236823F4702343F0807202
:10EA3000C4F384011643236040F82150266062B677
:10EA4000F8BD70474FF43026BCE74FF40026B9E715
:10EA50004FF44026B6E74FF42026B3E70D48E1E730
:10EA60000D48DFE70D48DDE7FFF764FFB3E70C482B
:10EA7000D8E7F8BDB06801000082FF1FF188FF1FD2
:10EA80009988FF1FC588FF1F6D88FF1F4188FF1FE2
:10EA9000B893FF1FE092FF1F1893FF1F6893FF1F9B
:10EAA0009893FF1F1A4B03EBC00010B4426802F1A9
:10EAB0004043A3F592217C2923D9A3F594217C29F5
:10EAC0000DD9A3F596217C291FD9A3F598217C297E
:10EAD00019D9A3F59A237C2B11D80E4C00E00E4CCB
:10EAE00072B613680D4823F08773C2F3840123F4D0
:10EAF000803343F08073136044F8210062B610BC89
:10EB00007047074CECE7074CEAE7074CE8E700BF23
:10EB1000B0680100B893FF1F1893FF1FEDE80000D5
:10EB2000E092FF1F9893FF1F6893FF1F30B4054BBF
:10EB3000054D064C002210211A602A6020601960E1
:10EB400030BC704714D0034004D0034000D00340D1
:10EB5000282838B52ED0002904464FDD5F4B1B789E
:10EB6000012505FA03F28A4202D8212837D938BD97
:10EB70000338C2B2012A3AD9202C4AD0192C48D0E5
:10EB8000574A126802FB011222FA03F31D2800F211
:10EB90009B80DFE800F0928B847D9999766F99993C
:10EBA0009999999999999968615A53994C99999910
:10EBB00099999945494B1B780B2B08D90C2B1CBFF5
:10EBC0000C3B19410846BDE83840FFF781BDC3F151
:10EBD0000C0399400846BDE83840FFF779BD294647
:10EBE000FFF786FE2946BDE83840FFF7A3BE3D4A41
:10EBF000126802FB011222FA03F3C7E72128B6D8F4
:10EC00000021FFF775FE20460121BDE83840FFF7DF
:10EC100091BE354A126802FB011222FA03F3B5E7EE
:10EC20003249334A0B604FF45173136038BD314998
:10EC3000314A0B604FF45173136038BD2F49304A8D
:10EC40000B6040F24443136038BD2E492E4A0B60DE
:10EC500040F24443136038BD2C492D4A0B6040F20A
:10EC60004443136038BD2B492B4A0B6040F24443A8
:10EC7000136038BD29492A4A0B6040F244431360AF
:10EC800038BD2849284A0B6040F24443136038BD20
:10EC90002649274A0B6040F24443136038BD25499A
:10ECA000254A0B6040F24443136038BD2349244A8F
:10ECB0000B604FF45173136038BD2249224A0B6038
:10ECC0004FF45173136038BD212C3FF650AF7F29AC
:10ECD000D4BF00210121204693E700BFC093FF1F4E
:10ECE000088003400890034008800B4010800B40D0
:10ECF00048A0044018800B404CA0044018800340FA
:10ED000008B004401080034004B004404080034039
:10ED100018C004403880034014C0044028800340D9
:10ED200010B00440208003400CB004403080034009
:10ED300010C00440488003401CC0044018900340A9
:10ED400034900440109003403090044038B11028B3
:10ED500028BF1020044AC3B2107813707047024ACB
:10ED60000123107813707047C093FF1F2DE9F843FB
:10ED70000E4680463249334D304603F05BFF47F67E
:10ED8000122300281ABF1D464FF002094FF0010957
:10ED9000002425FA04F003F057FD4FF05E510746BA
:10EDA00003F0AAFD0146304603F058FF30B90134A4
:10EDB000072CEED1E80903F047FD074631463846F7
:10EDC00003F04EFE4FF07C5103F08CFC03F080FF0B
:10EDD0004FF6FF729042A8F1030328BF1046012BA3
:10EDE00029D9B8F1170F17D8174B23FA08F303F0F6
:10EDF000010383F0010223B9B8F1190F0FD0BDE868
:10EE0000F883124B124D13491A6044EAC9042A6070
:10EE100008601C60BDE8F883B8F1200FECD10E4B00
:10EE20000E4D0F49002244EAC9041A602A600860A6
:10EE30001C60BDE8F8830B4B0B4D0C49F2E700BF9B
:10EE4000001BB740006CDC026006F000008003404D
:10EE5000048003400880034000800B4004800B4086
:10EE600008800B400090034004900340089003404A
:10EE7000212801D8FFF73CBD704700BF212806D8E4
:10EE8000044B53F8303093F80002C0B270470020B2
:10EE9000704700BFB0680100212801D8FFF74ABDC4
:10EEA000704700BF72B60C490C4B0D4A1B680868CE
:10EEB000126862B6520102D5322B88BF013009496F
:10EEC000C3F5BB334FF47A72FF33A1FB031302FB8C
:10EED00000F000EB9310704710A1FF1F18E000E056
:10EEE00004ED00E0ABAAAAAA2DE9F843054672B6E4
:10EEF000204F214B214A1B683C68126862B65201C0
:10EF000002D5322B88BF013495B3C3F5BB331C4EF9
:10EF1000DFF86490DFF86480FF334FF47A72A6FB69
:10EF2000031302FB04F404EB931472B6D9F8001037
:10EF30003A68D8F800E062B6C1F5BB33FF33A6FBF0
:10EF400003031EF0806FC4EB93134FF47A7002D06A
:10EF5000322988BF013200FB0233B3F57A7F04D334
:10EF6000013D05D004F57A74DFE702F0F7FBDCE73A
:10EF7000BDE8F88310A1FF1F18E000E004ED00E0F9
:10EF8000ABAAAAAAF8B52D4B2D49DFF8D0E0DFF8DF
:10EF9000D0C02C4E2C4D2D4C2D4A2E4F4FF400003E
:10EFA00018604FF0807018604FF0007018604FF0DC
:10EFB000806018604FF0006018600020086028230F
:10EFC0004BF6FF71CCF80010CEF8003033601360C0
:10EFD0002B6023603B60B3629362092245F8242CC6
:10EFE000C4F8D80F05F57F65C7F8D41F07F5FF27CC
:10EFF00007F5FA67C6F8F83F2B6006F5FF26C4F858
:10F00000D42F05F5FD2504F5FF24386006F2F476CB
:10F010001148316005F5FF6504F5FD642B60236040
:10F020000260FFF733FA1920FFF75EFF01F0F6FCEC
:10F0300040F21310BDE8F840FFF756BF08E100E0CA
:10F040000480034014800340248003402C8003404C
:10F050001C8003403480034000800B400C80034040
:10F06000088003402B4A2C491368F0B543F4006331
:10F0700013600A78294F2A4E2A4D2B4C2B49002326
:10F08000092A3B7033702B7023700B703DD01A2A05
:10F0900021D0274B1B780A2B25D01F2B30D01F28BF
:10F0A00027D8002002460125224B234C1A70234901
:10F0B0005D7004224FF0020E88273C26402598728E
:10F0C0009A704FF4004083F813E05A751F74DE7095
:10F0D00025700860F0BD1A4B40F213321A60144BD1
:10F0E0001B780A2BD9D1174B4FF451721F281A6085
:10F0F000D7D9C0F34432C0F3471500F01F00D3E75F
:10F10000114B4FF451721A60C9E7104B40F21332A1
:10F110001A60BEE734800440C193FF1F84A1FF1F23
:10F1200019A1FF1F8CA1FF1F85A1FF1F18A1FF1FA1
:10F13000C293FF1F00B006402FE400E004E100E0AE
:10F1400004D0044010B0044000D004400CB004408F
:10F15000144B14499B7803F0EC0200F003031343B3
:10F16000420700F00F0248BF43F01003042A8B70DF
:10F1700013D00C4B0B4A5B79C10603F0EF0348BF79
:10F1800043F0100353719379820603F0EF03054AAD
:10F1900048BF43F01003937170478B7943F04003ED
:10F1A0008B71E6E700B00640234B1B681B0542D578
:10F1B00010B5224C237823B102F0D0FA2378002B2B
:10F1C000FAD11F481F4A204B4FF40044002104602D
:10F1D000D1701B78092B1FD01A2B03D11B4B40F287
:10F1E00003121A601A4B1B7803F07F030A2B1DD001
:10F1F0001F2B03D1174B40F203121A60164A114B12
:10F200001648174912681C79DB79002303700B70CC
:10F210000AB10123137010BD124B40F203121A60A1
:10F220000B4B1B7803F07F030A2BE1D10E4B40F20E
:10F2300003121A60E2E770473480044018A1FF1FF0
:10F2400084E100E000B00640C193FF1F04D00440F9
:10F25000C293FF1F00D0044014A1FF1F84A1FF1F11
:10F2600019A1FF1F0CB0044010B004400A4A38B581
:10F270000546137803F0FF04002BFAD1012128463C
:10F28000FFF70AFE21462846FFF7F2FD034A044B2A
:10F2900052F835201A6038BD18A1FF1FB068010070
:10F2A00088A1FF1F09B140F08000174A13789842E7
:10F2B00016D010B4154C246824050FD503F07F0335
:10F2C0000A2B1CD01F2B11D0002900F07F0114BF86
:10F2D000602344230A290DD01F2902D0107010BCCE
:10F2E00070470B4943F440730B60F7E7084B002469
:10F2F0001C60E9E7074943F440730B60EEE7054BF8
:10F3000000241C60E0E700BFC293FF1F348004406C
:10F3100000D0044010B00440124B1A7882420CD046
:10F3200011490968090507D5092A16D01A2A0AD0F1
:10F3300009280DD01A2801D0187070470B4A40F2E6
:10F3400013311160F8E7094A002109281160F1D151
:10F35000074A40F213311160EEE7054A00211160BF
:10F36000E6E700BFC193FF1F3480044004D004408F
:10F370000CB004400D4B1B6813F4006305D021282A
:10F3800005D90B4B00201860704718467047094B91
:10F3900010B5074C53F8303023600121FFF77CFD96
:10F3A000236800221A70012010BD00BF3480044081
:10F3B00014A1FF1FB06801000C4B1B6813F400631D
:10F3C00006D0172806D00A4A537B03F0FE03537376
:10F3D00000207047074B064A40F202311960537B08
:10F3E00043F0010353730120704700BF3480044091
:10F3F00000B0064008B004402DE9F84F234B1B68CD
:10F400001A053BD5224B1B680BB101221A70DFF89D
:10F410009090204D99F80040DFF888801E4E01340E
:10F42000272C8ABF4FF0000A5FFA84FA5446074639
:10F43000AB462B789C4216D1FFF73AFA40281FDCE6
:10F4400033791B06F5D59BF800300133272B86BF97
:10F4500000221346DAB218F80330DBB2F3712A70D7
:10F460002B789C42E8D00D490B4BFFB20120BC2207
:10F4700008F80470087089F800A0DA70BDE8F88F09
:10F48000FF28D6DD02F06AF9D3E700BF34800440DC
:10F4900088A1FF1F85A1FF1F00B0064018A1FF1F14
:10F4A0008CA1FF1F1CA1FF1F2DE9F84F294B1B68E2
:10F4B0001A0548D5284B1B6805460BB101221A7066
:10F4C00005EB010A554540D2DFF89C80234CDFF85C
:10F4D0009C90234F0AE015F8012B09F80B20214AD4
:10F4E0000123AA45137088F800602ED098F80030E8
:10F4F000227803F1010BBBF1270F86BF0026B3462C
:10F500005FFA8BF69345E6D1BC22FA7005E03A79B2
:10F5100013060BD422789345DDD1FFF7C9F94028B3
:10F52000F5DDFF28F6DD02F019F9F3E72278013264
:10F53000272A86BF00210A46D1B219F80220D2B28A
:10F54000FA712170E6E7BDE8F88F054BBC22DA704E
:10F55000BDE8F88F3480044088A1FF1F85A1FF1FFC
:10F5600000B0064018A1FF1F8CA1FF1F1CA1FF1FA8
:10F5700010B5044C237823B102F0F0F82378002B67
:10F58000FAD110BD18A1FF1F064A074B1B7810784F
:10F59000DBB2C0B283422CBF273000F1FF30C01A6B
:10F5A000704700BF85A1FF1F8CA1FF1F054A064BB6
:10F5B00010781B78C0B2DBB2984238BF4030C01A16
:10F5C000704700BF84A1FF1F19A1FF1F30B4154B66
:10F5D000154C1A782378D2B2DBB29A421ED001338E
:10F5E0003F2B0ED91149124B087819680023C0B27D
:10F5F000237021B1D31A1A2B01DC00230B7030BC0D
:10F6000070470A480A49C05C0968DDB2C0B225707B
:10F610000029F4D09A4238BF4032EBE74FF0FF3078
:10F62000EDE700BF84A1FF1F19A1FF1F44A1FF1F29
:10F6300014A1FF1F084A094B12781B78DBB29A42CB
:10F6400007D00133402B28BF0023054AD05CC0B24D
:10F6500070474FF0FF30704784A1FF1F19A1FF1FB3
:10F6600044A1FF1F0D4B1B681B0516D530B40C4B76
:10F670000C4CDA780C480D4902F0CB024025DA70C8
:10F680005D74DA7842F03402DA7023780268DBB213
:10F690000B700AB10023137030BC704734800440F3
:10F6A00000B0064019A1FF1F14A1FF1F84A1FF1F76
:10F6B000F0B4384B1A7912F0300F2CD072B6997D15
:10F6C00001F0FF0200293DD062B6334F334938784C
:10F6D0000D78334E1C46C0B2EDB2431C402BE1798D
:10F6E00028BF0023AB4202F1FF32C9B21CBFF15464
:10F6F000184612F0FF02F0D12A4B1B68C2B23A70D2
:10F700004BB1A84236BFC5F14005401B4019272820
:10F71000C4BF01221A701F49CA78D2B2150616D486
:10F7200052060DD51B4B1B795B0609D51E4B1F4995
:10F730001B6800220A7003B11A70164B3C22DA7063
:10F74000F0BC70474022D9795A7462B6E3E70B796E
:10F750001C06E5D5164B174E1C783378E4B2DBB2A5
:10F760009C420ED0144D01E0A3420AD00133282B55
:10F7700028BF00230879E85CC0B2C871087D07285B
:10F78000F2D9DBB2034933700B79180644BF7C23EE
:10F79000CB70C5E700B0064084A1FF1F19A1FF1F71
:10F7A00044A1FF1F14A1FF1F88A1FF1F18A1FF1F65
:10F7B0008CA1FF1F85A1FF1F1CA1FF1F2DE9F84F82
:10F7C000214B1B6807460BB101221A70DFF88890A5
:10F7D0001E4D99F80040DFF884801D4E0134272C1F
:10F7E0008ABF4FF0000A5FFA84FA5446AB462B7882
:10F7F000A34216D1FFF75CF840281FDC33791B06C3
:10F80000F5D59BF800300133272B86BF0022134625
:10F81000DAB218F80330DBB2F3712A702B78A34206
:10F82000E8D00C490A4BFFB208F804700120AC2262
:10F83000087089F800A0DA70BDE8F88FFF28D6DDDF
:10F8400001F08CFFD3E700BF04A2FF1F01A2FF1F3E
:10F8500000C0064000A2FF1F08A2FF1F98A1FF1FC3
:10F860001C4BDFF894C01A681B49F0B542F4805273
:10F870001A4D1A60DFF884E0194F1A4E1A4C002313
:10F880008CF800304FF451722B701F2840F2133562
:10F890008EF800303B70337025600A6012D819462C
:10F8A0000124124A124D11701248547000212C2765
:10F8B000402693724FF4003491701174D7702E70FB
:10F8C0000460F0BDC0F34431C0F3471400F01F03DF
:10F8D000E7E700BF348004400CC0044095A1FF1F3F
:10F8E00001A2FF1F00A2FF1F08C0044000C0064085
:10F8F00031E400E004E100E094A1FF1F08A2FF1F33
:10F90000144B14499B7803F0EC0200F003031343FB
:10F91000420700F00F0248BF43F01003042A8B7027
:10F9200013D00C4B0B4A5B79C10603F0EF0348BFC1
:10F9300043F0100353719379820603F0EF03054AF5
:10F9400048BF43F01003937170478B7943F0400335
:10F950008B71E6E700C00640F8B5134B1B68DB046B
:10F960001FD5124C237823B101F0F8FE2378002B29
:10F97000FAD10F4B0F4A104D104F114E114C124837
:10F980004FF4003119600023D37040F20311396045
:10F99000316029681579D2792370037011B1012380
:10F9A0000B70F8BDF8BD00BF3480044000A2FF1FFB
:10F9B00084E100E000C0064090A1FF1F08C00440A1
:10F9C0000CC0044094A1FF1F95A1FF1F0A4A38B53F
:10F9D0000546137803F0FF04002BFAD101212846D5
:10F9E000FFF75AFA21462846FFF742FA034A044B2A
:10F9F00052F835201A6038BD00A2FF1FB068010020
:10FA000004A2FF1F09B140F080000F4A137898420A
:10FA100019D010B40D4C2468E40412D503F07F0310
:10FA2000082B02D10A4B00241C60002900F07F0340
:10FA300014BF60214421082B03D1054B41F44071D0
:10FA40001960107010BC7047C393FF1F34800440CE
:10FA50000CC00440704700BF0D4B1B6813F480536B
:10FA600005D0212805D90B4B002018607047184697
:10FA70007047094B10B5074C53F830302360012113
:10FA8000FFF70AFA236800221A70012010BD00BF98
:10FA90003480044090A1FF1FB06801000C4B1B682C
:10FAA00013F4805306D00E2806D00A4A537B03F085
:10FAB000FE03537300207047074B064A40F20231A1
:10FAC0001960537B43F0010353730120704700BF5B
:10FAD0003480044000C0064004C00440034B1B684F
:10FAE000DB0401D5FFF76ABE704700BF34800440D5
:10FAF00070B5094E04464518AC4204F101040AD021
:10FB00003368DB04F8D514F8010CFFF757FEAC425C
:10FB100004F10104F4D170BD3480044010B5044CEC
:10FB2000237823B101F01AFE2378002BFAD110BDFF
:10FB300000A2FF1F064A074B1B781078DBB2C0B249
:10FB400083422CBF273000F1FF30C01A704700BF3E
:10FB500001A2FF1F08A2FF1F054A064B10781B7861
:10FB6000C0B2DBB2984238BF4030C01A704700BF05
:10FB700094A1FF1F95A1FF1F30B4154B154C1A78A7
:10FB80002378D2B2DBB29A421ED001333F2B0ED97A
:10FB90001149124B087819680023C0B2237021B1B3
:10FBA000D31A1A2B01DC00230B7030BC70470A48B3
:10FBB0000A49C05C0968DDB2C0B225700029F4D0E2
:10FBC0009A4238BF4032EBE74FF0FF30EDE700BF1D
:10FBD00094A1FF1F95A1FF1FC0A1FF1F90A1FF1FB0
:10FBE000084A094B12781B78DBB29A4207D00133DE
:10FBF000402B28BF0023054AD05CC0B270474FF0AD
:10FC0000FF30704794A1FF1F95A1FF1FC0A1FF1FE8
:10FC1000054B064A1B7806491268DBB20B700AB125
:10FC200000231370704700BF95A1FF1F90A1FF1F15
:10FC300094A1FF1F30B42B4B1A7994061FD52A4884
:10FC4000DA790378294901333F2B0978C8BF0023AB
:10FC50008B42D2B203D0264CD9B2E2540170254A6D
:10FC6000116861B1244A1278D2B2934236BFC2F110
:10FC700040029B1A9B18272BC4BF01230B70194A03
:10FC8000D378DBB2180611D45A060DD5154B1B7963
:10FC90005B0609D5194B1A491B6800220A7003B18B
:10FCA0001A70104B2C22DA7030BC7047117909069B
:10FCB000EAD5144910480C780178C9B28C420DD0AD
:10FCC0004A1C272A84BF00210A460F4D054C98BFC5
:10FCD000D1B2AA5CD2B2E2710170D5E76C21D170C9
:10FCE000D2E700BF00C0064094A1FF1F95A1FF1FEF
:10FCF000C0A1FF1F90A1FF1F01A2FF1F04A2FF1FB1
:10FD000000A2FF1F08A2FF1F98A1FF1F21282FD8C4
:10FD1000184B195CFF292BD0174B184ADFF870C01D
:10FD200003EBC000F0B54368DFF868E0144F154DF1
:10FD3000154E00241C60DEF80030012043F0200343
:10FD40008840CEF8003014604FF4A07338602E6005
:10FD5000C2F800C0013BFDD113689B05FCD42023F1
:10FD6000013BFDD1094B09B233F8110080B2F0BD5F
:10FD700000207047C0690100B068010000500440D5
:10FD800008500440045004400000020300510440A5
:10FD900080014A0038800440431E032B14D872B6F9
:10FDA0000A4951F8230068B170B4094C058834F849
:10FDB0001320466841F82360521B24F8132062B6D2
:10FDC00070BC704762B670470020704764A2FF1F86
:10FDD000BCA3FF1F013803280BD872B6074B53F89A
:10FDE000203043B100205B680130002BFBD162B6AC
:10FDF0007047002070471846F9E700BFB8A2FF1F00
:10FE000030B472B62B4A13781D0706D52A4B196AEF
:10FE1000002936D0996A002941D053781C0706D5AD
:10FE2000254B196C00293ED0996C002939D0937864
:10FE3000190705D5204B196E002936D0996E89B166
:10FE4000D3781B0707D51C4BD3F880207AB3D3F89F
:10FE5000882011213AB162B6184B00221A7030BCCA
:10FE600000F058BE0D21154C154D227843F8315045
:10FE700003EBC1030830013A5860227062B630BC0F
:10FE8000704704220D4C0F4D217843F8325003EB9C
:10FE9000C20308304A1E5860227062B6EFE705219F
:10FEA000E1E70921DFE70822ECE70C22EAE710226C
:10FEB000E8E700BFA86A01000080FF1FE1A2FF1F62
:10FEC000C800400088004000431E032B1DD81B4A79
:10FED000400140F0100030B4104472B6184CE25C9F
:10FEE000032A1BD8DFE802F00212151703220D883F
:10FEF000E25410F0080F14BFC823882343EA0543D7
:10FF000008310360416062B630BC7047083002229D
:10FF1000EDE70522EBE708300422E8E7094A52F84A
:10FF2000230038B1084A52F82300416042F82310F8
:10FF300062B6E9E742F82310034AF7E70080FF1FA3
:10FF4000F0A2FF1FB8A2FF1FC8A2FF1F00BE00BF84
:10FF50002DE9F04FDFF820B3DFF820A387B044E0AD
:10FF6000AF4F4FEA930807EBC809013ED9F80420C8
:10FF700003F00803F6B2A2F1080003F0FF04002B1F
:10FF800040F00B8157F838301B0C99B222F8081C4E
:10FF9000002B00F0F980A34B22F8064C42F8044CE9
:10FFA00053F82620002A00F075819F4D55F8263021
:10FFB00058609E4C45F8260034F81630194424F851
:10FFC000161000F087FD002800F05D81984A994BDB
:10FFD00019F0080F00F1080018BF1346C9F8040013
:10FFE00047F8383008238BF800309BF80040E4B223
:10FFF00065071DD5904B1B78BBB190490A7802F07C
:020000021000EC
:10000000FF032AB1013BDBB20B70002B00F001852E
:100010008B490A7802F0FF032AB1013BDBB20B7077
:10002000002B00F02D8100F073FE04238BF80030CC
:1000300004F0080303F0FF02002B00F0DA809AF8C6
:100040000030DBB21E098BD19A08DFF8D49159F841
:10005000321009EBC200C1F38301013940680C2959
:100060007DD8DFE801F080807C7C7C7C7C7C467CD9
:100070007C7C0700D0F800E0724C4168724F734EF0
:100080006160C4F800E01FFA8EF140F2816E002535
:10009000674B49F83230012071453D60C9F8105076
:1000A000C9F8185030705E4A00F20881B1F5D06F7F
:1000B00080F08283B1F5817F00F0668300F28F8249
:1000C000802900F07483822940F0A782A18801F082
:1000D0007F01042900F2A1825D4B5E4A89000B4436
:1000E0001570557019788D0740F1808310700220CB
:1000F000F2E2554F3A6842B3574B544E574918886D
:1001000034780D784028864645F0020828BF4FF025
:10011000400E002C84F001043470CEEB00000CBFC4
:100120008824C82409EBC80680B285F0010544EA9A
:100130000E447260188049F8384072440D7018B946
:10014000BEF1400F18BF00223A603E4B1A88B2F54C
:10015000A06F04D100219A785970414B1A70414A1E
:10016000012313703EE7374C258842F221018D426E
:1001700000F05A8224683C49324D8C4200F00082E3
:100180002B4949F83210EAE7294A2A4B19F0080F9F
:1001900018BF134647F8383024E700F0BBFC334A59
:1001A000334952F82630002B78D058688C5D42F8DD
:1001B000260003F10802C9F80420032C05D8DFE863
:1001C00004F0120F150204228A551A8819F0080F3C
:1001D0000CBF8823C82343EA024347F8383001E7BD
:1001E00002228A55F1E703228A55EEE705228A5555
:1001F000EBE7E00700F13082210600F15F82A20701
:1002000006D51C4A1C4913780220DBB21370087013
:10021000E30602D5184B10221A7007B0BDE8F08F24
:100220000080FF1F64A2FF1F10A2FF1FBCA3FF1FBF
:10023000C800400088004000ECA2FF1F75A2FF1F0D
:1002400060A3FF1FD8A2FF1F0CA2FF1F74A2FF1FF5
:10025000C0200740E4A2FF1F20A2FF1FE0A2FF1F53
:10026000982007409420074021090003B8A2FF1FEF
:10027000F0A2FF1F88200740802007409020074001
:1002800000F0ACFFCFE6AC4A47F8380013780133F2
:100290001370A7E643F82600A84D8AE68B5D032B72
:1002A00000F26B8201A252F823F000BFE5FF0000CC
:1002B000E5FF0000AD060100A706010040F621158C
:1002C000A94200F0358100F29F81B1F5086F00F07E
:1002D000FF81B1F5106F40F0A0819948116AA478B0
:1002E00004700C0600F19382D9F828209549100675
:1002F00000F18882D9F830209249120600F17D82FF
:10030000D9F838208F49130600F17282D9F84020BD
:100310008C49150600F12E83D9F848208949140626
:1003200000F12383D9F850208649100600F1188384
:10033000D9F858208349120600F10D83D9F86020BE
:100340008049130600F12083D9F868207D491506FD
:1003500000F11583D9F870207A49140600F1DE8285
:10036000D9F878207749100600F1D382D9F8802097
:100370007449120600F1E982D9F888207149130600
:1003800000F1DD82D9F890206E49150600F1D18286
:10039000D9F898206B49140600F1C5826A486B4A67
:1003A0006B4901906B486C4C644D02940023049798
:1003B000059680461C4617460E460395386828B1B8
:1003C000456800F0A7FB2846002DF9D100233B60CB
:1003D000039B30681A46002342F8243028B1456850
:1003E00000F098FB2846002DF9D100223260019AD6
:1003F00098F800301146002241F8042B029A01912E
:10040000023B4FF0000122F81410032B09D8DFE85B
:1004100013F050010400500104004FF0010388F86C
:1004200000300134042C07F1040706F1040608F13A
:100430000108C3D1494C404D2278494B049F059E89
:100440000021100729701A7000F14E824549627828
:100450000A700021C9F83010C9F838101107DFF808
:10046000E48000F12C82A2783F49DFF8D8800A703E
:1004700000211207C9F85010C9F8581000F108827D
:10048000E2783A492F4C0A7013074FF00001C9F87F
:100490007010C9F8781000F1BF8133780293002200
:1004A00083F00105C9F89020C9F898200020019038
:1004B0008046864602462E490C7844F0020C09EB31
:1004C000CC030393029B002B039B5A600CBF882232
:1004D000C82242EA080384F0010249F83C30357032
:1004E0000A70DFF860C0234BDFF88480002840F0FA
:1004F0001681BEF1400F1BD142F0020C09EBCC0378
:10050000019ADFF840E05A60002D40F01E8105049A
:1005100045F088059DF808304EF83C500244337091
:100520000C701346402803D10020134A3B60108012
:10053000124A0123137012E6E1A2FF1F10A2FF1F4F
:10054000ECA2FF1F0080FF1FC8A2FF1F64A2FF1FB5
:10055000B8A2FF1FF0A2FF1FBCA3FF1FA86A0100E3
:10056000C4200740C8200740CC200740D0200740C7
:10057000E0A2FF1F74A2FF1F20A2FF1F94200740CC
:100580006C68B1498C427FF4FBAD0178A9297FF4F6
:10059000F7AD417845297FF4F3AD8178C2297FF426
:1005A000EFADC1786B297FF4EBADA849A84E087870
:1005B000347880F00105002C40F002000D700CBF73
:1005C0008821C82184F0010449F8301009EBC000EB
:1005D000A04934700025052445600C70D0E540F238
:1005E0000232914240F09480A28802F07F02042AF5
:1005F00013D865888DB998490290920011440A7801
:1006000042F002020A7051E740F62122914200F0C6
:10061000828042F2212291427DD08F4A0F231370B3
:100620008E4A012313709AE58849894E0D783778F0
:1006300085F0010E002F45F0020581F800E00CBFA7
:100640008821C82149F8351009EBC50587F0010755
:100650000021377069608DE5814B80487B491A61C4
:100660004FF0020E80F800E07B4F0A707D49196060
:1006700099607D4E7D4D7E4C9A610D213970FF2130
:100680003170DFF808E2297022707A4D7A4A8EF8CC
:1006900000109F27012406F8047C5D600470DA6076
:1006A00007B0BDE8F08F01238B559BE400238B55E9
:1006B00098E44FF0000388F80030B2E666496B4BCF
:1006C00080220D2008701A70A2077FF5A1AD98E571
:1006D0006A496B4A09781170E588854280F0898102
:1006E0005A490C78402DAE4644F0020C28BF4FF01A
:1006F000400E02EB0E0309EBCC0001930123426094
:100700004FEA0E48CEEB050002930025C822E0E632
:10071000B1F5A06F81D1012300250293C6E64028E0
:100720007FF6EAAE42F002020CEBC201019E4E607F
:10073000BDB19DF8085053491D703346403888F8C4
:10074000004040334CF83210EFE69DF8083033702B
:100750000504019B0C7045F0C80503444EF83C505D
:10076000E0E69DF808501D70019B3E4988F8004066
:10077000403840334CF83210D7E619F0080F0CBF60
:10078000022303238B552DE4A28802F07F02042A62
:100790003FF643AF6588002D7FF43FAF2E490290AE
:1007A000920011440A7822F002020A707EE6344A6E
:1007B0000220157055708FE733494A68002A3FF4CC
:1007C0002CAF6588B4F804E004E00C314A68002AD4
:1007D0003FF423AF0B88AB42F7D14B887345F4D17C
:1007E0002D0A032D0CBF1078088975E7022073E7E6
:1007F000C86B083800F08EF988E5486B083800F0BF
:1008000089F97DE5C86A083800F084F972E5506A14
:10081000083800F07FF967E500F05CF9002800F087
:10082000D68008300F4AC4F88400C4F8802000F055
:1008300051F9002800F0C5800830124AC9F88C0030
:10084000C9F8882029E600BF01000400E0A2FF1FCC
:1008500074A2FF1F75A2FF1FC0200740942007400D
:100860000080FF1F8800400088200740802007404C
:100870009820074024A2FF1F78A2FF1FECA2FF1FB1
:10088000E4A2FF1FC8004000AC6A01008C200740B2
:1008900000F020F9002800F0A68008305D4AC8F872
:1008A0006400C8F8602000F015F9002800F0958079
:1008B0000830594AC9F86C00C9F86820E0E500F032
:1008C00009F9002877D00830524AC8F84400C8F81F
:1008D000402000F0FFF8002867D008304E4AC9F8E1
:1008E0004C00C9F84820BEE500F0F4F8002856D0C6
:1008F0000830484AC9F82400C9F8202000F0EAF876
:10090000002846D00830444AC9F82C00C9F82820ED
:100910009CE5C86F083800F0FDF827E5486F0838F7
:1009200000F0F8F81CE5D1F89C00083800F0F2F867
:1009300034E5D1F89400083800F0ECF828E5D1F857
:100940008C00083800F0E6F81CE5D1F8840008387F
:1009500000F0E0F810E5C86D083800F0DBF8EDE4D1
:10096000486D083800F0D6F8E2E4C86C083800F0AA
:10097000D1F8D7E4486C083800F0CCF8CCE4C86E65
:10098000083800F0C7F8E5E4486E083800F0C2F80F
:10099000DAE42A78C9F8280001322A7056E52A7864
:1009A000C9F8200001322A70A8E72A78C9F848005F
:1009B00001322A7057E52A78C8F8400001322A70BF
:1009C00087E72A78C9F8880001322A7065E52A7815
:1009D000C4F8800001322A7029E72A78C9F8680033
:1009E00001322A704CE52A78C8F8600001322A707A
:1009F00059E74028864628BF4FF0400E02EB0E0311
:100A000001930123CEEB00004FEA0E48002502932C
:100A100051E500BE88004000C80040002DE9F843C1
:100A2000204C00F037FF002204F1A00023461A609A
:100A30005A60083383424FF00001F8D11A4A1B4F25
:100A400013681B4D1B481C4EDFF87880DFF878C018
:100A5000DFF87890DFF878E043F480231360C4F384
:100A600007233B70C4F307432B70240EFF2302F5CA
:100A700028320470114D88F8003011488CF800308D
:100A8000D4323370012389F8003070268EF80010BC
:100A90004FF40074102107F8183C2E700460117098
:100AA000BDE8F8830080FF1F348004409C2007408D
:100AB000B0200740B42007401020074049E400E080
:100AC00008E100E08020074088200740942007408C
:100AD0000021074072B60D480268B2FA82F30F2B6C
:100AE00010DC4FF00041D94022EA0102026062B6F8
:100AF000074803EBC303DB00C2180021C1501046B6
:100B00005160704762B60020704700BFC493FF1F5A
:100B1000BC83FF1F0D4B0E4AC31AA2FB03231B0904
:100B20000F2B0CD80B4A127852B972B60A484FF004
:100B30000041026821FA03F31A43026062B670476B
:100B4000064A1278002AF0D0FFF75AB9BC83FF1F7B
:100B5000398EE338E1A2FF1FC493FF1FECA2FF1FF1
:100B600038B50E4B0E4C1B68218805468BB1B1F58C
:100B7000917F05D20B4A4B1C55549BB2238038BD44
:100B80000022084898470021064A55540123238033
:100B900038BDB1F5917FEDD338BD00BF18A3FF1F5D
:100BA000C6A3FF1FCCA3FF1F2DE9F843214E224F00
:100BB0003168012380463B70B1B1204D4B8801EB79
:100BC0008302013300240F2BC2F808802C7004D854
:100BD0004B8000233B70BDE8F88340230B8003204B
:100BE000FFF772F93460F4E7DFF8549099F80030B9
:100BF000002BF0D0114D45F6215408E0013C12D0F5
:100C00002B7883B900F0AAFD99F800307BB103205E
:100C1000FFF7E0F80528F1D8FFF75CFF01463060E8
:100C20000028EBD0CAE701232B70BDE8F883BDE8AC
:100C3000F88300BF34A3FF1F08A3FF1F38A3FF1FC3
:100C4000ECA2FF1F1201F8B5D5B2A1B3012943D020
:100C50004378044600781B0643EA004040F47040A5
:100C600045F004068F1E3043FFF79EFF022F04F16C
:100C7000020314D9053414F8023C14F8032C14F8B8
:100C8000010C1B0443EA0223334343EA0060033FA1
:100C9000FFF78AFF022F234604F10304EBD8022F4B
:100CA00023D0012F0DD045F4774040F00500BDE87A
:100CB000F840FFF779BF14482843BDE8F840FFF734
:100CC00073BF187845F4770545F0060545EA00201E
:100CD000BDE8F840FFF768BF03780C4845EA0345D4
:100CE0002843BDE8F840FFF75FBF1A78587845F011
:100CF000774545F0070545EA022545EA0040BDE88D
:100D0000F840FFF751BF00BF06F0F70007F000F70B
:100D100038B5084B1C7824B9074D296809B14B88B0
:100D200003B938BD9B000B800320FFF7CDF82C6082
:100D300038BD00BF08A3FF1F34A3FF1F2DE9F041FA
:100D4000AD4E33680746002B00F092801D885A880C
:100D5000910803EB81010432AA428C6842D25A8086
:100D600004F00F064FEA1428A449A6F1080208F07F
:100D70000F00C4F30313062A00F101050B701AD902
:100D8000B31E012B5FFA88F04ED9052E48D0042EF1
:100D900000F0A481731F022B7FD90F2E0ED1F728EC
:100DA00042D8F02802D0964B1B883BB1FFF7D8FE03
:100DB0000020BDE8F08127B1BD4202D00020BDE88F
:100DC000F081082EC4F3033300F08780092E11D080
:100DD0000A2E40F094800A2BF0D18A4B8A4A1B6875
:100DE000A02181E01846FFF795FE0420FEF7D4FF0E
:100DF0003060B5E7092BE1D1270E00F07B81834BF2
:100E0000814A1B689021C4F307461170EDB2FCB211
:100E1000002B00F09D80224631462846984797E0F7
:100E2000F02843D9F72841D0F1380E28C6D801A3BD
:100E300053F820F0EB0F0100CF0F0100BD0F0100B0
:100E4000BD0D0100BD0D0100AF0F0100BD0D010082
:100E50008F100100BD0D0100591001007310010039
:100E6000970F0100BD0D01007F0F0100630F01000E
:100E7000674B1B78002BA1D00420FEF78DFF0346A3
:100E8000306000289AD00588002D7FF460AFFFF70E
:100E900041FE35602846BDE8F081FFF761FEC4F3EE
:100EA0000740FFF75DFE072E02D1200EFFF758FE28
:100EB000534B584A198858481468584D524A017083
:100EC00000270E0AF0201F802E7010700CB3012234
:100ED0005348A0470120BDE8F081082B7FF46EAF96
:100EE000504B494A1B688021C4F307461170EDB28C
:100EF000240E6BB3284622463146984728E00B2E35
:100F000011D10B2B7FF45AAF474B3F4A1B68B021DE
:100F1000EAE7464B1B68002B00F0FB8040489847EF
:100F20000120BDE8F0810C2E40F000810C2B7FF4F5
:100F300045AF3F4B344A1B68C0211170EDB2C4F37A
:100F40000746002B00F0C88028463146240E9847FB
:100F50003849314A314B0D7016701C700120BDE8C4
:100F6000F081354B1B68002B00F0D6809847C4F306
:100F70000746254BEDB2240E83F80080E8E72F4B9F
:100F80001B68002BF2D12E4B1B68A3B1FE209847A3
:100F9000C4F30746EDE72B4B1B68002BE6D1284B2B
:100FA0001B6843B1FC209847C4F30746E1E7264B92
:100FB0001B68002BDAD1C4F30746DAE7234B1B6822
:100FC000C4F30746002BD4D030469847D1E7204BD6
:100FD0001A68002AEFD0260C630C06F07F0003F499
:100FE0007E531843F6B29047C3E71A4B1B68C4F30D
:100FF0000746002BE8D1BCE740A3FF1FCAA3FF1F91
:10100000C6A3FF1F1CA3FF1FC4A3FF1F50A3FF1FE6
:10101000ECA2FF1F18A3FF1FC8A3FF1FC9A3FF1F38
:10102000CCA3FF1F48A3FF1F4CA3FF1F30A3FF1F2C
:101030000CA3FF1FCBA3FF1FF8A2FF1FFCA2FF1FE3
:1010400000A3FF1F3CA3FF1F2CA3FF1F44A3FF1FF0
:1010500014A3FF1F28A3FF1F3F4B1B68002B85D144
:101060003E4B1B68002BA6D0FA209847C4F30746D6
:101070007FE73B4B1B68002B7FF478AF374B1B6837
:10108000002B98D0FB209847C4F3074671E7354BF7
:101090001B68002B7FF46AAF304B1B68002B8AD093
:1010A000F8209847C4F3074663E70E2B7FF486AE1B
:1010B0002D4A2E4B1268E0211970002A47D0260CC9
:1010C000610C06F07F0301F47E511943EDB2A1F5E6
:1010D000005128469047F6B2240E39E7FFF740FD4D
:1010E000C4F30740FFF73CFD200EFFF739FD002059
:1010F000BDE8F0811E4B1D4A1B6880211170EDB2C6
:10110000C4F3074683B1314628463A4698473C46E1
:101110001EE70120BDE8F081104B1B68002B3FF457
:101120004AAFFF20984746E71C4611E70D2EBCD179
:101130000D2B7FF443AE0F4B0C4A1B68D02111706E
:10114000EDB2C4F30746002B7FF4FEAEC4E7C4F350
:101150000746EDB2240EFBE624A3FF1F00A3FF1FEA
:1011600004A3FF1FF4A2FF1F10A3FF1FC4A3FF1FB0
:1011700048A3FF1F20A3FF1F38B5164D2868E0B114
:1011800001884488A14213DD03191B7A83B104F15D
:101190000803C2180C1B002302E012F8011F21B142
:1011A0000133A342F9D1204638BD1C46204638BD44
:1011B000FFF7B0FC0020286038BD074B1B780BB947
:1011C000002038BD0220FEF7E7FD28600028D7D1B7
:1011D000F6E700BF5CA3FF1FECA2FF1F0D4B1B78BF
:1011E000BBB910B50C4C216803F0FF024B883F2BB4
:1011F00007DC07330B4401F1470003F8012F83425A
:10120000FBD140230B800120FEF75EFE002323600C
:1012100010BD704754A3FF1F58A3FF1F70B5EFF315
:10122000108272B60C4C206880B10C4E00254369C8
:10123000236073B19D6102B962B6457783689847B0
:10124000EFF3108272B620680028F0D102B962B6BE
:1012500070BD3360EFE700BF64A3FF1F68A3FF1FEB
:10126000FFF7DCBF024A136801331360704700BF09
:1012700010A1FF1F4B0803F1376303F5D83310B5F6
:101280000446B3FBF1F0FDF7EDFE044B1B7803B110
:1012900010BD2046BDE8104000F03EBB0094FF1F8B
:1012A00008B50846FEF7A8F8012008BD08B50846AD
:1012B000FEF7A2F8012008BD38B508460D4602F039
:1012C000FFFA044601462846FEF7EEF8204638BDF0
:1012D00010B5084614461146FEF7E6F8204610BD44
:1012E000FEF7C0B908B50846FEF766F8003018BF2B
:1012F000012008BD08B50846FEF73CF8003018BFCD
:10130000012008BD08461146FDF7CCBF0846FEF790
:1013100003B800BF0846FDF7A9BF00BFFDF744BFF3
:1013200010B54B0803F13760144600F5D830B0FB18
:10133000F1F0FDF797FE2046BDE81040FDF708BF2D
:10134000FEF778B9FEF742B9FEF730B9FEF710B9EB
:10135000FEF71AB90368064A1B68934205D110B517
:10136000C8B2FEF749F8012010BDC9B2184700BF46
:10137000AD1201000368064A1B68934205D110B5FF
:10138000C8B2FEF739F8012010BDC9B2184700BF36
:10139000AD1201000368064A1B68934205D110B5DF
:1013A000C8B2FEF729F8012010BDC9B2184700BF26
:1013B000AD1201000368064A1B68934205D110B5BF
:1013C000C8B2FEF719F8012010BDC9B2184700BF16
:1013D000AD1201004B0803F1B76303F5584310B594
:1013E0000446B3FBF1F0FEF73BFA044B1B7803B164
:1013F00010BD2046BDE8104000F08EBA0194FF1FDA
:1014000008B50846FEF76AFB012008BD08B5084686
:10141000FEF764FB012008BD38B508460D4602F012
:101420004FFA044601462846FEF762FB204638BDC7
:1014300010B5084614461146FEF75AFB204610BD6B
:10144000FEF7E6BB08B50846FEF728FB003018BFDC
:10145000012008BD08B50846FEF7FEFA003018BFA7
:10146000012008BD08461146FEF7CCBA0846FEF733
:10147000F1BA00BF0846FEF7A9BA00BFFEF76CBA82
:1014800010B54B0803F1B760144600F55840B0FBA7
:10149000F1F0FEF7E5F92046BDE81040FEF730BA5E
:1014A000FEF79EBBFEF768BBFEF756BBFEF736BBEA
:1014B000FEF740BB0368064A1B68934205D110B58E
:1014C000C8B2FEF70BFB012010BDC9B2184700BF20
:1014D0000D1401000368064A1B68934205D110B53C
:1014E000C8B2FEF7FBFA012010BDC9B2184700BF11
:1014F0000D1401000368064A1B68934205D110B51C
:10150000C8B2FEF7EBFA012010BDC9B2184700BF00
:101510000D1401000368064A1B68934205D110B5FB
:10152000C8B2FEF7DBFA012010BDC9B2184700BFF0
:101530000D140100704700BF0368F0B4FBB1002533
:1015400001249D60DC601B4C1A601C44241104F1D2
:1015500044056A11032692009E60174F0679174BC7
:1015600047F8241002F1604202F5614205F01F05C0
:10157000012000FA05F5E6541560F0BC7047104CE8
:10158000236843F40003236000BF0E4B0E4DA4F507
:101590008734A4F59E7401261E60234604609C686F
:1015A000002CD0D01033AB420360F8D1002303608D
:1015B0001846E2E7008FFCBFF093FF1F44E400E011
:1015C0003C80044000700340407103400168A9B1B1
:1015D0000B4BF0B40B441B110A4E0B4F0B4D46F84E
:1015E000237003F1440202F01F0401235211A340AF
:1015F000002445F822308C600460F0BC704700BFC6
:10160000008FFCBFF093FF1F3515010080E100E063
:10161000024A034B012111601B6818470C710340FB
:10162000F093FF1F024A034B012111605B681847CA
:101630001C710340F093FF1F024A034B012111600C
:101640009B6818472C710340F093FF1F024A034B1D
:1016500001211160DB6818473C710340F093FF1FC4
:10166000F8B50E4671B17AB10746144600253B68BD
:1016700016F8011B1B6838469847013C0544F6D113
:101680002846F8BD0846F8BD1046F8BD00B5064A24
:10169000036812885B6883B001A9ADF804200222B8
:1016A000984703B05DF804FBA46A0100F0B5074653
:1016B0008BB0002A33D0012A08BF0A2251B321245B
:1016C00000E0F4B2B1FBF2F502FB1511C8B2092932
:1016D00000F1300198BFC8B20AA988BF3730214451
:1016E00088BFC0B201F8240C661E2946002DE8D13F
:1016F00033B1013CE4B20AAB23442D2203F8242C7D
:101700003B6801AA11195B683846C4F12202984768
:101710000BB0F0BD30228DF825202124E8E70368C6
:10172000C9B21B6898470BB0F0BD00BF0029BABF13
:1017300049422D2300230A22FFF7B8BF08B5F0F76E
:1017400021FBF1F7FFFA00F009F8FAE701F014BB0A
:1017500001F01ABB704700BF704700BF2DE9F84386
:10176000314E337893B1314F3A787AB90122D907A3
:101770003A7036D49A0719D400225B073A7005D51F
:101780002B4B1A6812B1EFF305820AB1BDE8F8835A
:10179000EFF3108172B6186818B1264C2278002A2F
:1017A0002ED00029F2D162B6BDE8F883DFF8908030
:1017B00098F80020002ADFD0DFF88890002405E0A8
:1017C000013498F80030E4B2A34212D959F82450F9
:1017D0002B6828461B6998470028F1D02B69984749
:1017E000EEE7FFF7C9FCC8B9134B1B781BB9337878
:1017F000C0E73378C0E7337803F0FE033370B9E70E
:1018000045691D60012323705DB1AA6101B962B60B
:1018100000254577836898472570B7E700F092F870
:10182000E2E7064B1D60F1E70294FF1F75A3FF1F5F
:1018300070A3FF1F74A3FF1FE294FF1F6CA3FF1F81
:1018400084A3FF1F78A3FF1FF0B44D1E2E46002473
:1018500000E00134B0FBF2F302FB1300092800F1B1
:1018600030078ABF3730F8B2C0B206F8010F184609
:10187000002BEED10A1953704CB1107815F8016F96
:1018800028700133E01A834202F80169F5DB08464B
:10189000F0BC704770B584B072B6194B194D1A4838
:1018A000702241260F2480211A702E701A4604706F
:1018B000197013781B06FCD5144B186862B6144BCC
:1018C000144C984298BF00EB800001A998BF4000DB
:1018D0000A22FFF7B9FF01A92046002311F8012BC6
:1018E00001333AB10A2B20F8022FF7D116232370C7
:1018F00004B070BD5B00DBB2237004B070BD00BFEC
:1019000000000240070002400600024008000240BA
:101910007F969800CC94FF1F30B40749074C0A7893
:101920002378074D42F0020245F823000A70013384
:10193000237030BC704700BF0294FF1F84A3FF1FB9
:1019400078A3FF1F704700BF2DE9F043DFF8EC805C
:101950008BB006460F4600F073F898F9003001335B
:1019600004460D4637D03046394600F0DFF90028EE
:1019700031D02BA3D3E900233046394600F02CFEAA
:10198000814668BB28A3D3E900233046394600F0DE
:1019900005FE00B398F90030254ACDF820900424C4
:1019A00000200021022BCDE90467CDE902670094F5
:1019B0000192CDE906012CD0684600F0BDF940B394
:1019C000089B1BB101F0AAF9089B0360DDE9060141
:1019D0000BB0BDE8F083204629460BB0BDE8F0838C
:1019E000134A98F90030019203210022CDE90467DF
:1019F000CDE90267009108922BB90E4B4FF060427F
:101A0000CDE90623D8E70C490020022BCDE90601D9
:101A1000D2D101F083F922230360D1E7AFF3008034
:101A2000EF39FAFE422E864051302DD5104987C03D
:101A3000186B0100FFFFEF470000F07FE394FF1FEA
:101A40002DE9F04FB04F21F00042BA4283B00C466E
:101A50004FEAD17605460DD9AC4FBA4225D9C1F32C
:101A60001303034340F0EF800EB10020014603B0A2
:101A7000BDE8F08FA64B9A4200F2CC80A54B9A426B
:101A800000F2DE808AA3D3E9002300F063F900228C
:101A9000A14B00F0A1FD002800F005812846214659
:101AA00000229D4B00F056F9E1E783A3D3E9002320
:101AB00000F092FD002840F0CB802846214680A30C
:101AC000D3E9002300F06AFD0028CED1934B2846CD
:101AD00003EBC60821467CA3D3E9002300F0ECFA0F
:101AE000D8E9002300F036F900F080FD804600F0D0
:101AF0007DFA77A3D3E9002306460F4600F0DCFA0F
:101B000002460B462846214600F022F972A3D3E98B
:101B10000023CDE900013046394600F0CDFA824677
:101B20008B4652465B46DDE9000100F011F905469F
:101B30000C462A4623462846214600F0BDFA68A3F3
:101B4000D3E9002306460F4600F0B6FA66A3D3E9B0
:101B5000002300F0FDF832463B4600F0ADFA64A3E6
:101B6000D3E9002300F0F6F832463B4600F0A4FA31
:101B700061A3D3E9002300F0EBF832463B4600F0C6
:101B80009BFA5FA3D3E9002300F0E4F832463B461A
:101B900000F092FA02460B462846214600F0D8F89B
:101BA00006460F462846214632463B46B8F1000F0E
:101BB00056D000F081FA324604460D463B460020DE
:101BC0004FF0804100F0C4F802460B4620462946FB
:101BD00000F09CFB02460B465046594600F0B8F810
:101BE000DDE9002300F0B4F80B4602464A49002024
:101BF00000F0AEF86FF47F7398454FDA08F57A7805
:101C000001EB085100224FF0B87300F055FA03B011
